:020000041000EA
:10100000FFFFFFFFFFFFFFFFFFFFFFFFFFFFFFFFF0
:10101000FFFFFFFF00400F00FFFFFFFFFFFFFFFF8D
:10102000FFFFFFFFFFFFFFFFFFFFFFFFFFFFFFFFD0
:10103000FFFFFFFFFFFFFFFFFFFFFFFFFFFFFFFFC0
:10104000FFFFFFFFFFFFFFFFFFFFFFFFFFFFFFFFB0
:10105000FFFFFFFFFFFFFFFFFFFFFFFFFFFFFFFFA0
:10106000FFFFFFFFFFFFFFFFFFFFFFFFFFFFFFFF90
:10107000FFFFFFFFFFFFFFFFFFFFFFFFFFFFFFFF80
:10108000FFFFFFFFFFFFFFFFFFFFFFFFFFFFFFFF70
:10109000FFFFFFFFFFFFFFFFFFFFFFFFFFFFFFFF60
:1010A000FFFFFFFFFFFFFFFFFFFFFFFFFFFFFFFF50
:1010B000FFFFFFFFFFFFFFFFFFFFFFFFFFFFFFFF40
:1010C000FFFFFFFFFFFFFFFFFFFFFFFFFFFFFFFF30
:1010D000FFFFFFFFFFFFFFFFFFFFFFFFFFFFFFFF20
:1010E000FFFFFFFFFFFFFFFFFFFFFFFFFFFFFFFF10
:1010F000FFFFFFFFFFFFFFFFFFFFFFFFFFFFFFFF00
:10110000FFFFFFFFFFFFFFFFFFFFFFFFFFFFFFFFEF
:10111000FFFFFFFFFFFFFFFFFFFFFFFFFFFFFFFFDF
:10112000FFFFFFFFFFFFFFFFFFFFFFFFFFFFFFFFCF
:10113000FFFFFFFFFFFFFFFFFFFFFFFFFFFFFFFFBF
:10114000FFFFFFFFFFFFFFFFFFFFFFFFFFFFFFFFAF
:10115000FFFFFFFFFFFFFFFFFFFFFFFFFFFFFFFF9F
:10116000FFFFFFFFFFFFFFFFFFFFFFFFFFFFFFFF8F
:10117000FFFFFFFFFFFFFFFFFFFFFFFFFFFFFFFF7F
:10118000FFFFFFFFFFFFFFFFFFFFFFFFFFFFFFFF6F
:10119000FFFFFFFFFFFFFFFFFFFFFFFFFFFFFFFF5F
:1011A000FFFFFFFFFFFFFFFFFFFFFFFFFFFFFFFF4F
:1011B000FFFFFFFFFFFFFFFFFFFFFFFFFFFFFFFF3F
:1011C000FFFFFFFFFFFFFFFFFFFFFFFFFFFFFFFF2F
:1011D000FFFFFFFFFFFFFFFFFFFFFFFFFFFFFFFF1F
:1011E000FFFFFFFFFFFFFFFFFFFFFFFFFFFFFFFF0F
:1011F000FFFFFFFFFFFFFFFFFFFFFFFFFFFFFFFFFF
:101200001200000012000000FFFFFFFFFFFFFFFFC2
:10121000FFFFFFFFFFFFFFFFFFFFFFFFFFFFFFFFDE
:10122000FFFFFFFFFFFFFFFFFFFFFFFFFFFFFFFFCE
:10123000FFFFFFFFFFFFFFFFFFFFFFFFFFFFFFFFBE
:10124000FFFFFFFFFFFFFFFFFFFFFFFFFFFFFFFFAE
:020000040000FA
:1000000000040020990900002D0600007909000075
:1000100037060000410600004B060000000000000B
:10002000000000000000000000000000BD0900000A
:1000300055060000000000005F0600006906000091
:10004000730600007D060000870600009106000090
:100050009B060000A5060000AF060000B9060000E0
:10006000C3060000CD060000D7060000E106000030
:10007000EB060000F5060000FF060000090700007F
:10008000130700001D0700002707000031070000CC
:100090003B070000450700004F070000590700001C
:1000A000630700006D07000077070000810700006C
:1000B0008B070000950700009F070000A9070000BC
:1000C000B3070000BD070000C7070000D10700000C
:1000D000DB070000E5070000EF070000F90700005C
:1000E000030800000D0800001708000021080000A8
:1000F0002B080000350800003F08000049080000F8
:10010000530800001FB500F003F88DE80F001FBD75
:1001100000F038BC70B50B46010B184400F6FF70B8
:10012000040B4FF080500022090303692403406947
:1001300043431D1B104600F0E9F929462046BDE85F
:10014000704000F0E3B9F0B54FF6FF734FF4B475AB
:100150001A466E1E12E0A94201D3344600E00C4656
:10016000B1EB040130F8027B641E3B441A44F9D120
:100170009CB204EB134394B204EB12420029EAD17F
:1001800098B200EB134002EB124140EA0140F0BD8F
:10019000C34992B00446D1E90001CDE91001FF2224
:1001A0004021684600F094FB94E80F008DE80F00B2
:1001B000684610A902E004C841F8042D8842FAD12B
:1001C00010216846FFF7BFFF1090AA208DF8440069
:1001D00000F0FAF800F0DDF84FF01024A0691022CA
:1001E0006946803000F0DEF8A069082210A900F00E
:1001F000D9F800F0C2F870B504460068A94D072888
:1002000069D2DFE800F033041929561E2500D4E92D
:10021000026564682946304600F0FDF82A4621460A
:10022000304600F0BFF8AA002146304600F024FB1B
:10023000002800D0032070BD00F0D6FB4FF48050A2
:1002400007E0201D00F0C6F80028F4D100F0CCFB38
:1002500060682860002070BD241D94E807009200AB
:1002600000F00AFB0028F6D00E2070BD00F0BEF8AA
:100270000028FAD1D4E9010100EB81034FF080504E
:10028000026945696A43934209D84FF010225369C5
:1002900003EB81030169406941438B4201D9092085
:1002A00070BD5069401C01D10F2070BD2046FFF782
:1002B0006FFF00F09BF80028F7D1201D00F08AF8AE
:1002C0000028F2D160680028F0D100F07DF800F03D
:1002D00060F800F052F8072070BD10B50C461828E1
:1002E00002D00120086010BD2068FFF784FF206065
:1002F00010BD4FF01024A069401C05D0A569A66967
:1003000080353079AA2808D06069401C2DD06069FA
:100310000068401C29D060692CE010212846FFF7B6
:1003200012FF316881421CD1A16901F18002C03104
:1003300005E030B108CA51F8040D984201D10120FE
:1003400000E000208A42F4D158B1286810B1042896
:1003500003D0FEE7284600F070F85249686808604C
:1003600008E000F016F800F008F84FF4805001683B
:10037000491C01D000F012FBFEE7BFF34F8F4A4843
:1003800001684A4A01F4E06111430160BFF34F8FF5
:10039000FEE74FF010208169491C02D0806900F00F
:1003A0008CB870472DE9F04117460D4606460024EB
:1003B00006E03046296800F093F8641C2D1D361DB8
:1003C000BC42F6D3BDE8F0814FF0102080694FF4B5
:1003D00080519FE64FF080510A69496900684A439D
:1003E000824201D810207047002070474FF08050A3
:1003F0000169406941434FF01020826902F5805243
:10040000914201D2092070478069401C01D0002030
:1004100070470420704770B50C4605464FF480665F
:1004200008E0284600F049F8B44205D3A4F58064FA
:1004300005F58055002CF4D170BD4168044609B122
:10044000012600E000264FF010256869A26892009E
:1004500000F012FAF8B1A06881006869FFF75AFE4F
:10046000BEB16E694FF08050A56864680169426949
:100470005143A1420DD9016940694143A94208D9BC
:1004800029463046FFF7C7FF2A4621463046FFF788
:1004900089FFFFF772FFFFF797FFFFF77AFFF8E793
:1004A0000C0A0000000000200CED00E00400FA053A
:1004B000144801680029FCD07047134A02211160DA
:1004C00010490B68002BFCD00F4B1B1D18600868EF
:1004D0000028FCD00020106008680028FCD070477D
:1004E000094B10B501221A60064A1468002CFCD092
:1004F000016010680028FCD00020186010680028F7
:10050000FCD010BD00E4014004E5014070B50C468C
:10051000054600F073F810B900F07EF828B12146C6
:100520002846BDE8704000F007B821462846BDE8DF
:10053000704000F037B800007FB5002200920192B1
:10054000029203920A0B000B6946012302440AE05F
:10055000440900F01F0651F8245003FA06F635430B
:1005600041F82450401C8242F2D80D490868009A94
:1005700010430860081D0168019A1143016000F0F2
:100580003DF800280AD0064910310868029A104345
:100590000860091D0868039A104308607FBD0000C9
:1005A0000006004030B50F4C002200BF04EB0213E0
:1005B000D3F800582DB9D3F8045815B9D3F8085812
:1005C0001DB1521C082AF1D330BD082AFCD204EB1D
:1005D0000212C2F80008C3F804180220C3F8080881
:1005E00030BD000000E001404FF08050D0F83001F5
:1005F000082801D000207047012070474FF080503C
:10060000D0F83011062905D0D0F83001401C01D0B7
:1006100000207047012070474FF08050D0F8300123
:100620000A2801D0002070470120704708208F4918
:1006300009680958084710208C4909680958084773
:1006400014208A4909680958084718208749096809
:100650000958084730208549096809580847382053
:1006600082490968095808473C20804909680958A7
:10067000084740207D4909680958084744207B49BC
:1006800009680958084748207849096809580847FF
:100690004C20764909680958084750207349096871
:1006A00009580847542071490968095808475820D3
:1006B0006E490968095808475C206C49096809585F
:1006C0000847602069490968095808476420674954
:1006D00009680958084768206449096809580847A3
:1006E0006C20624909680958084770205F49096809
:1006F0000958084774205D49096809580847782057
:100700005A490968095808477C2058490968095816
:1007100008478020554909680958084784205349EB
:100720000968095808478820504909680958084746
:100730008C204E4909680958084790204B490968A0
:1007400009580847942049490968095808479820DA
:1007500046490968095808479C20444909680958CE
:100760000847A0204149096809580847A4203F4983
:10077000096809580847A8203C49096809580847EA
:10078000AC203A49096809580847B0203749096838
:1007900009580847B4203549096809580847B8205E
:1007A0003249096809580847BC2030490968095886
:1007B0000847C0202D49096809580847C4202B491B
:1007C000096809580847C82028490968095808478E
:1007D000CC202649096809580847D02023490968D0
:1007E00009580847D4202149096809580847D820E2
:1007F0001E49096809580847DC201C49096809583E
:100800000847E0201949096809580847E4201749B2
:10081000096809580847E820144909680958084731
:10082000EC201249096809580847F0200F49096867
:1008300009580847F4200D49096809580847F82065
:100840000A49096809580847FC20084909680958F5
:1008500008475FF480700549096809580847000097
:1008600003480449024A034B70470000000000207F
:10087000180A0000180A000040EA010310B59B079F
:100880000FD1042A0DD310C808C9121F9C42F8D0FA
:1008900020BA19BA884201D9012010BD4FF0FF30AB
:1008A00010BD1AB1D30703D0521C07E0002010BDC1
:1008B00010F8013B11F8014B1B1B07D110F8013B4D
:1008C00011F8014B1B1B01D1921EF1D1184610BD2E
:1008D00002F0FF0343EA032242EA024200F005B8B5
:1008E0007047704770474FF000020429C0F0128033
:1008F00010F0030C00F01B80CCF1040CBCF1020FD3
:1009000018BF00F8012BA8BF20F8022BA1EB0C01A7
:1009100000F00DB85FEAC17C24BF00F8012B00F89D
:10092000012B48BF00F8012B70474FF0000200B5C3
:10093000134694469646203922BFA0E80C50A0E802
:100940000C50B1F12001BFF4F7AF090728BFA0E8B0
:100950000C5048BF0CC05DF804EB890028BF40F87C
:10096000042B08BF704748BF20F8022B11F0804FBE
:1009700018BF00F8012B7047014B1B68DB68184754
:100980000000002009480A497047FFF7FBFFFFF706
:10099000B9FB00BD20BFFDE7064B1847064A1060B3
:1009A000016881F30888406800470000180A0000C9
:1009B000180A0000F3020000000000201EF0040FDF
:1009C0000CBFEFF30881EFF30981886902380078E2
:1009D000182803D100E00000074A1047074A1268B0
:1009E0002C3212681047000000B5054B1B68054A01
:1009F0009B58984700BD0000DB020000000000206B
:100A0000080A0000040000000010000000000000C0
:100A100000FFFFFF0090D003FFFFFFFFFFFFFFFF7E
:100A2000FFFFFFFFFFFFFFFFFFFFFFFFFFFFFFFFD6
:100A3000FFFFFFFFFFFFFFFFFFFFFFFFFFFFFFFFC6
:100A4000FFFFFFFFFFFFFFFFFFFFFFFFFFFFFFFFB6
:100A5000FFFFFFFFFFFFFFFFFFFFFFFFFFFFFFFFA6
:020000040000fa
:10100000c8130020415f020075c10000a75e020006
:1010100075c1000075c1000075c10000000000002e
:10102000000000000000000000000000cd5f020092
:1010300075c100000000000075c1000075c100000e
:10104000356002003b60020075c1000075c1000000
:1010500075c1000075c1000075c1000075c10000b8
:101060004160020075c1000075c1000047600200c8
:1010700075c100004d60020053600200596002001b
:1010800075c1000075c1000075c1000075c1000088
:1010900075c1000075c1000075c1000075c1000078
:1010a00075c100005f60020075c1000075c10000dd
:1010b00075c1000075c1000075c1000075c1000058
:1010c0006560020075c1000075c1000075c10000b7
:1010d00075c1000075c1000075c1000075c1000038
:1010e00075c1000075c1000075c1000075c1000028
:1010f00075c1000075c1000075c1000075c1000018
:1011000075c1000075c1000000f002f824f007ff6f
:101110000aa090e8000c82448344aaf10107da4552
:1011200001d124f0fcfeaff2090ebae80f0013f073
:10113000010f18bffb1a43f00103184708540200bf
:10114000285402000a444ff0000c10f8013b13f041
:10115000070408bf10f8014b1d1108bf10f8015b10
:10116000641e05d010f8016b641e01f8016bf9d103
:1011700013f0080f1ebf10f8014bad1c0c1b09d15a
:101180006d1e58bf01f801cbfad505e014f8016bcc
:1011900001f8016b6d1ef9d59142d6d3704700005e
:1011a0000023002400250026103a28bf78c1fbd870
:1011b000520728bf30c148bf0b6070471fb500f011
:1011c00003f88de80f001fbd24f0a6be70b51a4cc1
:1011d00005460a202070a01c00f0d5f85920a080f8
:1011e00029462046bde8704008f09ab908f0a3b936
:1011f00070b50c461149097829b1a0f160015e294a
:1012000008d3012013e0602804d0692802d043f2fb
:1012100001000ce020cc0a4e94e80e0006eb8000a2
:10122000a0f58050241fd0f8806e2846b04720607b
:1012300070bd012070470000080000201800002049
:10124000b06002003249884201d20120704700207c
:10125000704770b50446a0f500002e4eb0f1786fcf
:1012600002d23444a4f500042948844201d2012565
:1012700000e0002500f043f848b125b9b44204d39a
:101280002548006808e0012070bd002070bd002dd9
:10129000f9d1b442f9d321488442f6d2f3e710b52c
:1012a0000446a0f50000b0f1786f03d21948044459
:1012b000a4f5000400f023f84ff0804130b1164847
:1012c000006804e08c4204d2012003e01348844209
:1012d000f8d2002080f0010010bd10b520b1fff75a
:1012e000deff08b1012010bd002010bd10b520b1f7
:1012f000fff7afff08b1012010bd002010bd084866
:1013000008490068884201d10120704700207047d9
:1013100000700200000000201c00002008000020d7
:1013200058000020bebafeca10b5044600210120b4
:1013300000f041f800210b2000f03df800210820ca
:1013400000f039f80421192000f035f804210d20af
:1013500000f031f804210e2000f02df804210f20b8
:1013600000f029f80421c84300f025f806211620d2
:1013700000f021f80621152000f01df82046fff7a7
:1013800025ff002010bdca2101807047fff72ebf46
:101390001148704710487047104a10b514680f4b39
:1013a0000f4a08331a60fff723ff0c48001d046042
:1013b00010bd704770474907090e002804db00f193
:1013c000e02080f80014704700f00f0000f1e020ea
:1013d00080f8141d7047000003f900421005024018
:1013e00001000001fd48002101604160018170475a
:1013f0002de9ff4f93b09b46209f160004460dd069
:101400001046fff726ff18b1102017b0bde8f08f87
:101410003146012001f0d3fe0028f6d101258df8d8
:1014200042504ff4c050adf84000002210a92846a9
:1014300006f0d8fc0028e8d18df84250a8464ff4b9
:1014400028500025adf840001c2229466846079523
:101450000df015f89df81c000df11c0a20f00f008e
:10146000401c20f0f00010308df81c0020788df822
:101470001d0061789df81e000df1400961f34200e6
:1014800040f001008df81e009df8000008aa40f011
:1014900002008df800002089adf83000adf8325020
:1014a0006089adf83400cdf82ca060680e900aa9d0
:1014b000cdf82890684606f08afa0028a5d1606821
:1014c000fff70bff40b16068fff710ff20b96078ad
:1014d00000f00300022801d0012000e00020bf4cf2
:1014e00008aa0aa92072bdf8200020808df8428049
:1014f00042f60120adf840009df81e0020f00600e5
:10150000801c20f001008df81e000220adf8300094
:10151000adf8340014a80e90684606f058fa00287a
:1015200089d1bdf82000608036b1211d304600f021
:101530005ff90028c2d109e0bbf1000f05d00cf023
:1015400019fde8bb0cf016fdd0bba58017b1012f2b
:1015500043d04ae08df8428042f6a620adf8400024
:1015600046461c220021684607950cf088ff9df82e
:101570001c00adf8346020f00f00401c20f0f0009b
:1015800010308df81c009df81d0020f0ff008df834
:101590001d009df81e0020f0060040f00100801c98
:1015a0008df81e009df800008df8446040f00200a8
:1015b0008df80000cde90a9aadf8306011a800e07e
:1015c00011e00e9008aa0aa9684606f000fa002861
:1015d000a6d1bdf82000e08008e00cf0cbfc10b9eb
:1015e0000cf0c8fc08b103200fe7e58000200ce7f1
:1015f0003eb50446794d0820adf80000a88828b112
:101600002046fff726fe18b110203ebd06203ebd45
:101610002146012001f0d3fd0028f8d12088adf843
:1016200004006088adf80600a088adf80800e088e6
:10163000adf80a00a88801ab6a46002106f0cefd8d
:10164000bdf800100829e2d003203ebd7fb5634df0
:101650000446a88868b1002002900820adf8080070
:10166000cdf80cd02046fff7f4fd20b1102004b0d7
:1016700070bd0620fbe7a98802aa4ff6ff7006f0ae
:10168000efff0028f3d1bdf80810082901d003208e
:10169000ede7bdf800102180bdf802106180bdf8b3
:1016a0000410a180bdf80610e180e0e701b582b02a
:1016b0000220adf80000494802ab6a46408800218c
:1016c00006f08cfdbdf80010022900d003200ebded
:1016d0001cb5002100910221adf800100190fff728
:1016e000defd08b110201cbd3c486a4641884ff61b
:1016f000ff7006f0b5ffbdf800100229f3d00320fb
:101700001cbdfeb5354c06461546207a0f46c0076f
:1017100005d00846fff79dfd18b11020febd0f2033
:10172000febdf82d01d90c20febd3046fff791fd1e
:1017300018bb208801a905f04cfe0028f4d13078b0
:101740008df80500208801a906f026fd0028ebd1c0
:1017500000909df800009df8051040f002008df803
:101760000000090703d040f008008df80000208831
:10177000694606f0aefc0028d6d1adf808502088a6
:101780003b4602aa002106f029fdbdf80810a94237
:10179000cad00320febd7cb5054600200090019014
:1017a0000888adf800000c4628460195fff795fd26
:1017b00018b92046fff773fd08b110207cbd15b1a4
:1017c000bdf8000060b105486a4601884ff6ff7019
:1017d00006f046ffbdf8001021807cbd28020020e5
:1017e0000c20fae72f48c088002800d0012070475d
:1017f00030b5044693b000200d46014600901422f7
:1018000001a80cf03cfe1c22002108a80cf037feb9
:101810009df80000cdf808d020f00f00401c20f00b
:10182000f00010308df800009df8010006aa20f0ad
:10183000ff008df801009df8200001a940f0020092
:101840008df8200001208df8460042f60420adf806
:10185000440011a801902088adf83c006088adf8e4
:101860003e00a088adf84000e088adf842009df849
:10187000020020f00600801c20f001008df802001c
:101880000820adf80c00adf810000fa8059008a8ce
:1018900006f09df8002803d1bdf81800288000202c
:1018a00013b030bd28020020f0b5007b059f1e4616
:1018b00014460d46012800d0ffdf0c2030803a206e
:1018c0003880002c08d0287a032806d0287b0128ed
:1018d00000d0ffdf17206081f0bda889fbe72de96c
:1018e000f04786b0144691f80c900e9a0d46b9f167
:1018f000010f0bd01021007b2e8a8846052807d0c7
:10190000062833d0ffdf06b0bde8f0870221f2e7fa
:10191000e8890c2100eb400001eb400018803320e7
:101920001080002cefd0e889608100271ae0009633
:10193000688808f1020301aa696900f086ff06ebd6
:101940000800801c07eb470186b204eb4102bdf89a
:10195000040090810df1060140460e3213f096f816
:101960007f1cbfb26089b842e1d8cce73420108038
:10197000e889b9f1010f11d0122148430e301880c7
:10198000002cc0d0e88960814846b9f1010f00d031
:101990000220207300270df1040a1fe00621ece766
:1019a0000096688808f1020301aa696900f04dfffa
:1019b00006eb0800801c86b2b9f1010f12d007ebcc
:1019c000c70004eb4000bdf80410c18110220af1e9
:1019d000020110300cf029fd7f1cbfb26089b842b3
:1019e000ded890e707eb470104eb4102bdf80400a5
:1019f000d0810af102014046103213f047f8ebe7bc
:101a00002de9f0470e4688b090f80cc096f80c808f
:101a1000378af5890c20109902f10c044ff0000a66
:101a2000bcf1030f08d0bcf1040f3fd0bcf1070f8d
:101a30007ed0ffdf08b067e705eb850c00eb4c00bc
:101a4000188031200880002af4d0a8f1060000f0a8
:101a5000ff09558126e01622002101a80cf00ffd98
:101a600000977088434601aa716900f0eefebdf848
:101a700004002080bdf80600e080bdf80800208149
:101a8000a21c0df10a01484613f000f8b9f1000f4d
:101a900000d018b184f804a0a4f802a007eb080055
:101aa00087b20a346d1eadb2d5d2c3e705eb850c03
:101ab00000eb4c00188032200880002abad0a8f130
:101ac000050000f0ff09558137e000977088434614
:101ad00001aa716900f0b9fe9df80600bdf8041076
:101ae000e1802179420860f3000162f3410182083c
:101af00062f38201c20862f3c301020962f30411b6
:101b0000420962f34511820962f386112171c0090d
:101b10006071bdf80700208122460df10901484699
:101b200012f0b4ff18b184f802a0a4f800a000e0fd
:101b300007e007eb080087b20a346d1eadb2c4d2cd
:101b400078e7a8f1020084b205fb08f000f10e0c62
:101b5000a3f800c035230b80002aa6d055819481bc
:101b6000009783b270880e32716900f06efe61e7f3
:101b70002de9f84f1e460a9d0c4681462ab1607a2f
:101b800000f58070d080e089108199f80c000c2756
:101b90004ff000084ff00e0a0d2872d2dfe800f077
:101ba0009d070e1b272f374554697272720021461c
:101bb00048460095fff778febde8f88f207b9146f8
:101bc000082802d0032800d0ffdf3780302009e04a
:101bd000a9f80a80f0e7207b9146042800d0ffdfb7
:101be000378031202880b9f1000ff1d1e4e7207b64
:101bf0009146042800d0ffdf37803220f2e7207bb7
:101c00009146022800d0ffdf37803320eae7207baf
:101c10001746022800d0ffdf3420a6f800a0288055
:101c2000002fc9d0a7f80a80c6e7207b17460428f2
:101c300000d0ffdf3520a6f800a02880002fbbd001
:101c40004046a7f80a8012e0207b1746052802d0fc
:101c5000062800d0ffdf1020308036202880002f9b
:101c6000aad0e0897881a7f80e80b9f80e00b88173
:101c7000a2e7207b9146072800d0ffdf378037207e
:101c8000b0e72ae04ff0120018804ff0380017003c
:101c9000288091d0e0897881a7f80e80a7f810807d
:101ca00099f80c000a2805d00b2809d00c280dd073
:101cb000ffdf81e7207b0a2800d0ffdf01200ae058
:101cc000207b0b2800d0ffdf042004e0207b0c28c1
:101cd00000d0ffdf052038736ee7ffdf6ce770b5db
:101ce0000c46054601f0affb20b10078222804d253
:101cf000082070bd43f2020070bd0521284611f096
:101d00002df9206008b1002070bd032070bd30b4f3
:101d10004880087820f00f00c01c20f0f0009030c0
:101d200001f8080b1dca81e81d0030bc07f079bc22
:101d30002de9ff4784b00027824602970798904616
:101d4000894612300af067fa401d20f00306079812
:101d500028b907a95046fff7c2ff002854d1b9f1ae
:101d6000000f05d00798017b19bb052504681be00f
:101d700098f80000092803d00d2812d0ffdf46e0b4
:101d8000079903254868b0b3497b42887143914263
:101d900039d98ab2b3b2011d10f053ff044607804f
:101da00002e0079c042508340cb1208810b1032df3
:101db00029d02ce00798012112300af05efaadf824
:101dc0000c00024602ab2946504608f0b6fa07005e
:101dd00001d1a01c029007983a461230c8f80400be
:101de000a8f802a003a94046029b0af053fad8b112
:101df0000a2817d200e006e0dfe800f00709141413
:101e0000100b0d141412132014e6002012e61120fa
:101e100010e608200ee643f203000be6072009e671
:101e20000d2007e6032005e6bdf80c002346cde9aa
:101e300000702a465046079900f017fd57b9032d48
:101e400008d10798b3b2417b406871438ab2011d43
:101e500010f00bffb9f1000fd7d0079981f80c9063
:101e6000d3e72de9fe4f91461a881c468a468046e4
:101e7000fab102ab494608f060fa050019d04046b5
:101e8000a61c278811f0aff93246072629463b46a3
:101e9000009610f0bcfd20882346cde900504a464c
:101ea0005146404600f0e1fc002020800120bde8c2
:101eb000fe8f0020fbe710b586b01c46aab10423b4
:101ec0008df800301388adf808305288adf80a203c
:101ed0008a788df80e200988adf80c1000236a4628
:101ee0002146fff725ff06b010bd1020fbe770b5b7
:101ef0000d46052111f032f8040000d1ffdf29461c
:101f000004f11200bde870400af0a0b92de9f843d1
:101f10000d468046002607f081fb044628781028ed
:101f200078d2dfe800f0773b345331311231313170
:101f30000831313131312879001fc0b2022801d077
:101f4000102810d114bbffdf35e004b9ffdf0521f5
:101f5000404611f003f8007b032806d004280bd07c
:101f6000072828d0ffdf072655e02879801fc0b258
:101f7000022820d050b1f6e72879401fc0b20228cd
:101f800019d0102817d0eee704b9ffdf13e004b929
:101f9000ffdf287901280ed1172137e005214046bf
:101fa00010f0dcff070000d1ffdf07f1120140460f
:101fb0000af029f92cb12a4621464046fff7a7fe30
:101fc00029e01321404602f025fd24e004b9ffdf9b
:101fd0000521404610f0c2ff060000d1ffdf694630
:101fe00006f112000af019f9060000d0ffdfa988f7
:101ff000172901d2172200e00a46bdf800008242ec
:1020000002d9014602e005e01729c5d3404600f099
:102010003cfcd0e7ffdf3046bde8f883401d20f0f0
:10202000030219b102fb01f0001d00e00020104482
:10203000704713b5009848b10024684610f0abfd16
:10204000002c02d1f74a009911601cbd0124002028
:10205000f4e72de9f0470c461546242200212046de
:102060000cf00dfa05b9ffdfa87860732888dff857
:10207000b4a3401d20f00301af788946daf80000d0
:1020800010f0a7fd060000d1ffdf4ff0000826602a
:10209000a6f8008077b109fb07f1091d0ad0daf82c
:1020a000000010f096fd060000d1ffdf6660c6f864
:1020b000008001e0c4f80480298804f11200bde822
:1020c000f0470af091b82de9f047804601f112007f
:1020d0000d4681460af09ff8401dd24f20f00302c2
:1020e0006e7b14462968386810f09efd3eb104fbf3
:1020f00006f2121d03d06968386810f095fd0520be
:1021000010f0d4fe0446052010f0d8fe201a012855
:1021100002d1386810f052fd49464046bde8f0470c
:102120000af078b870b50546052110f017ff0400d5
:1021300000d1ffdf04f112012846bde870400af02b
:1021400062b82de9f04f91b04ff0000badf834b00c
:10215000adf804b047880c4605469246052138463e
:1021600010f0fcfe060000d1ffdf24b1a780a4f828
:1021700006b0a4f808b0297809220b20b2eb111f91
:102180007ed12a7a04f1100138274ff00c084ff065
:1021900001090391102a74d2dfe802f073f3f2f11f
:1021a0008008d3898ea03ddcf4efb7b7307b0228de
:1021b00000d0ffdfa88908ebc001adf80410302182
:1021c000adf83410002c25d06081b5f80e900027b2
:1021d0001de004ebc708317c88f80e10f189a8f8df
:1021e0000c10cdf800906888042304aa296900f037
:1021f0002cfbbdf81010a8f8101009f10400bdf870
:1022000012107f1c1ffa80f9a8f81210bfb2608963
:10221000b842ded80ee1307b022800d0ffdfe9892a
:1022200008ebc100adf804003020adf83400287b85
:102230000a90001fc0b20f90002cebd06181b5f85e
:102240001090002726e000bfcdf8009068886969eb
:1022500003aa0a9b00f0f9fa0a9804ebc70848445d
:102260001ffa80f908f10c0204a90f9812f00efc75
:1022700018b188f80eb0a8f80cb0bdf80c1001e049
:10228000d4e0d1e0a8f81010bdf80e107f1ca8f81b
:102290001210bfb26089b842d6d8cbe00da800902a
:1022a00001ab224629463046fff719fbc2e0307bde
:1022b000082805d0ffdf03e0307b082800d0ffdfcf
:1022c000e8891030adf804003620adf83400002c59
:1022d0003fd0a9896181f189a18127e0307b09285c
:1022e00000d0ffdfa88900f10c01adf80410372100
:1022f000adf83410002c2cd06081e8890090ab89b7
:10230000688804f10c02296956e0e8893921103007
:1023100080b2adf80400adf83410002c74d0a98957
:102320006181287a0e280ad002212173e989e1818e
:10233000288a0090eb8968886969039a3ce001214a
:10234000f3e70da8009001ab224629463046fff77f
:1023500057fb6fe0307b0a2800d0ffdf1220adf87a
:102360000400adf834704cb3a9896181a4f810b0b1
:10237000a4f80eb084f80c905ce020e002e031e0bc
:1023800039e042e0307b0b2800d0ffdf288aadf82f
:1023900034701230adf8040084b104212173a9898e
:1023a0006181e989e181298a2182688a00902b8aea
:1023b000688804f11202696900f047fa3ae0307b5c
:1023c0000c2800d0ffdf1220adf80400adf8347007
:1023d0003cb305212173a4f80ab0a4f80eb0a4f808
:1023e00010b027e00da8009001ab224629463046e8
:1023f000fff75afa1ee00da8009001ab22462946cd
:102400003046fff7b5fb15e034e03b21adf80400a2
:10241000adf8341074b3a4f80690a4f808b084f8aa
:102420000ab007e010000020ffdf03e0297a01294d
:1024300017d0ffdfbdf80400aaf800006cb1bdf8aa
:1024400034002080bdf804006080bdf834003928d5
:1024500003d03c2801d086f80cb011b00020bde8b4
:10246000f08f3c21adf80400adf8341014b1697a56
:10247000a172dfe7aaf80000efe72de9f8435688dc
:102480000f46804615460521304610f067fd0400d2
:1024900000d1ffdf123400943b46414630466a6863
:1024a0000af02cf8b8e570b50d46052110f056fd80
:1024b000040000d1ffdf294604f11200bde870409e
:1024c00009f0b6be70b50d46052110f047fd0400b9
:1024d00000d1ffdf294604f11200bde8704009f089
:1024e000d4be70b50546052110f038fd040000d1ba
:1024f000ffdf04f1080321462846bde870400422ae
:10250000afe470b50546052110f028fd040000d1a8
:10251000ffdf214628462368bde870400522a0e47d
:1025200070b50646052110f019fd040000d1ffdf4b
:1025300004f1120009f06ffe401d20f0030511e0c8
:10254000011d00880322431821463046fff789fc0d
:1025500000280bd0607babb2684382b26068011d7b
:1025600010f0b9fb606841880029e9d170bd70b5f1
:102570000e46054607f052f8040000d1ffdf0120a7
:10258000207266726580207820f00f00c01c20f059
:10259000f00030302070bde8704007f042b82de9ff
:1025a000f0438bb00d461446814606a9fff797fb12
:1025b000002814d14ff6ff7601274ff420588cb134
:1025c00003208df800001020adf8100007a805903a
:1025d00007aa204604a912f078fa78b107200bb0b8
:1025e000bde8f0830820adf808508df80e708df826
:1025f0000000adf80a60adf80c800ce00698a178f8
:1026000001742188c1818df80e70adf80850adf8c5
:102610000c80adf80a606a4602214846069bfff727
:1026200087fbdce708b501228df8022042f60202a2
:10263000adf800200a4603236946fff73cfc08bdbd
:1026400008b501228df8022042f60302adf8002001
:102650000a4604236946fff72efc08bd00b587b083
:1026600079b102228df800200a88adf80820498847
:10267000adf80a1000236a460521fff759fb07b0a1
:1026800000bd1020fbe709b1072314e407207047c1
:1026900070b588b00d461446064606a9fff71ffb25
:1026a00000280ed17cb10620adf808508df800004e
:1026b000adf80a40069b6a460821dc813046fff7e8
:1026c00037fb08b070bd05208df80000adf808504c
:1026d000f0e700b587b059b107238df80030adf8a9
:1026e0000820039100236a460921fff721fbc6e772
:1026f0001020c4e770b588b00c460646002506a930
:10270000fff7edfa0028dcd106980121123009f01c
:10271000b4fd9cb12178062921d2dfe801f0200523
:1027200005160318801e80b2c01ee28880b20ab16e
:10273000a3681bb1824203d90c20c2e71020c0e776
:10274000042904d0a08850b901e00620b9e7012986
:1027500013d0022905d004291cd005292ad007202e
:10276000afe709208df800006088adf80800e08828
:10277000adf80a00a068039023e00a208df800005d
:102780006088adf80800e088adf80a00a0680a2566
:10279000039016e00b208df800006088adf808006b
:1027a000a088adf80a00e088adf80c00a0680b2501
:1027b000049006e00c208df8000060788df8080089
:1027c0000c256a4629463046069bfff7b1fa78e7a2
:1027d00000b587b00d228df80020adf80810002359
:1027e0006a461946fff7a4fa49e700b587b071b108
:1027f00002228df800200a88adf808204988adf83b
:102800000a1000236a460621fff792fa37e71020e4
:1028100035e770b586b0064601200d46adf80810c4
:102820008df80000014600236a463046fff780fa23
:10283000040008d12946304605f0eafc0021304664
:1028400005f004fd204606b070bdf8b51c461546df
:102850000e46069f10f0b5fc2346ff1dbcb2314664
:102860002a46009410f09ff8f8bd30b41146dde917
:1028700002423cb1032903d0002330bc08f03bbe28
:102880000123fae71a8030bc704770b50c46054644
:10289000fff72dfb2146284605f0c9fc2846bde878
:1028a0007040012105f0d2bc4ff0e0224ff400400f
:1028b0000021c2f88001bff34f8fbff36f8f17481d
:1028c000016001601649900208607047134900b525
:1028d00000220a600a60124b4ff060721a600028f2
:1028e00008bf00bd0f4a104bdff840c001280cd0d4
:1028f00002281cbfffdf00bd032008601a604ff4f0
:10290000000000bfccf8000000bd022008601a6083
:102910004ff04070f6e700b5ffdf00bd00f5004066
:1029200008f50140a802002014f5004004f501401c
:1029300070b50b2000f0bdf9082000f0baf90021b5
:102940000b2000f0d4f90021082000f0d0f9f44c5d
:1029500001256560a5600020c4f84001c4f8440169
:10296000c4f848010b2000f0b5f9082000f0b2f9d6
:102970000b2000f091f9256070bd10b50b2000f020
:1029800098f9082000f095f9e5480121416081603f
:10299000e4490a68002afcd10021c0f84011c0f8bf
:1029a0004411c0f848110b2000f094f9bde8104024
:1029b000082000f08fb910b50b2000f08bf9bde8ae
:1029c0001040082000f086b900b530b1012806d0cb
:1029d000022806d0ffdf002000bdd34800bdd34849
:1029e00000bdd248001d00bd70b5d1494ff0004078
:1029f0000860d04dc00bc5f80803cf480024046020
:102a0000c5f840410820c43500f053f9c5f83c41f1
:102a1000ca48047070bd08b5c14a002128b1012818
:102a200011d002281cd0ffdf08bd4ff48030c2f85f
:102a30000803c2f84803bb483c300160c2f84011ab
:102a4000bde80840d0e74ff40030c2f80803c2f8f0
:102a50004803b44840300160c2f84411b3480ce068
:102a60004ff48020c2f80803c2f84803ad48443050
:102a70000160c2f84811ad48001d0068009008bd13
:102a800070b516460d460446022800d9ffdf002225
:102a9000a348012304f110018b4000eb8401c1f82d
:102aa000405526b1c1f84021c0f8043303e0c0f816
:102ab0000833c1f84021c0f8443370bd2de9f0411e
:102ac0001d46144630b1012833d0022838d0ffdf2c
:102ad000bde8f081891e002221f07f411046fff7fa
:102ae000cfff012d23d00020944d924f0126687016
:102af0003e61914900203c3908600220091d0860b0
:102b00008d490420303908608b483d34046008202a
:102b10006c6000f0dff83004c7f80403082000f010
:102b2000bbf88349f007091f08602e70d0e7012029
:102b3000dae7012b02d00022012005e00122fbe7a9
:102b4000012b04d000220220bde8f04198e70122c9
:102b5000f9e774480068704770b500f0d8f8704c19
:102b60000546d4f840010026012809d1d4f808030d
:102b7000c00305d54ff48030c4f80803c4f84061a1
:102b8000d4f8440101280cd1d4f80803800308d5f7
:102b90004ff40030c4f80803c4f84461012012f077
:102ba0005bffd4f8480101280cd1d4f80803400396
:102bb00008d54ff48020c4f80803c4f84861022007
:102bc00012f04aff5e48056070bd70b500f09ff8d6
:102bd0005a4d0446287850b1fff706ff687818b1bf
:102be0000020687012f038ff5548046070bd032063
:102bf000f8e74ff0e0214ff40010c1f800027047f1
:102c0000152000f067b84b4901200861082000f04a
:102c100061b848494ff47c10c1f80803002002460f
:102c200001eb8003c3f84025c3f84021401cc0b22b
:102c30000628f5d37047410a43f609525143c0f3c1
:102c4000080010fb02f000f5807001eb5020704787
:102c500010b5430b48f2376463431b0c5c020c60f5
:102c6000384c03fb0400384b4cf2f72443435b0d14
:102c700013fb04f404eb402000f580704012107048
:102c800008681844086010bd2c48406870472949fe
:102c90000120c1f800027047002809db00f01f0284
:102ca000012191404009800000f1e020c0f80011ae
:102cb000704700280ddb00f01f0201219140400900
:102cc000800000f1e020c0f88011bff34f8fbff308
:102cd0006f8f7047002809db00f01f02012191402f
:102ce0004009800000f1e020c0f8801270474907d9
:102cf000090e002804db00f1e02080f80014704782
:102d000000f00f0000f1e02080f8141d70470c481f
:102d1000001f00680a4a0d49121d1160704700002b
:102d200000b0004004b500404081004044b1004084
:102d300008f5014000800040408500403800002038
:102d400014050240f7c2ffff6f0c010001000001f3
:102d50000a4810b50468094909480831086012f0aa
:102d60000fff0648001d046010bd064900200860e2
:102d70004ff0e0210220c1f88002704710050240a8
:102d800001000001fc1f0040374901200860704726
:102d900070b50d2000f049f8344c0020c4f8000153
:102da0000125c4f804530d2000f050f825604ff0c1
:102db000e0216014c1f8000170bd10b50d2000f0d5
:102dc00034f82a48012141600021c0f80011bde813
:102dd00010400d2000f03ab8254810b50468244989
:102de0002448083108602149d1f80001012804d0a5
:102df000ffdf1f48001d046010bd1b48001d006858
:102e00000022c0b2c1f8002113f0e1fbf1e710b5d8
:102e1000164800bfd0f800110029fbd0fff7dcfff7
:102e2000bde810400d2000f011b800280ddb00f0c7
:102e30001f02012191404009800000f1e020c0f80c
:102e40008011bff34f8fbff36f8f7047002809dbee
:102e500000f01f02012191404009800000f1e020b4
:102e6000c0f880127047000004d5004000d0004038
:102e700010050240010000014ff0e0214ff000700a
:102e8000c1f8800101f5c071bff34f8fbff36f8fa1
:102e9000c1f80001394b802283f8002441f8800cee
:102ea000704700b502460420354903e001ebc0033a
:102eb0001b792bb1401ec0b2f8d2ffdfff2000bd4e
:102ec00041f8302001ebc00100224a718a710122d1
:102ed0000a7100bd2a4a002102ebc000017170474f
:102ee00010b50446042800d3ffdf254800ebc404d6
:102ef0002079012800d0ffdf6079a179401cc0b2a1
:102f0000814200d060714ff0e0214ff00070c1f8b5
:102f1000000210bd70b50425194e1a4c16e0217838
:102f200006ebc1000279012a08d1427983799a42dd
:102f300004d04279827156f8310080472078401cd5
:102f4000c0b22070042801d3002020706d1eedb2a5
:102f5000e5d270bd0c4810b504680b490b48083128
:102f60000860064890f800044009042800d0ffdffc
:102f7000fff7d0ff0448001d046010bd19e000e019
:102f8000e00500205400002010050240010000016f
:102f90000548064a0168914201d1002101600449b7
:102fa000012008607047000058000020bebafeca29
:102fb00040e5014070b50c46054609f03bfc214652
:102fc0002846bde870400af01cbd70477047704746
:102fd0001ef0040f0cbfeff30880eff30980014ae5
:102fe000104700009b6c01000ff20c0000f1000084
:102ff000694641f8080c20bf704700000004050630
:103000002cffffffdbe5b15100700200ca00ffff9b
:103010008c000000c1cf6a00fea0d9111c1006c3ad
:1030200089ccfc7a7b3b49141906a8c030b5f84d11
:103030000446062ca9780ed2dfe804f0030e0e0e2b
:103040000509ffdf08e0022906d0ffdf04e00329bd
:1030500002d0ffdf00e0ffdfac7030bd30b50446ca
:103060001038eb4d07280cd2dfe800f0040c060cfa
:103070000c0c0c00ffdf05e0287e112802d0ffdfda
:1030800000e0ffdf2c7630bd2de9f04111f088fe25
:10309000044613f0bbf8201ac5b206200ff006ff55
:1030a000044606200ff00aff211ad94c207e122870
:1030b00018d000200f1807200ff0f8fe0646072052
:1030c0000ff0fcfe301a3918207e13280cd0002097
:1030d0000144a078042809d000200844281ac0b26e
:1030e000bde8f0810120e5e70120f1e70120f4e7e8
:1030f000c74810b590f825004108c54800f12600e2
:1031000005d00df05bffbde8104006f0a9b80df04a
:1031100036fff8e730b50446a1f120000d460a2835
:103120004ad2dfe800f005070c1c2328353a3f445b
:10313000ffdf42e0207820283fd1ffdf3de0b448a8
:103140008178052939d0007e122836d020782428ad
:1031500033d0252831d023282fd0ffdf2de0207851
:1031600022282ad0232828d8ffdf26e0207822280a
:1031700023d0ffdf21e0207822281ed024281cd075
:1031800026281ad0272818d0292816d0ffdf14e0c7
:103190002078252811d0ffdf0fe0207825280cd0db
:1031a000ffdf0ae02078252807d0ffdf05e0207840
:1031b000282802d0ffdf00e0ffdf257030bd1fb5fb
:1031c00004466a46002001f0a5feb4b1bdf8022015
:1031d0004ff6ff700621824201d1adf80210bdf812
:1031e0000420824201d1adf80410bdf808108142dc
:1031f00003d14ff44860adf8080068460ef048fb74
:1032000006f02ef804b010bd70b514460d46064603
:10321000fef71ff858b90db1a54201d90c2070bdb9
:10322000002408e056f82400fef713f808b1102037
:1032300070bd641ce4b2ac42f4d3002070bd2de933
:10324000f04105461f4690460e4600240068fef7f2
:103250004df830b9a98828680844401efef746f8a2
:1032600008b110203ce728680028a88802d0b8429e
:1032700002d850e00028f5d0092031e72968085d20
:10328000b8b1671cca5d152a2ed03cdc152a3ad28b
:10329000dfe802f03912222228282a2a313139396e
:1032a00039393939393939392200085d30bb641c64
:1032b000a4b2a242f9d833e00228ddd1a01c085cf8
:1032c00088f80000072801d2400701d40a2007e748
:1032d000307840f0010015e0c143c90707e001283c
:1032e00007d010e00620fbe60107a1f1805100297c
:1032f000f5d01846f4e63078810701d50b20efe6cb
:1033000040f0020030702868005d384484b2a8881c
:10331000a04202d2b0e74ff4485382b2a242add8e5
:103320000020dde610b5027843f2022354080122a2
:10333000022c12d003dc3cb1012c16d106e0032c88
:1033400010d07f2c11d112e0002011e080790324ed
:10335000b4eb901f09d10a700be08079b2eb901f9b
:1033600003d1f8e780798009f5d0184610bdff2019
:103370000870002010bd08b500208df8000024481a
:1033800090f82e1049b190f82f0002280ed0032893
:103390000ed0ffdf9df8000008bd1d4869462530ae
:1033a00001f007fe0028f5d0ffdff3e7032000e07f
:1033b00001208df80000ede738b50c46054669465a
:1033c00001f0f7fd00280dd19df80010207861f381
:1033d0004700207055f8010fc4f80100a888a4f830
:1033e0000500002038bd38b51378a8b1022813d0e5
:1033f000ff281ad007a46d46246800944c7905eb89
:103400009414247864f347031370032809d00fe061
:10341000f40100200302ff0123f0fe0313700228d1
:10342000f3d1d8b240f0010005e043f0fe00107087
:10343000107820f0010010700868c2f80100888838
:10344000a2f8050038bd02210ff088bd38b50c4642
:103450000978222901d2082038bdadf800008df886
:10346000022068460df0ecfd05f0fafe050003d1e0
:1034700021212046fff74efe284638bd1cb500200e
:103480008df80000cdf80100adf80500fb4890f87c
:103490002e00022801d0012000e000208df8070056
:1034a00068460df055fe002800d0ffdf1cbd00224d
:1034b0000a80437892b263f3451222f040020a80f8
:1034c00000780c282bd2dfe800f02a06090e11162e
:1034d000191c1f220c2742f0110009e042f01d00c8
:1034e00008800020704742f0110012e042f0100006
:1034f00040f00200f4e742f01000f1e742f0010072
:10350000eee742f0010004e042f00200e8e742f09a
:10351000020040f00400e3e742f00400e0e7072087
:1035200070472de9ff478ab00025bdf82c60824620
:103530001c4691468df81c50700703d56068fdf756
:1035400088fe68b9cd4f4ff0010897f82e0058b1aa
:1035500097f82f00022807d16068fdf7c7fe18b161
:1035600010200eb0bde8f087300702d5a089802872
:103570003ed8700705d4b9f1000f02d097f82400a7
:10358000a0b3e07dc0f300108df81b00627d072022
:10359000032162b3012a2dd0022ae2d0042ae0d10d
:1035a0008df81710f00628d4a27d07202ab3012a2f
:1035b00023d0022a24d0042ad3d18df8191000bfb9
:1035c0008df81590606810b307a9fff7abfe0028cf
:1035d000c7d19df81c00ff2816d0606850f8011f65
:1035e000cdf80f108088adf8130014e000e001e082
:1035f0000720b6e78df81780d4e78df81980dfe74c
:1036000002208df81900dbe743f20220a9e7cdf88c
:103610000f50adf81350e07b40b9207c30b9607c8e
:1036200020b9a07c10b9e07cc00601d0062098e744
:103630008df800a0bdf82c00adf80200a068019044
:10364000a068029004f10f0001f0a7fc8df80c00b7
:10365000fff791fe8df80d009df81c008df80e000f
:103660008df816508df81850e07d08a900f00f0075
:103670008df81a0068460ef047fa05f0f1fd70e784
:10368000f0b58fb000258df830508df814508df8be
:10369000345006468df828500195029503950495ff
:1036a00019b10fc901ac84e80f00744ca07805284b
:1036b00001d004280cd101986168884200d120b95a
:1036c0000398e168884203d110b108200fb0f0bd23
:1036d000207dc00601d51f2700e0ff273b460daa2d
:1036e00005a903a8fff7abfd0028efd1a08ac10709
:1036f00002d0c00600d4ee273b460aaa0ca901a8b6
:10370000fff79dfd0028e1d19df81400c00701d00e
:103710000a20dbe7a08a410708d4a17d31b19df8da
:103720002810890702d043f20120cfe79df8281026
:10373000c90709d0400707d4208818b144f2506166
:10374000884201d90720c1e78df818508df819601b
:10375000bdf80800adf81a000198079006a80ef011
:10376000dff905f07dfd0028b0d18df820508df8ef
:103770002160bdf81000adf822000398099008a858
:103780000ef0f0f905f06cfd00289fd101ad241d6d
:1037900095e80f0084e80f00002097e770b586b029
:1037a0000d46040005d0fdf7a1fd20b1102006b0a4
:1037b00070bd0820fbe72078c107a98802d0ff2947
:1037c00002d303e01f2901d20920f0e7800763d468
:1037d000fff75afc38b12178c1f3c100012804d0a9
:1037e000032802d005e01320e1e7244890f82400e4
:1037f000c8b1c8074ff001064ff0000502d08df8a0
:103800000f6001e08df80f50fff7b5fd8df8000057
:1038100020786946c0f3c1008df8010060788df80a
:103820000250c20801d00720c1e730b3c20701d05f
:103830008df80260820705d59df8022042f0020251
:103840008df80220400705d59df8020040f00400e5
:103850008df80200002022780b18c2f38002da7083
:1038600001eb40026388d380401ca388c0b253811f
:103870000228f0d3207a78b905e001e0f4010020b5
:103880008df80260e6e7607a30b9a07a20b9e07a74
:1038900010b9207bc00601d0062088e704f108009b
:1038a00001f07bfb8df80e0068460df05afd05f027
:1038b000d7fc002889d18df810608df81150e08870
:1038c000adf81200adf8145004a80df09dfd05f000
:1038d000c7fc002888d12078c00701d0152000e05f
:1038e0001320fff7bbfb002061e72de9ff47022013
:1038f000fd4e8df804000027708eadf80600b84626
:1039000043f202094ce001a80ff08ffa050006d03f
:10391000708ea8b3a6f83280adf806803ee0039c16
:10392000a07f01072dd504f124000090a28ebdf8e0
:103930000800214604f1360301f0cafc050005d059
:103940004d452ad0112d3cd0ffdf3ae0a07f20f07a
:103950000801e07f420862f3c711a177810861f393
:103960000000e07794f8210000f01f0084f82000a8
:103970002078282826d129212046fff7cbfb21e0fb
:1039800014e040070ad5bdf8080004f10e0101f06b
:103990001afb05000dd04d4510d100257f1cffb24c
:1039a00002200ff083fa401cb842acd8052d11d08c
:1039b00008e0a07f20f00400a07703e0112d00d0e4
:1039c000ffdf0025bdf806007086052d04d02846cf
:1039d00004b0c7e5a6f832800020f9e770b50646c6
:1039e000fff731fd054605f019fe040000d1ffdfa9
:1039f0006680207820f00f00801c20f0f00020303e
:103a000020700320207295f83e006072bde870407f
:103a100005f007be2de9f04786b0040000d1ffdfb6
:103a20002078b14d20f00f00801c20f0f0007030a5
:103a3000207060680178491f1b2933d2dfe801f04c
:103a4000fe32323255fd320efdfd42fc323232780a
:103a5000fcfcfbfa32fcfcf9f8fcfc00c6883046a2
:103a6000fff7f1fc0546304607f03bfce0b160682b
:103a7000007a85f83e0021212846fff74bfb3046af
:103a8000fef750fb304603f0e7fe3146012013f00d
:103a900063f8a87f20f01000a877fff726ff002822
:103aa00000d0ffdf06b05de5207820f0f000203088
:103ab00020700320207266806068007a607205f0d2
:103ac000b0fdd8e7c5882846fff7bdfc00b9ffdf89
:103ad00060680079012800d0ffdf6068017a06b0d5
:103ae0002846bde8f04707f0e1bdc6883046fff73d
:103af000aafc050000d1ffdf05f093fd60683146a8
:103b00000089288160684089688160688089a8810f
:103b1000012013f021f80020a875a87f00f0030011
:103b20000228bfd1fff7e1fe0028bbd0ffdfb9e7d5
:103b3000007928b10228b5d03c28b3d0ffdfb1e727
:103b400005f06ffd6668b6f806a0307a361d0128cc
:103b500006d0687e814605f0effa070003d101e048
:103b6000e878f7e7ffdf0022022150460ff0edf979
:103b7000040000d1ffdf22212046fff7cbfa307985
:103b8000012800d00220a17f804668f30101a177bf
:103b9000308b2081708b6081b08ba08184f8229063
:103ba0008df80880b8680090f86801906a46032193
:103bb00050460ff0caf900b9ffdfb888adf8100021
:103bc000b8788df8120004aa052150460ff0bdf90f
:103bd00000b9ffdfb888adf80c00f8788df80e005a
:103be00003aa042150460ff0b0f900b9ffdf062107
:103bf00006f1120001f005fa40b37079800700d594
:103c0000ffdf7179e07d61f34700e075d6f80600cb
:103c1000a0617089a083062106f10c0001f0f1f982
:103c2000f0b195f825004108607861f3470006e09f
:103c300041e039e071e059e04ee02fe043e0607090
:103c4000d5f82600c4f80200688d12e0e07d20f06f
:103c5000fe00801ce075d6f81200a061f08ad9e75a
:103c6000607820f0fe00801c6070f068c4f80200ec
:103c7000308ae080b8f1010f04d0b8f1020f05d00e
:103c8000ffdf0fe70320fff7d1f90be7287e1228ab
:103c900000d0ffdf1120fff7e1f903e706b020466f
:103ca000bde8f04701f0a0bd05f0bbfc15f8300ff2
:103cb00040f0020005e005f0b4fc15f8300f40f0cc
:103cc00004002870eee6287e13280ad01528d8d1e3
:103cd0005ff01600fff7c2f906b0bde8f04705f047
:103ce000a0bc1420f6e70000f4010020a978052903
:103cf00009d00429c5d105f094fc022006b0bde826
:103d0000f047fff793b900790028bad0e87801f0be
:103d10002bf905f086fc0320f0e7287e122802d15b
:103d2000687e01f021f91120d4e72de9f05f054606
:103d300000784ff000080009dff8b4a891460c465f
:103d4000464601286ed002286dd007280bd00a28dd
:103d50006ad0ffdfa9f8006014b1a4f80080668083
:103d60000020bde8f09f6968012704f108000b7886
:103d70004ff0020b5b1f4ff6ff721b2b7ed2dfe86a
:103d800003f0647d7d7d0e7d7d7d7d7d7d217d7d4e
:103d90007d2bfdfcfbfa7d14d2f9e7f8f700c8880b
:103da0004ff01208102621469ae14ff01c080a260f
:103db000bcb38888a0806868807920726868c07900
:103dc0006072c7e74ff01b08142654b3032020721b
:103dd00068688088a080bde70a793c2abad00d1daa
:103de0004ff010082c26e4b16988a180298b6182ec
:103df000298b2182698ba182a98be1826b79024692
:103e0000a91d1846fff7effa2979002001290cd0e7
:103e100084f80fb0ff212176e06120626062a06229
:103e200098e70fe03be15ee199e1e77320760af164
:103e3000040090e80e00daf81000c4e90930c4e983
:103e4000071287e7a9f800608ae72c264ff01d08c3
:103e5000002cf7d0a28005460f1d897b008861f3f6
:103e600000002880b97a490861f341002880b97ab6
:103e7000890861f382002880b97a00e00ce1c90862
:103e800061f3c3002880b97aaa1c0911491c61f3a7
:103e9000041000f07f0028807878b91cfff7a3fa9f
:103ea000387d05f1090207f11501fff79cfa387b0f
:103eb00001f0b6f82874787b01f0b2f86874f87ee7
:103ec000a874787ae874387f2875b87b6875388a62
:103ed000e882daf81c10a961b97a504697f808a070
:103ee000c1f34111012904d0008c504503d2824610
:103ef00009e0ffdf10e0022903d0288820f06000ed
:103f000009e0504504d1288820f06000403002e0ec
:103f1000288840f060002880a4f824a0524607f1c9
:103f20001d01a8699be011264ff02008002c89d0c4
:103f3000a280686804f10a02007920726868007b38
:103f4000607269688b1d48791946fff74cfa01e7e2
:103f50000a264ff02108002ce9d08888a0806868e4
:103f6000807920726868c07960729af8301006e033
:103f700078e06be052e07fe019e003e03ae021f006
:103f80000401a6e00b264ff02208002ccfd0c888f1
:103f9000a0806868007920726868007a01f040f8b3
:103fa00060726868407a01f03bf8a072d2e61c2685
:103fb0004ff02608002cbad0a28068684079607261
:103fc0006868007aa0720af1040090e80e00daf83e
:103fd0001000c4e90530c4e90312686800793c2880
:103fe00003d0432803d0ffdfb4e62772b2e684f89b
:103ff00008b0afe610264ff02408002c97d0888830
:10400000a0806868807920816868807a60816868ab
:104010000089a08168688089e0819be610264ff0c6
:104020002308002c98d08888a0806868c0882081e8
:1040300068680089608168684089a08168688089b3
:10404000e0819af8301021f0020142e030264ff072
:104050002508002c9ad0a2806968282249680af0b5
:10406000e4f977e62a264ff02f08002c8ed0a280a4
:1040700069682222091df2e714264ff01b08002c64
:1040800084d0a280686800790128b0d02772dae96c
:104090000710c4e903105de64a46214660e0287a2d
:1040a000012803d0022817d0ffdf53e610264ff077
:1040b0001f08002ca2d06888a080a8892081e889e8
:1040c0006081288aa081688ae0819af8301021f006
:1040d00001018af830103de64ff01208102668887a
:1040e00000f07cff36e6287ac8b3012838d00228d1
:1040f00036d0032801d0ffdf2ce609264ff0110847
:10410000002c8fd06f883846fff79df990f822a0d9
:10411000a780687a2072042138460ef031ff05210d
:1041200038460ef02dff002138460ef029ff012100
:1041300038460ef025ff032138460ef021ff0221fc
:1041400038460ef01dff062138460ef019ff0721f4
:1041500038460ef015ff504600f006fffae5ffe77f
:104160002846bde8f05f01f0c9bc70b5012803d056
:10417000052800d0ffdf70bd8db22846fff763f938
:10418000040000d1ffdf20782128f4d005f046faa2
:1041900080b1017821f00f01891c21f0f00110316c
:1041a00001700221017245800020a075bde87040b9
:1041b00005f037ba21462846bde870401322fff7c4
:1041c00045b92de9f04116460c00804600d1ffdfcd
:1041d000307820f00f00801c20f0f000103030709c
:1041e0002078012804d0022818d0ffdfbde8f08134
:1041f0004046fff728f9050000d1ffdf0320a8752e
:1042000005f00ffa94e80f00083686e80f00f8482a
:1042100010f8301f41f001010170e7e74046fff759
:1042200012f9050000d1ffdfa1884ff6ff700027cb
:10423000814202d1e288824203d0814201d1e088ea
:1042400040b105f0eef994e80f00083686e80f005b
:10425000af75cbe7a87d0128c8d17823002241465d
:1042600012f0d0fb0220a875c0e738b505460c4611
:104270000846fcf7eeff70bb232d4ad006dc202d4c
:104280000dd0212d23d0222d06d13de0242d46d066
:10429000252d32d03f2d47d00725284638bd002197
:1042a000052012f02ffc08b1112038bda01c0df024
:1042b00042fb04f0d5ff0500efd100220823114690
:1042c000052012f09ffb0528e7d0ffdfe5e76068d7
:1042d000fdf703f808b1102038bd618820886a46d0
:1042e0000df0d2fd04f0bcff0500d6d160680028b7
:1042f000d3d0bdf800100180cfe7a07800f0010115
:1043000020880df0f2fd17e0206801f0a3fe0546bd
:10431000c3e7207800f001000cf024fe0ce0618877
:1043200020880df02cfd07e0207800f001008df8ca
:10433000000068460df04af904f092ffe7e770b517
:1043400005460c460846fcf7aaff08b1102070bdd0
:10435000202d07d0212d0dd0222d0bd0252d09d0b9
:10436000072070bd2088a11c0cf0d0febde8704075
:1043700004f076bf062070bd9d482530704708b513
:10438000342200219a480af07af80120fef74efe06
:104390001120fef763fe96496846263105f0d4f8f1
:1043a00093489df8002010f8251f62f3470121f083
:1043b00001010170002141724ff46171a0f80710f2
:1043c00002218172fef794fe00b1ffdffdf70af8cb
:1043d00001f0d3f908bd10b50c464022002120465b
:1043e0000af04df8a07f20f00300a0772020207075
:1043f0000020a07584f8230010bd70472de9fc4112
:104400000746fcf726ff10b11020bde8fc81784e6e
:1044100006f12501d6f825000090b6f82950adf830
:10442000045096f82b408df806403846fef7c4ff3e
:104430000028ead1fef75cfe0028e6d0009946f895
:10444000251fb580b471e0e710b50446fcf727ffdf
:1044500008b1102010bd66486549224690f8250035
:1044600026314008fef7bfff002010bd3eb50446d0
:104470000d460846fcf713ff08b110203ebd14b1ed
:1044800043f204003ebd5a488078052803d0042832
:1044900001d008203ebd694602a80af019fc2a4650
:1044a00069469df80800fef79eff00203ebdfeb560
:1044b0000d4604004ff0000711d00822fef7a4febd
:1044c000002811d1002608e054f826006946fef7be
:1044d00029ff002808d1761cf6b2ae42f4d30cf0c6
:1044e00088fc10b143f20320febd414e86f82470d3
:1044f0000cb300271be000bf54f8270002a9fef709
:1045000011ff00b1ffdf9df808008df8000054f89e
:10451000270050f8011fcdf801108088adf8050084
:1045200068460cf08bfc00b1ffdf7f1cffb2af428e
:10453000e2d386f824500020febd2de9f0478ab072
:104540001546894604001fd00f4608222946fef76b
:104550005bfe002811d1002614e000bf54f82600ad
:104560006946103000f025fd002806d147b157f804
:104570002600fcf76efe18b110200ab0bde8f087e7
:10458000761cf6b2ae42e9d30026a5f101081be085
:1045900006f1010a0af0ff0712e000bf54f82600f6
:1045a000017c4a0854f827100b7cb2eb530f05d15d
:1045b00006221130113109f00bff58b17f1cffb2f8
:1045c000af42ebd30af0ff064645e1db4e4624b18d
:1045d000012003e043f20520cfe700200cf053fc5c
:1045e00010b90cf05cfc28b143f20420c5e70000d0
:1045f000f401002064b300270df1170826e000bf86
:1046000054f827006946103000f0d3fc00b1ffdffa
:1046100054f82700102250f8111fcdf8011080889f
:10462000adf8050054f827100df1070009f0fdfe64
:1046300096b156f827101022404609f0f6fe68465b
:104640000cf0e1fb00b1ffdf7f1cffb2af42d7d31c
:10465000fef714ff002090e7404601f0effceee784
:1046600030b585b00446fdf7bdf830b906200ef030
:104670001dfc10b1062005b030bd2046fcf7e9fd59
:1046800018b96068fcf732fe08b11020f3e76088c3
:104690004af2b811884206d82078f94d28b101288d
:1046a00006d0022804d00720e5e7fef721fd18e038
:1046b0006078022804d0032802d043f20220dae70f
:1046c00085f82f00c1b200200090adf80400022947
:1046d0002cd0032927d0ffdf68460cf06ffc04f0d4
:1046e000bffd0028c7d1606801f09bfc207858b15d
:1046f00001208df800000df1010001f09ffc6846db
:104700000df059fc00b1ffdf207885f82e00fef790
:10471000b5fe608860b1a88580b20cf0acfb00b13a
:10472000ffdf0020a7e78df80500d5e74020fae776
:104730004ff46170efe710b50446fcf7b0fd20b907
:10474000606838b1fcf7c9fd08b1102010bd606881
:1047500001f074fcca4830f82c1f6180c178617088
:1047600080782070002010bd2de9f843144689465a
:104770000646fcf794fda0b94846fcf7b7fd80b9a2
:104780002046fcf7b3fd60b9bd4da878012800d1e3
:104790003cb13178ff2906d049b143f20400bde8ad
:1047a000f8831020fbe7012801d00420f7e7ccb301
:1047b000052811d004280fd069462046fef777fe61
:1047c0000028ecd1217d49b1012909d0022909d065
:1047d000032909d00720e2e70820e0e7024604e0c9
:1047e000012202e0022200e003228046234617460f
:1047f00000200099fef795fe0028d0d1a0892880de
:10480000a07be875bdf80000a882af75bdf8001068
:10481000090701d5a18931b1a1892980c00704d038
:10482000032003e006e08021f7e70220fef7fefb0d
:1048300086f800804946bde8f8430020fef720bf17
:104840007cb58f4c05460e46a078022803d003287d
:1048500001d008207cbd15b143f204007cbd0720c7
:104860000ef02cfb10b9a078032806d0fef70cfc44
:1048700028b1a078032804d009e012207cbd1320c1
:104880007cbd304600f053fb0028f9d1e670fef7fe
:1048900072fd0af05af901208df800008df8010030
:1048a0008df802502088adf80400e07d8df80600f8
:1048b00068460df027fa04f0d3fc0028e0d1a07878
:1048c000032805d05ff00400fef7b0fb00207cbd9c
:1048d000e07800f03cfb0520f6e71cb510b143f290
:1048e00004001cbd664ca078042803d0052801d024
:1048f00008201cbd00208df8000001218df801105a
:104900008df8020068460df0fdf904f0a9fc0028be
:10491000efd1a078052805d05ff00200fef786fbf6
:1049200000201cbde07800f01ffb0320f6e72de916
:10493000fc4180460e4603250846fcf7d7fc0028bc
:1049400066d14046fef77ffd040004d0207822287f
:1049500004d2082059e543f2020056e5a07f00f09a
:1049600003073eb1012f0cd000203146fef727fc93
:104970000500efd1012f06d0022f1ad0ffdf284605
:1049800043e50120f1e7a07d3146022801d011b1b5
:1049900007e0112039e56846fcf758fe0028d9d118
:1049a0006946404606f045fe0500e8d10120a075a5
:1049b000e5e7a07d032804d1314890f83000c00716
:1049c00001d02eb30ee026b1a07f40071ed40021f7
:1049d00000e00121404606f04cfe0500cfd1a07555
:1049e000002eccd03146404600f0edfa05461128a5
:1049f000c5d1a07f4107c2d4316844f80e1f716849
:104a0000616040f0040020740025b8e71125b6e786
:104a10001020fae470b50c460546fef714fd0100bf
:104a200005d022462846bde87040fef70fbd43f290
:104a3000020070bd10b5012807d1114b9b78012be6
:104a400000d011b143f2040010bd0cf046fabde8ed
:104a5000104004f005bc012300f090ba00231a4670
:104a6000194600f08bba70b506460c460846fcf7ae
:104a7000f0fb18b92068fcf712fc18b1102070bdcb
:104a8000f4010020f84d2a7e112a04d0132a00d305
:104a90003eb10820f3e721463046fef77ffe60b1c5
:104aa000ede70920132a0dd0142a0bd0a188ff2985
:104ab000e5d31520fef7d2fa0020d4e90012c5e9ab
:104ac0000712dce7a1881f29d9d31320f2e71cb510
:104ad000e548007e132801d208201cbd00208df877
:104ae000000068460cf090fc04f0bafb0028f4d1fa
:104af0001120fef7b3fa00201cbd2de9f04fdff8be
:104b000068a3814691b09af818009b4615460c465a
:104b1000132803d3fff7dbff00281fd12046fcf743
:104b200098fbe8bb2846fcf794fbc8bb20784ff005
:104b30000107c0074ff0000102d08df83a7001e084
:104b40008df83a1020788846c0f3c1008df8000037
:104b500060788df80910c10803d0072011b0bde8b6
:104b6000f08fb0b3c10701d08df80970810705d56a
:104b70009df8091041f002018df80910400705d594
:104b80009df8090040f004008df809009df8090027
:104b9000810703d540f001008df80900002000e0f6
:104ba00015e06e4606eb400162884a81401ca288ef
:104bb000c0b20a820328f5d32078c0f3c1000128cf
:104bc00025d0032823d04846fcf743fb28b110200a
:104bd000c4e7ffe78df80970d8e799f800004008ae
:104be00008d0012809d0022807d0032805d043f2b5
:104bf0000220b3e78df8028001e08df8027048468c
:104c000050f8011fcdf803108088adf80700fef7bb
:104c1000b2fb8df801000021424606eb41002b88d3
:104c2000c3826b888383ab884384eb880385491cec
:104c3000c285c9b282860329efd3e088adf83c0073
:104c400068460cf0b9fc002887d19af81800554640
:104c5000112801d0082081e706200ef02ff938b185
:104c60002078c0f3c100012804d0032802d006e058
:104c7000122073e795f8240000283ff46eaffef78a
:104c800003fa022801d2132068e7584600f04ff9d2
:104c900000289dd185f819b068460cf0d3fd04f0ca
:104ca000dffa040094d1687e00f051f91220fef77b
:104cb000d5f9204652e770b56b4d287e122801d0f9
:104cc0000820dce60cf0c1fd04f0cafa040005d1ae
:104cd000687e00f049f91120fef7c0f92046cee6c3
:104ce00070b5064615460c460846fcf7d8fa18b9c2
:104cf0002846fcf7d4fa08b11020c0e62a4621461f
:104d000030460df0a1f804f0abfa0028f5d1217877
:104d10007f29f2d10520b2e67cb505460c4608464f
:104d2000fcf797fa08b110207cbd2846fef78bfbf4
:104d300020b10078222804d208207cbd43f2020072
:104d40007cbd494890f83000400701d511207cbd5a
:104d50002078c00802d16078c00801d007207cbd4f
:104d6000adf8005020788df8020060788df80300cf
:104d70000220adf8040068460bf0a1fe04f070fac2
:104d80007cbd70b586b014460d460646fef75bfb4b
:104d900028b10078222805d2082006b06fe643f239
:104da0000200fae72846fcf7a1fa20b944b12046f0
:104db000fcf793fa08b11020efe700202060a080f4
:104dc000294890f83000800701d51120e5e703a9b4
:104dd00030460bf0c4fe10b104f042fadde7adf846
:104de0000060bdf81400adf80200bdf81600adf883
:104df0000400bdf81000bdf81210adf80600adf8c3
:104e000008107db1298809b1adf80610698809b18b
:104e1000adf80210a98809b1adf80810e98809b108
:104e2000adf80410dcb1bdf80610814201d9081ab2
:104e30002080bdf80210bdf81400814201d9081a83
:104e40006080bdf80800bdf80410bdf816200144cc
:104e5000bdf812001044814201d9081aa0806846aa
:104e60000bf03bffb8e70000f40100201cb57449cb
:104e70000968cde9001068460cf0a0fb04f0f0f9d9
:104e80001cbd1cb500200090019068460cf096fbfc
:104e900004f0e6f91cbd70b505460c460846fcf763
:104ea000fef908b11020eae5214628460cf078f911
:104eb000bde8704004f0d4b93eb505460c4608463e
:104ec000fcf7edf908b110203ebd002000900190e4
:104ed0000290adf800502089adf8080020788df8d8
:104ee0000200606801902089adf808006089adf883
:104ef0000a0068460cf066f904f0b2f93ebd0eb542
:104f0000adf800000020019068460cf05bf904f059
:104f1000a7f90ebd10800888508048889080c88806
:104f200010818888d080002050819081704710b512
:104f3000044604f001f930b1407830b1204604f065
:104f400014fc002010bd052010bd122010bd10b5ae
:104f500004f0f2f8040000d1ffdf607800b9ffdf51
:104f60006078401e607010bd10b504f0e5f80400d4
:104f700000d1ffdf6078401c607010bd1cb5adf83b
:104f800000008df802308df803108df8042068467b
:104f90000cf01dff04f064f91cbd0cb529a2d2e988
:104fa0000012cde900120079694601eb501000783b
:104fb0000cbd0278520804d0012a02d043f202202c
:104fc0007047fef7afb91fb56a46fff7a3ff684603
:104fd0000cf06efc04f044f904b010bd70b50c0088
:104fe00006460dd0fef72ffa050000d1ffdfa680a0
:104ff00028892081288960816889a081a889e08129
:105000003de510b500231a4603e0845c2343521c9f
:10501000d2b28a42f9d30bb1002010bd012010bddd
:1050200000b540b1012805d0022803d0032804d0e0
:10503000ffdf002000bdff2000bd042000bd0000f8
:1050400024620200070605040302010010b50446ad
:10505000fcf7fff808b1102010bd2078c0f3021053
:10506000042807d86078072804d3a178102901d82c
:10507000814201d2072010bde078410706d4217992
:105080004a0703d4000701d4080701d5062010bd44
:10509000002010bd10b513785c08837f64f3c7133c
:1050a000837713789c08c37f64f30003c377107879
:1050b000c309487863f34100487013781c090b78e2
:1050c00064f347130b701378db0863f30000487038
:1050d0005078487110bd10b5c4780b7864f30003a4
:1050e0000b70c478640864f341030b70c478a4089f
:1050f00064f382030b70c478e40864f3c3030b7099
:105100000379117863f30001117003795b0863f38d
:105110004101117003799b0863f3820111700079da
:10512000c00860f3c301117010bd70b514460d4680
:10513000064604f073fa80b10178182221f00f01bd
:10514000891c21f0f001a03100f8081b214609f06c
:105150006cf9bde8704004f064ba29463046bde8f9
:1051600070401322fef772b92de9f047064608a8f1
:10517000904690e8300489461f46142200212846b4
:1051800009f07df90021caf80010b8f1000f03d032
:10519000b9f1000f03d114e03878c00711d02068ae
:1051a000fcf77df8c0bbb8f1000f07d120681230c2
:1051b00028602068143068602068a8602168caf8f8
:1051c00000103878800724d56068fcf786f818bb93
:1051d000b9f1000f21d0fff7cff80168c6f86811c8
:1051e0008188a6f86c11807986f86e0101f015fdb2
:1051f000f94fef60626862b196f8680106f26911d2
:1052000040081032fef7eff810223946606809f0c6
:105210000cf90020bde8f08706e0606820b1e86086
:105220006068c6f86401f4e71020f3e730b505467e
:1052300008780c4620f00f00401c20f0f0011031df
:1052400021700020607095f8230030b104280fd041
:10525000052811d0062814d0ffdf20780121b1ebfa
:10526000101f04d295f8200000f01f00607030bdc0
:1052700021f0f000203002e021f0f000303020700a
:10528000ebe721f0f0004030f9e7f0b591b00227ec
:1052900015460c4606463a46adf80870092103aba0
:1052a00005f04bf80490002810d004208df804007d
:1052b0008df80170e034099605948df818500aa90c
:1052c00068460ff046fb00b1ffdf012011b0f0bdd2
:1052d00010b588b00c460a99adf80000cbb118683b
:1052e000cdf80200d3f80400cdf80600adf80a208e
:1052f000102203a809f099f868460cf049fb03f066
:10530000afff002803d1a17f41f01001a17708b0c1
:1053100010bd0020cdf80200e6e72de9f84f064663
:10532000808a0d4680b28246fef78df804463078ba
:10533000dff8a48200274ff00209a8f120080f2807
:1053400070d2dfe800f06ff23708387d8cc8f1f0da
:10535000eff35ff3f300a07f00f00300022809d011
:105360005ff0000080f0010150460df0f7fd0500f0
:1053700003d101e00120f5e7ffdf98f85c10c907d1
:1053800002d0d8f860000be0032105f11d0011f0f8
:10539000fcf8d5f81d009149b0fbf1f201fb1200b9
:1053a000c5f81d0070686867b068a8672078252870
:1053b00000d0ffdfcae0a07f00f00300022809d080
:1053c0005ff0000080f0010150460df0c7fd0600bf
:1053d00003d101e00120f5e7ffdf3078810702d536
:1053e0002178252904d040f001003070bde8f88f05
:1053f00085f80090307f287106f11d002d36c5e933
:105400000206f3e7a07f00f00300022808d0002086
:1054100080f0010150460df0a1fd040004d102e02e
:105420000120f5e7a7e1ffdf2078c10604d50720ba
:1054300028703d346c60d9e740f008002070d5e753
:10544000e07f000700d5ffdf307cb28800f0010369
:1054500001b05046bde8f04f092106f04cb804b940
:10546000ffdf716821b1102204f1240008f0ddff94
:1054700028212046fdf74efea07f00f00300022801
:105480000ed104f12400002300901a462146504614
:10549000fff71eff112807d029212046fdf73afe0d
:1054a000307a84f82000a1e7a07f000700d5ffdf55
:1054b00014f81e0f40f008002070e782a761e76132
:1054c000c109607861f34100014660f382016170b7
:1054d000307ae0708ae7a07f00f00300022809d04c
:1054e0005ff0000080f0010150460df037fd040030
:1054f00003d101e00120f5e7ffdf022104f185007f
:1055000011f043f80420287004f5b4706860b4f812
:1055100085002882304810387c346c61c5e90280ef
:1055200064e703e024e15be02de015e0a07f00f0fc
:105530000300022807d0002080f0010150460df042
:105540000dfd18b901e00120f6e7ffdf32462146e4
:105550005046bde8f84fe8e504b9ffdf2078212880
:10556000a1d93079012803d1e07f40f00800e0772d
:10557000324621465046fff7d8fd2046bde8f84f99
:105580002321fdf7c7bd3279aa8005f1080309215f
:10559000504604f0d2fee86010b10520287025e7df
:1055a000a07f00f00300022808d0002080f0010155
:1055b00050460df0d3fc040003d101e00120f5e7d3
:1055c000ffdf04f1620102231022081f0df04dfbe2
:1055d00007703179417009e75402002040420f0002
:1055e000a07f00f00300022808d0002080f0010115
:1055f00050460df0b3fc050003d101e00120f5e7b2
:10560000ffdf95f8840000f0030001287ad1a07f25
:1056100000f00307e07f10f0010602d0022f04d152
:1056200033e095f8a000c0072bd0d5f8601121b366
:1056300095f88320087c62f387000874a17fca096b
:10564000d5f8601162f341000874d5f8601166f373
:1056500000000874aeb1d5f86001102204f12401f5
:10566000883508f0e2fe287e40f001002876287890
:1056700020f0010005f8880900e016b1022f04d0df
:105680002de095f88800c00727d0d5f85c1121b32c
:1056900095f88320087c62f387000874a17fca090b
:1056a000d5f85c1162f341000874d5f85c1166f31b
:1056b000000008748eb1d5f85c01102204f12401b9
:1056c000883508f0b2fe287840f0010005f8180b84
:1056d000287820f0010005f8a009022f44d000200e
:1056e00000eb400005ebc00090f88800800709d56a
:1056f00095f87c00d5f86421400805f17d01103251
:10570000fdf771fe8df8009095f884006a4600f070
:1057100003008df8010095f888108df8021095f8b7
:10572000a0008df803002146504601f05ffa207872
:10573000252805d0212807d0ffdf2078222803d98b
:1057400022212046fdf7e6fca07f00f0030002289e
:105750000cd0002080f0010150460df011fc002813
:105760003ff44faeffdf41e60120b9e70120f1e74a
:10577000706847703ae6ffdf38e670b5fe4c0025ea
:1057800084f85c5025660ff0b0f804f11001204653
:1057900003f000ff84f8305070bd70b50d46fdf782
:1057a00052fe040000d1ffdf4ff4b87200212846fa
:1057b00008f065fe04f124002861a07f00f00300da
:1057c000022809d05ff0010105f1e0000ff08ef82a
:1057d000002800d0ffdf70bd0221f5e70a46014630
:1057e00002f1e0000ff0a3b870b50546406886b03e
:1057f00001780a2906d00d2933d00e292fd0ffdfda
:1058000006b070bd86883046fdf71dfe040000d14d
:10581000ffdf20782128f3d028281bd168680221d7
:105820000e3001f0d8f9a8b168680821801d01f098
:10583000d2f978b104f1240130460cf065fa03f096
:105840000ffd00b1ffdf06b02046bde87040292102
:10585000fdf760bc06b0bde8704003f0e2be012178
:1058600001726868c6883046fdf7edfd040000d17e
:10587000ffdfa07f00f00301022902d120f0100019
:10588000a077207821280ad06868017a09b10079c8
:1058900080b1a07f00f00300022862d0ffdfa07f6c
:1058a00000f003000228abd1fef71ff80028a7d0b4
:1058b000ffdfa5e703f0b5fea17f08062bd5e07f4b
:1058c000c00705d094f8200000f01f00102820d059
:1058d0005ff0050084f82300207829281dd02428b3
:1058e000ddd13146042011f037f922212046fdf7a1
:1058f00011fca07f00f00300022830d05ff0000010
:1059000080f0010130460df03bfb0028c7d0ffdfdf
:10591000c5e70620dee70420dce701f003000228eb
:1059200008d0002080f0010130460df017fb050083
:1059300003d101e00120f5e7ffdf25212046fdf737
:10594000e9fb03208df80000694605f1e0000ef048
:10595000e5ff0228a3d00028a1d0ffdf9fe70120a8
:10596000cee703f05efe9ae72de9f04387b0994653
:10597000164688460746fdf766fd04004bd02078a2
:10598000222848d3232846d0e07f000743d4a07fb5
:1059900000f00300022809d05ff0000080f0010150
:1059a00038460df0dbfa050002d00ce00120f5e7e7
:1059b000a07f00f00300022805d001210022384614
:1059c0000df0c3fa05466946284601f036f90098fd
:1059d00000b9ffdf45b10098e03505612078222845
:1059e00006d0242804d007e000990020086103e0d5
:1059f00025212046fdf78efb00980121417047626a
:105a0000868001a9c0e902890ef0a3ff022802d016
:105a1000002800d0ffdf07b0bde8f08370b586b086
:105a20000546fdf710fd017822291ed9807f00f080
:105a30000300022808d0002080f0010128460df064
:105a40008dfa04002fd101e00120f5e7ffdf2ae005
:105a5000b4f85e0004f1620630440178427829b15e
:105a600021462846fff711fcb0b9c9e6adf804207d
:105a70000921284602ab04f060fc03900028f4d012
:105a800005208df80000694604f1e0000ef046ffa5
:105a9000022801d000b1ffdf02231022314604f1b9
:105aa0005e000df018f9b4f860000028d0d1a7e628
:105ab00010b586b00446fdf7c6fc017822291bd933
:105ac000807f00f00300022808d0002080f0010150
:105ad00020460df043fa040003d101e00120f5e770
:105ae000ffdf06208df80000694604f1e0000ef0ab
:105af00015ff002800d0ffdf06b010bd2de9f05fd4
:105b000005460c4600270078904601093e4604f100
:105b1000080bba4602297dd0072902d00a2909d1eb
:105b200046e0686801780a2905d00d2930d00e2991
:105b30002ed0ffdfbbe114271c26002c6bd0808801
:105b4000a080fdf780fc5fea000900d1ffdf99f833
:105b500017005a46400809f11801fdf744fc68682f
:105b6000c0892082696851f8060fc4f8120048689d
:105b7000c4f81600a07e01e03402002020f00600e8
:105b800040f00100a07699f81e0040f020014de0a1
:105b90001a270a26002cd1d0c088a080fdf753fc1c
:105ba000050000d1ffdf59462846fff73ffb7ee1a5
:105bb0000cb1a88ba080287a0b287dd006dc0128a8
:105bc0007bd0022808d0032804d135e00d2875d0f9
:105bd0000e2874d0ffdf6ae11e270926002cadd005
:105be000a088fdf730fc5fea000900d1ffdf287bc9
:105bf00000f003000128207a1bd020f00100207261
:105c0000297b890861f341002072297bc90861f36f
:105c1000820001e041e1f2e02072297b090961f391
:105c2000c300207299f81e0040f0400189f81e1050
:105c30003de140f00100e2e713270d26002caad039
:105c4000a088fdf700fc8146807f00f00300022859
:105c500008d0002080f00101a0880df07ff9050038
:105c600003d101e00120f5e7ffdf99f81e0000f005
:105c70000302022a50d0686f817801f003010129e4
:105c8000217a4bd021f00101217283789b0863f3c4
:105c9000410121728378db0863f3820121728378ea
:105ca0001b0963f3c3012172037863f306112172a8
:105cb000437863f3c71103e061e0a9e090e0a1e05d
:105cc000217284f809a0c178a172022a29d0027930
:105cd000e17a62f30001e1720279520862f3410154
:105ce000e1720279920862f38201e1720279d208cc
:105cf00062f3c301e1724279217b62f300012173f7
:105d00004279520862f3410121734279920862f3a9
:105d100082012173407928e0a86fade741f00101cd
:105d2000b2e74279e17a62f30001e1724279520806
:105d300062f34101e1724279920862f38201e172f9
:105d40004279d20862f3c301e1720279217b62f3e6
:105d5000000121730279520862f341012173027933
:105d6000920862f3820121730079c00860f3c301d5
:105d7000217399f80000232831d9262140e0182703
:105d80001026e4b3a088fdf75efb8346807f00f019
:105d90000300022809d0002080f00101a0880df046
:105da000ddf85fea000903d101e00120f4e7ffdf3d
:105db000e868a06099f8000040f0040189f800103c
:105dc00099f80100800708d5012020739bf8000096
:105dd00023286cd92721584651e084f80ca066e0ae
:105de00015270f265cb1a088fdf72dfb8146062202
:105df0005946e86808f0affb0120a073a0e041e03d
:105e000048463ce016270926e4b3287b20724ee082
:105e1000287b19270e26acb3c4f808a0a4f80ca060
:105e2000012807d0022805d0032805d0042803d074
:105e3000ffdf0de0207207e0697b042801f00f010d
:105e400041f0800121721ed0607a20f00300607260
:105e5000a088fdf7f8fa05460078212827d02328e6
:105e600000d0ffdfa87f00f00300022813d000203d
:105e700080f00101a0880df083f822212846fdf76b
:105e800049f914e004e0607a20f00300401cdee7ea
:105e9000a8f8006010e00120eae70cb16888a08053
:105ea000287a68b301280ad002284fd0ffdfa8f86b
:105eb00000600cb1278066800020bde8f09f1527a8
:105ec0000f26002ce4d0a088fdf7bdfa807f00f0fb
:105ed0000300022808d0002080f00101a0880df006
:105ee0003df8050003d101e00120f5e7ffdfd5f81b
:105ef0001d000622594608f02efb84f80ea0d6e7b6
:105f000017270926002cc3d0a088fdf79cfa8146ec
:105f1000807f00f00300022808d0002080f00101fb
:105f2000a0880df01bf8050003d101e00120f5e782
:105f3000ffdf6878800701d5022000e00120207291
:105f400099f800002328b2d9272159e719270e26ee
:105f5000002c9dd0a088fdf776fa5fea000900d1f9
:105f6000ffdfc4f808a0a4f80ca084f808a0a07a69
:105f700040f00300a07299f81e10c90961f3820075
:105f8000a07299f81f2099f81e1012ead11f05d0af
:105f900099f8201001f01f0110292bd020f00800e3
:105fa000a07299f81f10607a61f3c3006072697a79
:105fb00001f003010129a2d140f00400607299f8b8
:105fc0001e0000f003000228e87a16d0217b60f35f
:105fd00000012173aa7a607b62f300006073ea7aa1
:105fe000520862f341012173a97a490861f3410023
:105ff00060735ce740f00800d2e7617b60f300016a
:106000006173aa7a207b62f300002073ea7a520857
:1060100062f341016173a97a490861f34100207379
:1060200045e710b5f74c30b10146102204f12000cd
:1060300008f0fbf9012084f8300010bd10b50446cb
:1060400000f0ebfdef4920461022bde81040203162
:1060500008f0ebb970b5eb4d06004ff0000413d01b
:10606000fbf7f7f808b110240ce00621304608f0e1
:1060700059fa411c05d028665ff0010085f85c00e4
:1060800000e00724204670bd0020f7e7007810f0fc
:106090000f0204d0012a05d0022a0cd110e0000919
:1060a00009d10ae00009012807d0022805d00328f9
:1060b00003d0042801d007207047087000207047e3
:1060c0000620704705282ad2dfe800f003070f17e3
:1060d0001f00087820f0ff001ee0087820f00f0075
:1060e000401c20f0f000103016e0087820f00f007f
:1060f000401c20f0f00020300ee0087820f00f0067
:10610000401c20f0f000303006e0087820f00f004e
:10611000401c20f0f000403008700020704707203d
:1061200070472de9f041804688b00d4600270846ab
:10613000fbf7dcf8a8b94046fdf785f9040003d069
:106140002078222815d104e043f2020008b0bde80f
:10615000f08145b9a07f410603d500f00300022875
:1061600001d01020f2e7a07fc10601d4010702d5bb
:106170000db10820eae7e17f090701d50d20e5e729
:1061800000f0030002280dd165b12846fef75eff3e
:106190000700dbd1fbf726fb20b9e878800701d5a3
:1061a0000620d3e7a07f00f00300022808d00020db
:1061b00080f0010140460cf0d1fe060002d00fe055
:1061c0000120f5e7a07f00f0030002280ed0002098
:1061d00080f00101002240460cf0b7fe060007d017
:1061e000a07f00f00300022804d009e00120efe7bf
:1061f0000420abe725b12a4631462046fef74aff88
:106200006946304600f019fd009800b9ffdf00999b
:10621000022006f1e0024870c1f824804a610022a1
:106220000a81a27f02f00302022a1cd00120087119
:10623000287800f00102087e62f3010008762a78cf
:10624000520862f3820008762a78920862f3c3004b
:1062500008762a78d20862f30410087624212046b2
:10626000fcf758ff33e035b30871301d8861307892
:10627000400908777078c0f340004877287800f02c
:106280000102887f62f301008877a27fd20962f35e
:1062900082008877e27f62f3c3008877727862f3c6
:1062a00004108877a878c87701f1210228462031a8
:1062b000fef711ff03e00320087105200876252171
:1062c0002046fcf727ffa07f20f04000a07701a91f
:1062d00000980ef03efb022801d000b1ffdf3846e7
:1062e00034e72de9ff4f9346474a0d4699b09a4649
:1062f00007ca0aab002783e807001998fdf7a3f83f
:10630000060006d03078262806d008201db0bde84b
:10631000f08f43f20200f9e7b07f00f00309b9f112
:10632000020f11d04db95846fef790fe0028edd16e
:10633000b07f00f00300022806d0bbf1000f11d09f
:10634000fbf750fa20b10de0bbf1000f4fd109e08f
:1063500006200cf0abfd28b19bf80300800701d5a7
:106360000620d3e7b07f00f00300022808d0002009
:1063700080f0010119980cf0f1fd040003d101e057
:106380000120f5e7ffdf852d27d007dcedb1812d5a
:106390001dd0822d1dd0832d08d11ce0862d1ed04e
:1063a000882d1ed0892d1ed08a2d1ed00f20207141
:1063b0000f281cd003f032f9d8b101208df83c0031
:1063c000201d10902079b0b156e10020efe70120a8
:1063d000ede70220ebe70320e9e70520e7e70620e9
:1063e000e5e70820e3e70920e1e70a20dfe70720e7
:1063f0008ce711208ae7b9f1020f07d0a56f07d10a
:10640000a06f06e0340200202c620200656ff6e700
:10641000606f80462dd04ff0010001904ff00200d8
:1064200000905a4621463046fef734fe9bf80000a5
:1064300000f00101a87861f30100a870b17fc909db
:1064400061f38200a870f17f61f3c300a8706178e6
:1064500061f30410a8702078400928706078c0f3b8
:10646000400068709bf80200e87000206871287195
:1064700003e00220019001200090a87898f8021013
:10648000c0f3c000c1f3c001084003902cd05046b7
:10649000faf7dffec0bbdaf80c00faf7dafe98bbb9
:1064a000daf81c00faf7d5fe70bbdaf80c00a06031
:1064b000daf81c00e060607898f8012042ea5001a8
:1064c00061f34100607098f80210c0b200ea111147
:1064d00061f30000607000202077009906f117003a
:1064e000022907d0012106e0607898f8012002ea2d
:1064f0005001e5e7002104eb810148610199701c1e
:10650000022902d0012101e028e0002104eb8101f1
:106510004861a87800f00300012857d198f80200dc
:1065200000f00300012851d1b9f1020f04d02a1d57
:10653000691d5846fef7cffd287998f804100840e9
:106540008df83400697998f8052011408df83810dd
:1065500008433bd05046faf77cfe08b11020d5e640
:106560000af110018b46b9f1020f17d0084600213d
:1065700004f18c03cde9000304f5ae7202920dab79
:106580002046039afef7f0fd0028e8d1b9f1020f8a
:1065900008d0504608d14ff0010107e050464ff0b7
:1065a0000101e5e75846f5e74ff0000104f1a403c7
:1065b000cde9000304f5b072029281f001010eab47
:1065c0002046039afef7d0fd0028c8d160788007e6
:1065d00033d4a87898f80210c0f38000c1f380018a
:1065e00008432ad0297898f800000aaab9f1020fc6
:1065f00006d032f811204300da4002f003070ae027
:1066000032f810204b00da4012f0030705d0012fba
:106610000ad0022f0ad0032f06d0039a6ab10129ab
:1066200006d0042904d008e00227f6e70127f4e7a2
:10663000012801d0042800d10427b07f40f0800059
:10664000b077f17f039860f30001f17760788007fd
:1066500005d50320a071039870b9002029e002201d
:10666000022f18d0012f18d0042f2ad00020a0719b
:10667000b07f20f08000b07725213046fcf74afd3e
:106680000fa904f1e0000ef049f910b1022800d082
:10669000ffdf00203ae6a071dfe7a0710d220021a4
:1066a00004f1200007f0ebfe207840f0020020709b
:1066b00001208df85c0017aa3146199800f096fa6f
:1066c000dae70120a071d7e72de9f04387b09046c3
:1066d000894604460025fcf7b6fe060006d0307851
:1066e000272806d0082007b0bde8f08343f2020057
:1066f000f9e7b07f00f00300022809d05ff0000046
:1067000080f0010120460cf029fc040003d101e0d7
:106710000120f5e7ffdfa7795fea090005d001282e
:1067200021d0b9f1020f26d110e0b8f1000f22d12b
:10673000012f05d0022f05d0032f05d0ffdf2ee05b
:106740000c252ce001252ae0022528e04046faf736
:1067500080fdb0b9032f0ed11022414604f11d0077
:1067600007f063fe1be0012f02d0022f03d104e0eb
:10677000b8f1000f13d00720b5e74046faf769fdde
:1067800008b11020afe71022002104f11d0007f02e
:1067900076fe0621404607f0c5fec4f81d002078ad
:1067a000252140f0020020703046fcf7b3fc207831
:1067b000c10713d020f00100207002208df80000e6
:1067c00004f11d0002908df804506946c3300ef0ac
:1067d000a5f8022803d010b1ffdf00e025770020e4
:1067e00081e730b587b00d460446fcf72cfe98b122
:1067f000807f00f00300022811d0002080f001010a
:1068000020460cf0abfb04000ed02846faf721fd21
:1068100038b1102007b030bd43f20200fae7012082
:10682000ece72078400701d40820f3e7294604f17b
:106830003d002022054607f0f8fd207840f01000ca
:10684000207001070fd520f00800207007208df878
:106850000000694604f1e00001950ef05ff802289f
:1068600001d000b1ffdf0020d4e770b50d46064629
:10687000fcf7e9fd18b10178272921d102e043f2a4
:10688000020070bd807f00f00300022808d00020c5
:1068900080f0010130460cf061fb040003d101e0ff
:1068a0000120f5e7ffdfa079022809d16078c00751
:1068b00006d02a4621463046fef7e7fc10b10fe02d
:1068c000082070bdb4f860000e280bd204f16201fc
:1068d00002231022081f0cf0c8f901210170457035
:1068e000002070bd112070bd70b5064614460d46df
:1068f0000846faf7aefc18b92046faf7d0fc08b102
:10690000102070bda6f57f40ff380ed03046fcf752
:106910009afd38b1417822464b08811c1846fcf795
:1069200062fd07e043f2020070bd2046fdf78cfdda
:106930000028f9d11021e01d0ff027fee21d2946a5
:1069400004f1170000f089f9002070bd2de9f04135
:1069500004468ab01546884600270846faf7c6fc62
:1069600018b92846faf7c2fc18b110200ab0bde8e1
:10697000f0812046fcf767fd060003d03078272819
:106980001bd102e043f20200f0e7b07f00f0030009
:10699000022809d05ff0000080f0010120460cf0d1
:1069a000ddfa040003d101e00120f5e7ffdf2078e4
:1069b000400702d56078800701d40820d6e7b07f71
:1069c00000f00300022803d0a06f03d1a16f02e002
:1069d000606ffae7616f407800b19db1487810b1ff
:1069e000b8f1000f0ed0adb1ea1d06a8e16800f0c5
:1069f00034f9102206a905f1170007f0e9fc18b1d7
:106a0000042707e00720b1e71022e91d04f12d005b
:106a100007f00bfdb8f1000f06d0102208f10701b6
:106a200004f11d0007f001fd2078252140f002004f
:106a300020703046fcf76efb2078c10715d020f09f
:106a40000100207002208df8000004f11d0002906a
:106a5000103003908df804706946b3300df05eff7e
:106a6000022803d010b1ffdf00e0277700207de788
:106a7000f8b515460e460746fcf7e5fc040004d0c1
:106a80002078222804d00820f8bd43f20200f8bd87
:106a9000a07f00f00300022802d043f20500f8bdf9
:106aa0003046faf7d6fb18b92846faf7d2fb08b1f8
:106ab0001020f8bd00953288b31c21463846fef7f9
:106ac00007fc112815d00028f3d1297c4a08a17fa2
:106ad00062f3c711a177297ce27f61f30002e277bc
:106ae000297c890884f82010a17f21f04001a1773a
:106af000f8bda17f0907fbd4d6f80200c4f8360020
:106b0000d6f80600c4f83a003088a086102229463c
:106b100004f1240007f089fc287c4108e07f61f340
:106b20004100e077297c61f38200e077287c8008cf
:106b300084f82100a07f40f00800a0770020d3e770
:106b400070b50d4606460bb1072070bdfcf77bfc07
:106b5000040007d02078222802d3a07f800604d426
:106b6000082070bd43f2020070bdadb12946304629
:106b70000bf0caf802f074fb297c4a08a17f62f38b
:106b8000c711a177297ce27f61f30002e277297cbb
:106b9000890884f8201004e030460bf0d8f802f0a1
:106ba0005ffba17f21f02001a17770bd70b50d467c
:106bb000fcf749fc040005d02846faf770fb20b129
:106bc000102070bd43f2020070bd29462046fef73a
:106bd0002dfb002070bd04e010f8012b0ab100204d
:106be0007047491e89b2f7d20120704770b515462b
:106bf000064602f013fd040000d1ffdf207820f0ec
:106c00000f00801c20f0f000203020706680286883
:106c1000a060bde8704002f004bd10b5134c94f8bc
:106c20003000002808d104f12001a1f110000df07e
:106c3000b7fe012084f8300010bd10b190f8b920e3
:106c40002ab10a4890f8350018b1002003e0b830a6
:106c500001e0064834300860704708b5002300930f
:106c600013460a460cf079fb08bd000034020020f0
:106c700018b18178012938d101e0102070470188ce
:106c800042f60112881a914231d018dc42f6010214
:106c9000a1eb020091422ad00cdc41b3b1f5c05ff8
:106ca00025d06ff4c050081821d0a0f57060ff38cf
:106cb0001bd11ce001281ad002280ad117e0b0f538
:106cc000807f14d008dc012811d002280fd00328bf
:106cd0000dd0ff2809d10ae0b0f5817f07d0a0f5db
:106ce0008070033803d0012801d0002070470f20a6
:106cf00070470a281fd008dc0a2818d2dfe800f005
:106d0000191b1f1f171f231d1f21102815d008dc5a
:106d10000b2812d00c2810d00d2816d00f2806d121
:106d20000de011280bd084280bd087280fd003202a
:106d300070470020704705207047072070470f20dc
:106d4000704704207047062070470c20704743f2bc
:106d50000200704738b50c46050041d06946fff780
:106d600095f9002819d19df80010607861f30200b0
:106d700060706946681cfff789f900280dd19df8fd
:106d80000010607861f3c5006070a978c1f341011b
:106d9000012903d0022905d0072038bd217821f030
:106da000200102e0217841f020012170410704d048
:106db000a978c90861f386106070607810f0380f08
:106dc00007d0a978090961f3c710607010f0380f77
:106dd00002d16078400603d5207840f04000207052
:106de000002038bd70b50446002008801546606854
:106df000fff7b0ff002816d12089a189884211d859
:106e000060688078c0070ad0b1f5007f0ad840f2e8
:106e10000120b1fbf0f200fb1210288007e0b1f571
:106e2000ff7f01d90c2070bd01f2012129800020d3
:106e300070bd10b50478137864f300031370047800
:106e4000640864f3410313700478a40864f38203b4
:106e500013700478e40864f3c303137004782409fe
:106e600064f3041313700478640964f34513137016
:106e70000078800960f38613137031b10878c10778
:106e800001d1800701d5012000e0002060f3c71385
:106e9000137010bd4278530702d002f0070306e0da
:106ea00012f0380f02d0c2f3c20300e001234a7887
:106eb00063f302024a70407810f0380f02d0c0f33a
:106ec000c20005e0430702d000f0070000e0012007
:106ed00060f3c5024a7070472de9f04f95b00d0080
:106ee000824613d012220021284607f0c8fa4ff636
:106ef000ff7b05aa0121584607f089f800242646a1
:106f000037464ff420586ff4205972e0102015b026
:106f1000bde8f08f9df81e0001280ad1bdf81c10b5
:106f200041450bd011eb09000ad001280cd00228f2
:106f30000cd0042c0ed0052c0fd10de0012400e064
:106f40000224bdf81a6008e0032406e00424bdf81a
:106f50001a7002e0052400e00624bdf81a1051451d
:106f600047d12c74beb34ff0000810aa4ff0070aa7
:106f7000cde90282cde900a80df13c091023cdf83e
:106f8000109042463146584607f011f908bbbdf84b
:106f90003c002a46c0b210a90df078fdc8b9ae81f8
:106fa000cfb1cde900a80df1080c0aae40468ce83f
:106fb0004102132300223946584607f0f8f840b939
:106fc000bdf83c00f11cc01ec0b22a1d0df05efdd4
:106fd00010b103209be70ae0bdf82900e881062ce8
:106fe00005d19df81e00a872bdf81c002881002064
:106ff0008de705a807f017f800288bd0fff779fe7a
:1070000085e72de9f0471c46dde90978ddf8209099
:1070100015460e00824600d1ffdf0cb1208818b162
:10702000d5b11120bde8f087022d01d0012100e08b
:10703000002106f1140005f0b3fea8f80000024696
:107040003b462946504603f078f9c9f8000008b9d4
:10705000a41c3c600020e5e71320e3e7f0b41446ed
:10706000dde904528db1002314b1022c09d101e0f5
:10707000012306e00d7cee0703d025f00105012376
:107080000d742146f0bc04f036ba1a80f0bc70478b
:107090002de9fe4f91461a881c468a468046fab171
:1070a00002ab494603f049f9050019d04046a61c39
:1070b00027880cf098f83246072629463b4600966a
:1070c0000bf0a5fc20882346cde900504a465146e6
:1070d0004046fff7c3ff002020800120bde8fe8f5f
:1070e0000020fbe72de9f04786b082460ea89046c7
:1070f00090e8b000894604aa05a903a88de8070016
:107100001e462a4621465046fff77bff039901b1f0
:1071100001213970002818d1fa4904f1140204ab96
:107120000860039805998de8070042464946504695
:1071300006f0e9f9a8b1092811d2dfe800f0050846
:107140000510100a0c0c0e00002006b06ae7112092
:10715000fbe70720f9e70820f7e70d20f5e7032014
:10716000f3e7bdf810100398cde9000133462a4635
:1071700021465046fff772ffe6e72de9f04389b05c
:107180001646dde910870d4681461c461422002173
:1071900003a807f074f9012002218df810108df872
:1071a0000c008df81170adf8146064b1a278d207ac
:1071b00009d08df81600e088adf81a00a088adf867
:1071c0001800a068079008a80095cde90110424674
:1071d00003a948466b68fff785ff09b0bde8f08357
:1071e000f0b58bb000240646069407940727089450
:1071f00005a80994019400970294cde903400d4637
:1072000010232246304606f0d2ff78b90aa806a914
:10721000019400970294cde90310bdf814300022c8
:107220002946304606f061fd002801d0fff761fdd8
:107230000bb0f0bd06f0f2bb2de9fc410c468046d8
:10724000002602f0ebf9054620780d287ed2dfe813
:1072500000f0bc0713b325bd49496383af959b007c
:10726000a848006820b1417841f010014170ade0bc
:10727000404602f003faa9e0042140460bf06efefe
:10728000070000d1ffdf07f11401404605f01dfda6
:10729000a5bb13214046fdf7bdfb97e00421404606
:1072a0000bf05cfe070000d1ffdfe088adf80000c6
:1072b0000020b8819df80000010704d5c00602d562
:1072c000a088b88105e09df8010040067ed5a08821
:1072d000f88105b9ffdf22462946404601f0c0fc8f
:1072e000022673e0e188adf800109df80110090650
:1072f0000fd5072803d006280ad00ae024e004218d
:1073000040460bf02bfe060000d1ffdfa088f08185
:107310000226cdb9ffdf17e0042140460bf01efe28
:10732000070000d1ffdf07f1140006f0aefb90f07c
:10733000010f02d1e079000648d5387c022640f0e2
:107340000200387405b9ffdf224600e03de029461f
:10735000404601f085fc39e0042140460bf0fefd7b
:10736000017c002d01f00206c1f340016171017c36
:1073700021f002010174e7d1ffdfe5e702260121d8
:10738000404602f0adf921e0042140460bf0e6fd55
:107390000546606800902089adf804000122694626
:1073a000404602f0bef9287c20f0020028740de06f
:1073b000002dc9d1ffdfc7e7022600214046fbf7b9
:1073c00081f8002dc0d1ffdfbee7ffdf3046bde80a
:1073d000fc813eb50c0009d001466b4601aa002095
:1073e00006f06aff20b1fff784fc3ebd10203ebdd1
:1073f00000202080a0709df8050002a900f0070081
:10740000fef760fe50b99df8080020709df8050059
:1074100002a9c0f3c200fef755fe08b103203ebd2d
:107420009df8080060709df80500c109a07861f31f
:107430000410a0709df80510890961f3c300a070c5
:107440009df80410890601d5022100e0012161f3b5
:1074500042009df8001061f30000a07000203ebdc6
:1074600070b5144606460d4651ea040005d075b1c4
:107470000846f9f732ff78b901e0072070bd2946c8
:10748000304606f080ff10b1bde8704031e454b1e1
:107490002046f9f722ff08b1102070bd2146304682
:1074a000bde8704095e7002070bd2de9fc5f0c46fb
:1074b00090460546002701780822007a3e46b2eb46
:1074c000111f7dd104f10a0100910a31821e4ff093
:1074d000020a04f1080b0191092a72d2dfe802f0d6
:1074e000ede005f528287baace00688804210bf082
:1074f00035fd060000d1ffdfb08928b152270726ed
:10750000c3e000009802002051271026002c7dd0f7
:107510006888a0800120a071a88900220099fff747
:107520009fff002873d1a8892081288ae081d1e0bb
:10753000b5f81290072824d1e87b000621d5512701
:1075400009f1140086b2002ce1d0a889002200992c
:10755000fff786ff00285ad16888a08084f806a02b
:10756000a88920810120a073288a2082a4f8129083
:10757000a88a009068884b46a969019a01f04cfbe3
:10758000a8e0502709f1120086b2002c3ed0a8894d
:1075900000225946fff764ff002838d16888a08090
:1075a000a889e080287a072813d002202073288a2f
:1075b000e081e87bc0096073a4f81090a88a01e01c
:1075c00085e082e0009068884b4604f11202a969c8
:1075d000d4e70120eae7b5f81290512709f1140029
:1075e00086b2002c66d0688804210bf0b7fc834675
:1075f0006888a080a88900220099fff731ff002841
:107600006ed184f806a0a889208101e052e067e0ed
:107610000420a073288a2082a4f81290a88a0090df
:1076200068884b46a969019a01f0f6faa989abf876
:107630000e104fe06888fbf706ff074668880421b4
:107640000bf08cfc064607b9ffdf06b9ffdf687b4d
:10765000c00702d05127142601e0502712264cb350
:107660006888a080502f06d084f806a0287b594651
:1076700001f0e2fa2ee0287ba11df9e7fe49a88976
:107680004989814205d1542706269cb16888a0808b
:1076900020e053270be06888a080a889e08019e0eb
:1076a000688804210bf05afc00b9ffdf5527082633
:1076b000002cf0d1a8f8006011e056270726002c16
:1076c000f8d06888a080002013e0ffdf02e00128e6
:1076d00008d0ffdfa8f800600cb12780668000208a
:1076e000bde8fc9f57270726002ce3d06888a080c0
:1076f000687aa071eee7401d20f0030009b1414314
:10770000091d01eb4000704713b5db4a00201071e2
:10771000009848b1002468460bf03dfa002c02d1d5
:10772000d64a009911601cbd01240020f4e770b511
:107730000d461446064686b05c220021284606f017
:107740009efe04b9ffdfa0786874a27821882846dd
:1077500001f09dfa0020a881e881228805f114013a
:10776000304605f096fa6a460121304606f04ffc95
:107770001ae000bf9df80300000715d5bdf80610fc
:107780003046fff72dfd9df80300bdf8061040f0d0
:1077900010008df80300bdf80300adf81400ff23be
:1077a0003046059a06f0b7fd684606f03cfc002816
:1077b000e0d006b070bd10b50c4601f1140005f024
:1077c000a0fa0146627c2046bde8104001f094ba60
:1077d00030b50446a84891b04ff6ff75c18905aa97
:1077e000284606f014fc30e09df81e00a0422ad086
:1077f00001282ad1bdf81c00b0f5205f03d042f665
:107800000101884221d1002002ab0aaa0ca90190f3
:1078100083e8070007200090bdf81a10102300220b
:10782000284606f0c4fc38b9bdf828000baac0b23f
:107830000ca90df02bf910b1032011b030bd9df84b
:107840002e00a04201d10020f7e705a806f0ebfbcf
:107850000028c9d00520f0e770b5054604210bf0db
:107860007dfb040000d1ffdf04f114010c46284623
:1078700005f02bfa21462846bde8704005f02cbae9
:1078800070b58ab00c460646fbf7ddfd050014d046
:107890002878222827d30cb1a08890b101208df838
:1078a0000c0003208df8100000208df8110054b159
:1078b000a088adf81800206807e043f202000ab083
:1078c00070bd0920fbe7adf8180005900421304693
:1078d0000bf044fb040000d1ffdf04f1140005f0bd
:1078e00026fa000701d40820e9e701f097fe60b10d
:1078f00008a802210094cde9011095f8232003a9de
:1079000030466368fff7eefbd9e71120d7e72de992
:10791000f04fb2f802a0834689b01546894650461a
:10792000fbf791fd0746042150460bf017fb00269c
:10793000044605964ff002080696adf81c6007b99c
:10794000ffdf04b9ffdf4146504603f03bff50b96b
:1079500007aa06a905a88de8070042462146504619
:107960006368fff74efb444807ab0660dde905128c
:1079700004f11400cdf80090cde90320cde90131e8
:1079800097f82320594650466b6805f019fa06000f
:107990000ad0022e04d0032e14d0042e00d0ffdf14
:1079a00009b03046bde8f08fbdf81c000028f7d0c4
:1079b0000599cde900104246214650466368fff71d
:1079c0004dfbede7687840f008006870e8e72de9c6
:1079d000f04f99b004464ff000082748adf81c80de
:1079e000adf82080adf82480a0f80880adf81480b0
:1079f000adf81880adf82c80adf8288000791646d7
:107a00000d464746012808d0022806d0032804d096
:107a1000042802d0082019b0c4e72046f9f719fc61
:107a200070bb2846f9f715fc50bb6068f9f75efc9f
:107a300030bb606848b160892189884202d8b1f5bd
:107a4000007f01d90c20e6e780460eaa06a9284649
:107a5000fff7c8f90028ded168688078c0f34100dc
:107a6000022808d19df8190010f0380f03d02869ba
:107a7000f9f733fc20b904e098020020140000203c
:107a800022e005a92069fff765f90028c3d1206924
:107a900048b1607880079df8150000f0380001d5e6
:107aa000f0b300e0e0bb9df8140080060ed59df811
:107ab000150010f0380f03d06068f9f70efc18b904
:107ac0006068f9f713fc08b11020a4e70aa96069ff
:107ad000fff740f900289ed1606940b19df8290068
:107ae00000f0070101293cd110f0380f39d00ba963
:107af000a069fff72ff900288dd19df82800800696
:107b00002fd49df82c0080062bd4a06950b19df88d
:107b10002d0000f00701012923d110f0380f00e0fb
:107b20001fe01ed0e06818b10078d0b11c2818d230
:107b30000faa611c2046fff77cf90121384661f34a
:107b40000f2082468df85210b94642f603000f46c8
:107b5000adf850000df13f0218a928680cf0b5fff0
:107b600008b1072057e79df8600015a9cdf80090ef
:107b7000c01ccde9019100f0ff0b00230bf20122a4
:107b8000514614a806f06ef9f0bbbdf854000c90f5
:107b9000fe482a8929690092cde901106b89bdf858
:107ba00038202868069906f05df901007ed120781a
:107bb0004ff0020ac10601d480062bd5cdf80c90f7
:107bc000606950b90aa906a8fff764f99df8290071
:107bd00020f00700401c8df829009df8280008a916
:107be00040f0c8008df828008df8527042f602105f
:107bf000adf8500003aacdf800a0cde90121002383
:107c000040f2032214a800e01ee00a9906f02af9c7
:107c100001004bd1dd484d4608385b460089adf880
:107c20003d000fa8cde90290cdf80490cdf810905a
:107c30004ff007090022cdf80090bdf854104ff620
:107c4000ff7006f052f810b1fff753f8e3e69df825
:107c50003c00000624d52946012060f30f218df851
:107c600052704ff424500395adf8500062789df89f
:107c70000c00002362f300008df80c006278cdf850
:107c800000a0520862f341008df80c0003aacde970
:107c9000012540f2032214a806f0e4f8010005d102
:107ca000606888b32069a8b905a900e084e006a847
:107cb000fff7f0f86078800706d49df8150020f0f3
:107cc00038008df8150005e09df8140040f04000e4
:107cd0008df814008df8527042f60110adf8500086
:107ce000208940f20121b0fbf1f201fb1202606831
:107cf00009abcdf80080cde90103002314a8059954
:107d000006f0b0f8010057d12078c00728d00395bd
:107d1000a06950b90ba906a8fff7bcf89df82d0083
:107d200020f00700401c8df82d009df82c008df8e8
:107d3000527040f040008df82c0042f60310adf870
:107d4000500007a903aacdf800a0cde90121002326
:107d500040f2032214a80b9906f084f801002bd1fd
:107d6000e06868b32946012060f30f218df8527056
:107d700042f60410adf85000e068002302788df858
:107d8000582040788df85900e06816aa4088adf870
:107d90005a00e06800798df85c00e068c088adf8b2
:107da0005d00cdf80090cde901254ff4027214a8d2
:107db00006f058f8010003d00c9800f0c9ff2ae63d
:107dc000724803210838017156b100893080bdf82e
:107dd00024007080bdf82000b080bdf81c00f08049
:107de000002018e670b501258ab016460b4601281a
:107df00002d0022816d104e08df80e504ff4205026
:107e000003e08df80e5042f60100adf80c005bb1b6
:107e10000024601c60f30f2404aa08a918460cf083
:107e200054fe18b107204ae5102048e504a99df842
:107e300020205648cde90021801e029000232146d3
:107e400003a802f2012206f00df810b1fef751ff6f
:107e500035e54e4808380eb1c188318005710020e3
:107e60002de5f0b593b0074601268df83e6041f64a
:107e70000100adf83c0012aa0fa93046fff7b2ff8f
:107e8000002849d1414c0025083cefb31c220021b9
:107e900002a806f0f4fa9df808008df83e6040f064
:107ea00020008df8080042f60520adf83c000e9544
:107eb0009df83a00119520f00600801c8df83a00dc
:107ec0009df838006a4620f0ff008df838009df8d4
:107ed000390009a920f0ff008df839000420adf821
:107ee0002c00adf830000ea80a9011a80d900fa834
:107ef0000990adf82e5002a8fff769fd00280bd1bc
:107f0000bdf80000608100e008e0bdf80400a08139
:107f1000401ce0812571002013b0f0bd6581a58172
:107f2000bdf84800f4e72de9f74f1849a0b0002448
:107f3000083917940a79a146012a04d0022a02d0ee
:107f4000082023b02ee5ca88824201d00620f8e737
:107f500021988a46824201d10720f2e7012021467a
:107f600060f30f21adf848004ff6ff780691adf8a9
:107f70004a808df86e0042f6020b8df872401ca903
:107f8000adf86cb0adf87040139101e0a002002094
:107f9000adf8508012a806f075f800252e462f4641
:107fa0000dab072212a9404606f06ff878b10a28f7
:107fb0005dd195b38eb3adf86450adf866609df8b1
:107fc0005e008df8144019ac012864d06be09df878
:107fd0003a001fb3012859d1bdf8381059451fd1b7
:107fe00018a809a901940294cde903100720009074
:107ff000bdf8361010230022404606f0d8f8b0bb7a
:10800000bdf86000042801d006284ad1bdf824102c
:10801000219881423ad10f2093e73ae0012835d1e7
:10802000bdf83800b0f5205f03d042f60101884268
:108030002cd1baf80600bdf83610884201d10127cc
:1080400000e0002705b19eb1219881421ed118a8f9
:1080500009aa01940294cde90320072000900d465f
:1080600010230022404606f0a2f800b902e02de0fd
:108070004e460be0bdf86000022801d0102810d158
:10808000c0b217aa09a90cf001fd50b9bdf836908d
:1080900086e7052055e705a917a8221d0cf015fd58
:1080a00008b103204de79df814000023001dc2b263
:1080b0008df8142022980092cde901401ba8069962
:1080c00005f0d0fe10b902228af80420fef711fe56
:1080d00037e710b50b46401e88b084b205aa0021d0
:1080e0001846fef7a6fe00200df1080c06aa05a909
:1080f00001908ce807000720009001230022214610
:108100004ff6ff7005f0f1fd0446bdf81800012898
:1081100000d0ffdf2046fef7ecfd08b010bdf0b543
:10812000f74f044687b038790e46032804d0042858
:1081300002d0082007b0f0bd04aa03a92046fef72c
:1081400051fe0500f6d160688078c0f34100022836
:108150000ad19df80d0010f0380f05d02069f9f70d
:10816000bcf808b11020e5e7208905aa21698de84f
:1081700007006389bdf810202068039905f072fe9e
:1081800010b1fef7b6fdd5e716b1bdf8140030808a
:10819000042038712846cde7f8b50c0006460cd00f
:1081a00001464ff6ff7500236a46284606f084f81c
:1081b00028b100bffef79dfdf8bd1020f8bd69464f
:1081c0002046fef7c7fd0028f8d1a078314600f020
:1081d00001032846009a06f09ef8ebe730b587b019
:1081e000144600220df1080c05ad01928ce82c001c
:1081f000072200920a46014623884ff6ff7005f0d9
:1082000074fdbdf814102180fef773fd07b030bd7a
:1082100070b50d4604210af0a1fe040000d1ffdf75
:10822000294604f11400bde8704004f079bd70b532
:108230000d4604210af092fe040000d1ffdf29461a
:1082400004f11400bde8704004f08dbd70b50d461a
:1082500004210af083fe040000d1ffdf294604f167
:108260001400bde8704004f0a5bd70b505460421ba
:108270000af074fe040000d1ffdf2146284623687f
:10828000bde870400122fef703bf70b50646042129
:108290000af064fe040000d1ffdf04f1140004f0d2
:1082a00030fd401d20f0030511e0011d0088002273
:1082b000431821463046fef7ebfe00280bd0607cc9
:1082c000abb2684382b2a068011d0af004fda06849
:1082d00041880029e9d170bd70b5054604210af036
:1082e0003dfe040000d1ffdf214628466368bde85b
:1082f00070400222fef7ccbe70b50e46054601f076
:108300008df9040000d1ffdf0120207266726580c4
:10831000207820f00f00001d20f0f0004030207089
:10832000bde8704001f07db910b50446012900d0c8
:10833000ffdf2046bde810400121faf7c3b82de960
:10834000f04f97b04ff0000a0c008346adf814a030
:10835000d04619d0e06830b1a068a8b10188adf866
:108360001410a0f800a05846fbf76df8070043f280
:10837000020961d0387822285cd3042158460af0db
:10838000edfd050005d103e0102017b0bde8f08f2a
:10839000ffdf05f1140004f0b4fc401d20f00306db
:1083a000a078012803d0022801d00720ede721881a
:1083b00007aa584605f02bfe30bb07a805f033fe90
:1083c00010bb07a805f02ffe48b99df8260001282c
:1083d00005d1bdf82400a0f52451023902d04ff494
:1083e0005050d2e7e068b0b1cde902a0072000907c
:1083f00005aacdf804a00492a2882188bdf8143003
:10840000584605f072fc10b1fef773fcbde7a16899
:10841000bdf8140008809df81f00c00602d543f285
:108420000140b2e70b9838b1a1780078012905d056
:1084300080071ad40820a8e74846a6e7c007f9d065
:1084400002208df83c00a8684ff00009a0b1697cbb
:108450004288714391420fd98ab2b3b2011d0af02a
:10846000f0fb8046a0f800a006e003208df83c0059
:10847000d5f800804ff001099df8200010f0380f6a
:1084800000d1ffdf9df820001e49c0f3c200084460
:1084900097f8231010f8010c884201d90f2074e7d7
:1084a0002088adf8400014a90095cde9019143461c
:1084b00007220fa95846fef715fe002891d19df816
:1084c000500050b9a078012807d1687cb3b270433e
:1084d00082b2a868011d0af0c8fb002055e770b5fc
:1084e000064615460c460846fef7c2fb002805d195
:1084f0002a4621463046bde8704073e470bd12e55f
:1085000098020020fc2f000070b51e4614460d0096
:1085100009d044b1616831b138b1fc49c9888142a0
:1085200003d0072070bd102070bd2068fef7a0fbaf
:108530000028f9d1324621462846bde87040fff7b1
:1085400046ba70b515460c0006d038b1ef49098916
:10855000814203d0072070bd102070bd2068fef757
:1085600087fb0028f9d129462046bde87040d6e5b2
:1085700070b5064686b00d4614461046f8f78ffed5
:10858000d0bb6068f8f7b2feb0bba6f57f40ff38fd
:1085900003d03046faf757ff80b128466946fef708
:1085a0009bfc00280cd19df810100f2008293dd20b
:1085b000dfe801f008060606060a0a0843f2020090
:1085c00006b070bd0320fbe79df80210012908d119
:1085d000bdf80010b1f5c05ff2d06ff4c052d142c7
:1085e000eed09df8061001290dd1bdf80410a1f5bb
:1085f0002851062907d200e029e0dfe801f0030353
:1086000004030303dce79df80a1001290fd1bdf82c
:108610000810b1f5245fd3d0a1f60211b1f50051d5
:10862000ced00129ccd0022901d1c9e7ffdf606893
:1086300078b9002305aa2946304605f03dfe10b161
:10864000fef757fbbce79df81400800601d410200c
:10865000b6e76188224628466368fff7bffdafe7ab
:108660002de9f043814687b0884614461046f8f756
:1086700016fe18b1102007b0bde8f083002306aa4b
:108680004146484605f018fe18b100bffef731fb21
:10869000f1e79df81800c00602d543f20140eae771
:1086a0000025072705a8019500970295cde90350fd
:1086b00062884ff6ff734146484605f078fd060094
:1086c00013d16068f8f7ebfd60b960680195cde9fa
:1086d000025000970495238862884146484605f079
:1086e00066fd0646bdf8140020803046cee739b15d
:1086f000864b0a889b899a4202d843f2030070474e
:108700001de610b586b0814c0423adf814306389a2
:1087100043b1a4898c4201d2914205d943f20300ae
:1087200006b010bd0620fbe7adf810100021009147
:108730000191adf8003002218df8021005a90291d7
:1087400004a90391adf812206946fff7f8fde7e7a9
:108750002de9fc4781460d460846f8f77afd88bbaf
:108760004846faf770fe5fea00080ad098f8000061
:10877000222829d3042148460af0f0fb070005d13e
:1087800003e043f20200bde8fc87ffdf07f11400bd
:1087900004f0cdfa06462878012803d0022804d038
:1087a0000720f0e7b0070fd502e016f01c0f0bd042
:1087b000a8792c1dc00709d0e08838b1a068f8f767
:1087c00048fd18b11020dee70820dce721882a7870
:1087d0000720b1f5847f35d01edc40f20315a1f2ed
:1087e0000313a94226d00edcb1f5807fcbd003dc89
:1087f000f9b1012926d1c6e7a1f58073013bc2d0aa
:10880000012b1fd113e0012bbdd0022b1ad0032b5b
:10881000b9d0042b16d112e0a1f20912082a11d204
:10882000dfe802f00b04041010101004abe7022a7a
:10883000a9d007e0012aa6d004e0320700e0f20642
:10884000002aa0dacdb200f0e9fe50b198f823007a
:10885000cde90005fa89234639464846fef78dfce6
:1088600091e711208fe72de9f04f8bb01f46154699
:108870000c4683460026faf7e6fd28b10078222848
:1088800005d208200bb081e543f20200fae7b808f0
:1088900001d00720f6e7032f00d100274ff6ff791c
:1088a000ccb1022d73d32046f8f720fd30b904eb8c
:1088b0000508a8f10100f8f719fd08b11020e1e75b
:1088c000ad1e38f8028caab22146484605f055fe86
:1088d00040455cd1adb20d49b80702d58889401c2e
:1088e00000e001201ffa80f8f80701d08f8900e02e
:1088f0004f4605aa4146584605f089fb4ff0070a46
:108900004ff00009dcb320460be000009802002085
:10891000408810283bd8361d304486b2ae4236d24d
:10892000a01902884245f3d351e000bf9df817001b
:1089300002074cd594b304eb0608361db8f8023094
:10894000b6b2102b23d89a19aa4220d8b8f8002022
:1089500091421cd1c0061cd5cde900a90df1080c2f
:108960000aaaa11948468ce80700b8f800100022ae
:10897000584605f0baf920b1fef7bbf982e726e0c8
:1089800005e0b8f80200bdf82810884201d00b209d
:1089900078e7b8f80200304486b207e0ffe7c00687
:1089a00004d55846fef71cfc002888d19df8170016
:1089b000bdf81a1020f010008df81700bdf8170050
:1089c000adf80000ff235846009a05f0a4fc05a866
:1089d00005f029fb18b9bdf81a10b942a6d904212f
:1089e00058460af0bbfa040000d1ffdfa2895ab151
:1089f000cde900a94d46002321465846fef7bdfbb0
:108a00000028bbd1a5813de700203be72de9ff4fc2
:108a10008bb01e4617000d464ff0000412d0b00870
:108a200002d007200fb0b1e4032e00d100265db1c3
:108a30000846f8f752fc28b93888691e0844f8f748
:108a40004cfc08b11020ede7c74ab00701d5d18929
:108a500000e00121f0074ff6ff7802d0d089401ed8
:108a600000e0404686b206aa0b9805f0d0fa4ff017
:108a700000094ff0070b0df1140a38e09df81b00b8
:108a8000000734d5cdf80490cdf800b0cdf80890ab
:108a9000cde9039a434600220b9805f088fb60bba2
:108aa00005b3bdf814103a8821442819091d8a42db
:108ab00030d3bdf81e2020f8022bbdf8142020f87a
:108ac000022bcde900b9cde90290cdf810a0bdf898
:108ad0001e10bdf8143000220b9805f068fb08b199
:108ae00003209fe7bdf814002044001d84b206a8af
:108af00005f099fa20b10a2806d0fef7faf891e7b6
:108b0000bdf81e10b142b9d934b17db13888a11c6d
:108b1000884203d20c2085e7052083e722462946b8
:108b2000404605f02afd014628190180a41c3c801e
:108b3000002077e710b50446f8f7b1fb08b1102024
:108b400010bd8948c0892080002010bdf0b58bb0d1
:108b50000d4606461422002103a805f090fc0120d2
:108b60008df80c008df8100000208df81100adf884
:108b700014503046faf767fc48b10078222812d327
:108b8000042130460af0eaf9040005d103e043f27b
:108b900002000bb0f0bdffdf04f11400074604f043
:108ba000c6f8800601d40820f3e7207c022140f0bb
:108bb0000100207409a80094cde90110072203a93f
:108bc00030466368fef78efa20b1217c21f0010166
:108bd0002174dee729463046f9f765fc08a93846d6
:108be00004f094f800b1ffdfbdf82040172c01d24b
:108bf000172000e02046a84201d92c4602e0172c9d
:108c000000d2172421463046fff711fb214630469b
:108c1000f9f76df90020bce7f8b51c4615460e467d
:108c2000069f0af0cefa2346ff1dbcb231462a4603
:108c3000009409f0b8fef8bd70b50c4605460e224a
:108c40000021204605f01bfc002020802db1012dc5
:108c500001d0ffdf70bd062000e00520a07170bdcf
:108c600010b548800878134620f00f00001d20f052
:108c7000f00080300c4608701422194604f10800f8
:108c800005f0d3fb00f0cdfc3748046010bd2de9a2
:108c9000f047dff8d890491d064621f0030117463a
:108ca0000c46d9f8000009f094ff050000d1ffdf61
:108cb0004ff000083560a5f800802146d9f8000083
:108cc00009f087ff050000d1ffdf7560a5f800807f
:108cd0007fb104fb07f1091d0bd0d9f8000009f0a2
:108ce00078ff040000d1ffdfb460c4f80080bde865
:108cf000f087c6f80880fae72de9f0411746491dcc
:108d000021f00302194d064601681446286809f04f
:108d10008bff22467168286809f086ff3fb104fb8b
:108d200007f2121d03d0b168286809f07dff042006
:108d30000af0bcf8044604200af0c0f8201a012802
:108d400004d12868bde8f04109f038bfbde8f081e2
:108d500010b50c4605f02af900b1ffdf2046bde84a
:108d60001040fdf7c6bf000098020020140000204c
:108d700038b50c468288817b19b14189914200d96e
:108d80000a462280c188121d90b26a4609f0e8f8ae
:108d9000bdf80000032800d30320c1b2208801f0f1
:108da00027f838bd38b50c468288817b19b1018916
:108db000914200d90a462280c188121d90b26a46ab
:108dc00009f0cef8bdf80000022800d30220c1b29d
:108dd000208801f00df8401cc0b238bd2de9ff5fbe
:108de00082468b46fb4814460bf10302d0e9011082
:108df000cde9021022f0030201a84ff49071019214
:108e000009f0c9fef44e002c02d1f449019a8a609f
:108e1000019901440191b57f05f1010504d1e8b242
:108e20000bf0ccfd00b1ffdf019800eb0510c01c7a
:108e300020f0030101915cb9707ab27a1044c2b299
:108e400000200870308c80b204f00fff00b1ffdf0b
:108e50000198316a08440190214601a800f08bff77
:108e600080460198c01c20f003000190b37af27a8a
:108e7000717a04b1002009f084ff0199084401903f
:108e8000214601a800f0bfffd34800273d4690f8d7
:108e900001900ce0284600f051ff0646817880885a
:108ea000f9f7bcf871786d1c00fb0177edb24d4508
:108eb000f0d10198c01c20f00300019004b1002003
:108ec0003946f9f7b6f80199002708440190c248dd
:108ed0003d4690f801900ce0284600f02fff064632
:108ee000c1788088fef707fc71786d1c00fb017764
:108ef000edb24d45f0d10198c01c20f00300019067
:108f000004b100203946fef7fffb01994ff000093c
:108f100008440190b0484d4647780ee0284600f0de
:108f20000dff0646807b30b106f1080002f06ef9b5
:108f3000727800fb02996d1cedb2bd42eed1019832
:108f4000c01c20f00300019004b10020a3494a781e
:108f5000494602f05ff9019908440190214601a8b1
:108f600000f0bcfe0198c01d20f007000190daf867
:108f70000010814204d3a0eb0b01b1f5803f04db6c
:108f80004ff00408caf8000004e0caf80000b8f185
:108f9000000f03d0404604b0bde8f09f74bb904979
:108fa0000020019a0df06cfefbf7e9f98a4c207f56
:108fb0000090607f012823d0002318b30022864848
:108fc00000211030f8f714fa00b1ffdfe07ffef760
:108fd00048ff00b1ffdf80484ff4f67200214030b7
:108fe00005f04dfa7c480421403080f8e91180f802
:108ff000ea11062180f8eb11032101710020cae774
:109000000123dae702aadae770b5734c064640346a
:10901000207804eb4015e078083598b9a01990f84d
:10902000e80100280fd0a0780f2800d3ffdf20220e
:109030000021284605f023fa687866f3020068707c
:109040000120e070284670bd2de9f04105460c4630
:1090500000270078052190463e46b1eb101f00d056
:10906000ffdf287a50b101280ed0ffdfa8f800609a
:109070000cb1278066800020bde8f0810127092619
:1090800074b16888a08008e00227142644b168887b
:10909000a0802869e060a88a2082287b2072e5e70a
:1090a000a8f80060e7e730b54b4c012000212070a4
:1090b0006170207260720322a272e0726177217780
:1090c00021732174052121831f216183607445a1cf
:1090d00061610a21a177e077404d4ff4b0602062d2
:1090e0006868c11c21f00301814200d0ffdf68687d
:1090f000606030bd30b5394c1568636810339d42ef
:1091000002d20420136030bd334b5d785a6802eb05
:109110000512107051700320d0801720908001201c
:10912000d0709070002090735878401c5870606820
:1091300010306060002030bd70b50646264800241f
:10914000457807e0204600f0f9fd0178b14204d0ef
:10915000641ce4b2ac42f5d1002070bdf7b50746ff
:1091600008780c4610b3fff7e7ff0546a7f1200685
:10917000202f06d0052e19d2dfe806f00f3838155b
:109180001a0000f0e6fd0db1697800e00021401af8
:10919000a17880b20844ff2808d8a07830b1a08810
:1091a000022831d202e0608817282dd20720febda8
:1091b000207a48b361881729f8d3a1881729f5d3f5
:1091c000a1790029f2d0e1790029efd0402811d906
:1091d000ece7000038620200b40300201800002011
:1091e000000000206e52463578000000242f0bd17d
:1091f000207a48b161884ff6fb70814202d8a1887d
:10920000814201d90420febd65b9207802aa01215e
:10921000fff770ff0028f6d12078fff78dff0500db
:1092200000d1ffdf052e18d2dfe806f0030b0e0891
:109230001100a0786870a088e8800fe06088a8809e
:109240000ce0a078a87009e0a078e87006e054f877
:10925000020fa8606068e86000e0ffdf0020febd4c
:109260001a2835d00ddc132832d2dfe800f01b318c
:10927000203131272723252d313129313131312f2b
:109280000f00302802d003dc1e2821d107207047b0
:109290003a3809281cd2dfe800f0151b0f1b1b1bf6
:1092a0001b1b07000020704743f20400704743f285
:1092b00002007047042070470d2070470f20704750
:1092c0000820704711207047132070470620704710
:1092d0000320704710b5007800f0010008f032fe5e
:1092e000bde81040bce710b5007800f0010008f0c0
:1092f00032febde81040b3e70eb5017801f0010180
:109300008df80010417801f001018df8011001780d
:10931000c1f340018df802104178c1f340018df88e
:109320000310017889088df80410417889088df8b8
:10933000051081788df80610c1788df80710007936
:109340008df80800684607f046fefff789ff0ebd5e
:109350002de9f84fdff8f883fe4c00264ff49077a4
:109360001fe0012000f092fd0120fff74dfe0546b1
:109370003946d8f8080009f02cfc686000b9ffdf16
:10938000686807f0f3fcb0b12846faf743fb2846bb
:1093900000f082fd28b93a466968d8f8080009f05b
:1093a00043fc94f9e9010428dbda022009f07efd90
:1093b00007460025a5e03a466968d8f8080009f094
:1093c00033fcf2e7b8f802104046491c89b2a8f80d
:1093d0000210b94201d3002141800221b8f80200f5
:1093e00009f0bcfd002864d0b8f80200694608f016
:1093f00018fdfff735ff00b1ffdf9df8000078b1e1
:10940000b8f8020009f0effe5fea000900d1ffdfc3
:10941000484609f05cf918b1b8f8020002f0c0f94a
:10942000b8f8020009f0cdfe5fea000900d1ffdfc5
:10943000484609f044f9e0bb0321b8f8020009f0fe
:109440008dfd5fea000b47d1ffdf45e0dbf8100040
:1094500010b10078ff2849d0022000f017fd02204b
:10946000fff7d2fd8246484609f035facaf80400f3
:1094700000b9ffdfdaf8040009f0fdfa00210090de
:109480000170b8f802105046aaf8021002f08ef8e7
:10949000484609f0f2fa00b9ffdf504600f0fcfc44
:1094a00018b99af80100000704d50098cbf810000d
:1094b00012e024e0dbf8100038b10178491c11f00b
:1094c000ff01017008d1ffdf06e000221146484687
:1094d00000f002fc00b9ffdf94f9ea01022805db85
:1094e000b8f8020002f029f80028afd194f9e90198
:1094f000042804db484609f024fb00b101266d1c5a
:10950000edb2bd4204d294f9ea010228bff65aaf87
:10951000002e7ff422afbde8f84f032000f0b6bc68
:1095200010b58b4ce06008682061aff2db10f9f7f2
:10953000b8fc607010bd8748002140380170844835
:10954000017085494160704770b505464ff0805005
:109550000c46d0f8a410491c05d1d0f8a810c94376
:109560000904090c0bd050f8a01f01f0010129706b
:10957000416821608068a080287830b970bd0621dc
:1095800020460df002f801202870607940f0c000fc
:10959000607170bd70b54ff080540d46d4f88010e6
:1095a000491c0bd1d4f88410491c07d1d4f8881079
:1095b000491c03d1d4f88c10491c0cd0d4f880106d
:1095c0000160d4f884104160d4f888108160d4f828
:1095d0008c10c16002e010210cf0d7ffd4f890008d
:1095e000401c0bd1d4f89400401c07d1d4f898004b
:1095f000401c03d1d4f89c00401c09d054f8900fb3
:10960000286060686860a068a860e068e86070bd75
:109610002846bde8704010210cf0b7bf4d480079d6
:10962000f2e470b54b4ce07830b3207804eb401096
:10963000407a00f00700204490f9e801002800dc9f
:10964000ffdf2078002504eb4010407a00f007008f
:10965000011991f8e801401e81f8e8012078401cca
:10966000c0b220700f2800d12570a078401ca070d7
:109670000cf014fee57070bdffdf70bd3eb5054611
:10968000032109f06bfc0446284609f09afd0546c3
:1096900004b9ffdf206918b10078ff2800d1ffdf8f
:1096a00001aa6946284600f017fb60b9ffdf0ae00f
:1096b000002202a9284600f00ffb00b9ffdf9df849
:1096c000080000b1ffdf9df80000411e8df800107a
:1096d000eed220690199884201d1002020613ebd6f
:1096e00070b50546a0f57f400c46ff3800d1ffdf7e
:1096f000012c01d0ffdf70bdfff790ff040000d107
:10970000ffdf207820f00f00401d20f0f0005030e7
:10971000207065800020207201202073bde8704019
:109720007fe72de9f04116460d460746fff776ff25
:10973000040000d1ffdf207820f00f00401d20f052
:10974000f00050302070678001202072286805e00a
:1097500018000020f4030020481400202061a8888d
:10976000a0822673bde8f0415be77fb5fff7e4fc1c
:10977000040000d1ffdf02a92046fff7f9fa0546f1
:1097800003a92046fff70efb8df800508df801006d
:10979000bdf80800001dadf80200bdf80c00001d6a
:1097a000adf80400e088adf80600684608f0b4fba8
:1097b000002800d0ffdf7fbd2de9f05ff84e814625
:1097c000307810b10820bde8f09f4846f7f767fdf4
:1097d00008b11020f7e7f34c207808b9fff763fcd5
:1097e000a17a607a4d460844c4b200f0b2faa042b1
:1097f00007d2201ac1b22a460020fff77bfc0028be
:10980000e1d17168e748c91c002721f003017160ac
:10981000b3463e463d46ba463c4690f801800ae0d3
:10982000204600f08bfa4178807b0e4410fb0155f6
:10983000641ce4b27f1c4445f2d10aeb870000ebc4
:10984000c600d84e00eb85005c46f17a012200eba1
:109850008100dbf80410451829464846fff7befa98
:10986000070012d00020fff767fc05000bd005f1c0
:109870001300616820f00300884200d0ffdf707899
:10988000401e7070656038469de7002229464846b4
:10989000fff7a4fa00b1ffdfd9f8000060604ff6cf
:1098a000ff7060800120207000208ce72de9f041de
:1098b0000446bb4817460e46007810b10820bde8a4
:1098c000f0810846f7f7c5fc08b11020f7e7b54d61
:1098d000287808b9fff7e7fb601e1e2807d8012c7f
:1098e00022d13078fe281fd8a8770020e7e7a4f11e
:1098f00020001f2805d8e0b23a463146bde8f041c5
:109900002ce4a4f140001f2805d831462046bde8cc
:10991000f04100f0e9baa4f1a0001f2804d800200b
:10992000a02c03d0a12c06d00720c8e7317801f085
:109930000101e977c3e731680922f82901d38b07d0
:1099400001d01046bbe76b7c03f00303012b04d16d
:109950006b8bd7339cb28c42f3d82962afe72de9e9
:10996000f04781460e460846f7f799fc48b9484645
:10997000f7f7b3fc28b909f1030020f003014945ca
:1099800002d01020bde8f08786484ff0000a403032
:10999000817869b14178804600eb411408343788fa
:1099a00032460021204600f085fa050004d027e069
:1099b000a6f800a00520e5e7b9f1000f24d0308813
:1099c000b84201d90c251fe0607800f00705284651
:1099d00000f05cfa08eb0507324697f8e8014946c3
:1099e000401c87f8e801204607f5f47700f062fa9a
:1099f00005463878401e3870032000f047fa2db134
:109a00000c2d01d0a6f800a02846bbe76078644e74
:109a100000f00701012923d002290cd0032934d0fa
:109a2000ffdf98f801104046491cc9b288f80110c0
:109a30000f2935d036e0616821b1000702d4608873
:109a4000fff71cfe98f8ea014746012802d170781a
:109a5000f9f746fa97f9ea010428e2dbffdfe0e7cd
:109a6000616821b14ff49072b06809f0ddf898f8a0
:109a7000e9014746032802d17078f9f731fa97f9de
:109a8000e9010428cddbffdfcbe7c00602d5608803
:109a9000fff7f4fd98f9eb010628c2dbffdfc0e712
:109aa00080f801a08178491e8170617801f007017a
:109ab00001eb080090f8e811491c80f8e811a3e7d1
:109ac00070b50d460446f7f7c4fb18b92846f7f7fa
:109ad000e6fb08b1102070bd29462046bde8704065
:109ae0000af0a4bf70b505460af0c3ffc4b2284609
:109af000f7f7f3fb08b1102070bd35b128782c7052
:109b000018b1a04201d0072070bd2046fdf760fecd
:109b1000052805d10af0b1ff012801d0002070bd51
:109b20000f2070bd70b5044615460e460846f7f77f
:109b300090fb18b92846f7f7b2fb08b1102070bdaa
:109b4000022c03d0102c01d0092070bd2a463146ca
:109b500020460af09bff0028f7d0052070bd70b5a5
:109b600014460d460646f7f774fb38b92846f7f752
:109b700096fb18b92046f7f7b0fb08b1102070bd6e
:109b80002246294630460af0a0ff0028f7d00720d9
:109b900070bd3eb50446f7f782fb28b110203ebdec
:109ba00018000020b4030020684607f085f9fff78d
:109bb00057fb0028f3d19df806002070bdf808007f
:109bc0006080bdf80a00a0800020e8e770b5054677
:109bd0000c460846f7f781fb20b93cb12068f7f73f
:109be0005efb08b1102070bda08828b12146284630
:109bf000bde87040fdf744be092070bd70b5054654
:109c00000c460846f7f725fb30b9681e1e2814d805
:109c10002046f7f71efb08b1102070bd032d01d9b7
:109c2000072070bd05b9ffdff94800eb850050f84b
:109c3000041c2046bde870400847a5f120001f28fd
:109c400005d821462846bde87040faf70ebbf02d36
:109c50000cd0f12d13d0bf2de2d1a078218800f0d7
:109c6000010001f059fb88b1002070bda068f7f732
:109c7000f0fa0028d0d1204608f0b3f902e02078ad
:109c800008f0d2f9bde87040fff7eaba082070bdcd
:109c900070b504460d460846f7f701fb30b9601e63
:109ca0001e280fd82846f7f7d4fa08b1102070bd47
:109cb000012c03d0022c01d0032c01d1062070bd51
:109cc000072070bda4f120001f28f9d8294620469e
:109cd000bde87040faf733bb08f0c0bc7cb5044661
:109ce000cc48007b00f0010511bb04f0ebfb0db18b
:109cf000226800e00022c8484178c06806f0a9fd4b
:109d0000c5481030c0788df8000010b1012802d08d
:109d100004e0012000e000208df80000684607f014
:109d20003bf9bb4824380068019001a807f0eefe1b
:109d3000002d02d02068283020607cbd30b5b54da4
:109d400004466878a04200d8ffdf686800eb041082
:109d500030bd70b5af4800252c46467807e0204658
:109d6000fff7ecff4078641c2844c5b2e4b2b4426b
:109d7000f5d1284670bd2de9f0410c4607464ff05d
:109d8000000800f0edf80646ff2801d94ff013084f
:109d90003868c01c20f003023a6054ea080421d15c
:109da0009c48f3b2072124300cf0fcfd09e0072c9d
:109db00010d2dfe804f0060408080a0406009748f9
:109dc00004e0974802e0974800e097480cf00afe4c
:109dd000054600e0ffdfa54200d0ffdf641ce4b2cf
:109de000072ce4d3386800eb06103860404666e57f
:109df000021d5143452900d245210844c01cb0fb37
:109e0000f2f0c0b270472de9fc5f064681484ff082
:109e100000088b464746444690f8019022e02046d1
:109e2000fff78cff050000d1ffdf687869463844f2
:109e3000c7b22846fef79cff824601a92846fef7d6
:109e4000b1ff0346bdf804005246001d81b2bdf8c3
:109e50000000001d80b209f0fff86a78641c00fb66
:109e60000288e4b24c45dad13068c01c20f003000f
:109e70003060bbf1000f00d000204246394609f0a7
:109e8000f9f8316808443060bde8fc9f6149403111
:109e900008710020c87070475e494031ca782ab105
:109ea0000a7801eb42110831814201d0012070474c
:109eb000002070472de9f04106460078154600f075
:109ec0000f0400201080601e0f46052800d3ffdf1e
:109ed0004f482a46183800eb8400394650f8043cb5
:109ee0003046bde8f04118472de9f041494e0c4697
:109ef000402806d0412823d042282bd0432806d121
:109f000023e0a07861780d18e178814201d907201b
:109f1000d5e42078012801d91320d0e4ff2d08d8fa
:109f20000af03eff07460cf071f9381a801ea8426d
:109f300001da1220c3e42068b060207930730de0ac
:109f4000bde8f041084600f036b808780228ded8af
:109f5000307703e008780228d9d870770020aee483
:109f60002de9f047dff8ac900026344699f8090057
:109f700099f80a2099f801700244d5b299f80b209b
:109f8000104400f0ff0808e02046fff7d7fe817b71
:109f9000407811fb0066641ce4b2bc42f4d199f82d
:109fa000091099f80a0029442944414400b10120cc
:109fb00008443044e6e438b50446407800f0030035
:109fc000012803d002280bd0072038bd606858b1a3
:109fd000f7f78cf9d0b96068f7f77ff920b915e089
:109fe0006068f7f736f988b969462046fcf74ef8fd
:109ff0000028ead1607800f00300022816d19df80d
:10a00000000098b16068f7f768f978b1102038bda2
:10a010005c620200b4030020180000206b410000c5
:10a0200035b30000b52f0000af4701006189f82962
:10a030000dd8208988420ad8607800f003020a48c7
:10a04000012a06d1d731026a89b28a4201d2092097
:10a05000dde794e80e0000f1100585e80e000ab96e
:10a06000002101830020d2e7b40300202de9f04154
:10a07000074614468846084601f08afd064608eb66
:10a0800088001c22796802ebc0000d18688c58b15a
:10a090004146384601f08bfd014678680078c200e1
:10a0a000082305f120000ce0e88ca8b141463846b1
:10a0b00001f084fd0146786808234078c20005f16c
:10a0c000240008f008fe38b1062121726681d0e92b
:10a0d0000010c4e9031009e0287809280bd00520f6
:10a0e000207266816868e060002028702046bde824
:10a0f000f04101f02ebd072020726681f4e72de9c2
:10a10000f04116460d460746406801eb85011c22ca
:10a1100002ebc1014418204601f072fd40b100215c
:10a12000708865f30f2160f31f4106200cf014fdc9
:10a1300009202070324629463846bde8f04195e7af
:10a140002de9f0410e46074600241c21f07816e068
:10a1500004eb8403726801ebc303d25c6ab1fff7be
:10a160005dfa050000d1ffdf6f802a4621463046a8
:10a17000fff7c5ff0120bde8f081641ce4b2a042f6
:10a18000e6d80020f7e770b5064600241c21c07809
:10a190000ae000bf04eb8403726801ebc303d51827
:10a1a0002a782ab1641ce4b2a042f3d8402070bde2
:10a1b00028220021284604f062f9706880892881ed
:10a1c000204670bd70b5034600201c25dc780ce0ed
:10a1d00000eb80065a6805ebc6063244167816b1c5
:10a1e000128a8a4204d0401cc0b28442f0d8402077
:10a1f00070bdf0b5044600201c26e5780ee000bfd7
:10a2000000eb8007636806ebc7073b441f788f426b
:10a2100002d15b78934204d0401cc0b28542efd893
:10a220004020f0bd0078032801d0002070470120b5
:10a2300070470078022801d0002070470120704745
:10a240000078072801d000207047012070472de9d1
:10a25000f041064688461078f1781546884200d3ca
:10a26000ffdf2c781c27641cf078e4b2a04201d8f0
:10a27000201ac4b204eb8401706807ebc1010844e2
:10a28000017821b14146884708b12c7073e72878de
:10a29000a042e8d1402028706de770b514460b88c5
:10a2a0000122a240134207d113430b8001230a224b
:10a2b000011d08f0dafc047070bd2de9ff4f81b07c
:10a2c0000878dde90e7b9a4691460e4640072cd46d
:10a2d000019808f088ff040000d1ffdf07f10408af
:10a2e00020461ffa88f108f0c5f8050000d1ffdf0d
:10a2f000204629466a4608f010fb0098a0f8037033
:10a30000a0f805a0284608f0b6fb017869f306011d
:10a310006bf3c711017020461ffa88f108f0edf8c1
:10a3200000b9ffdf019806f002fa06eb0900017f91
:10a33000491c017705b0bde8f08f2de9f84f0e46b6
:10a340009a4691460746032108f008fe0446008d10
:10a35000dff8b885002518b198f80000b0421ed18a
:10a36000384608f040ff070000d1ffdf09f1040183
:10a37000384689b208f07ef8050010d038462946e4
:10a380006a4608f0cafa009800210a4601808170e6
:10a3900006f08afa0098c01dcaf8000021e098f87b
:10a3a0000000b04216d104f1260734f8341f012012
:10a3b00000fa06f911ea090f00d0ffdf2088012317
:10a3c00040ea090020800a22391d384608f068fc5e
:10a3d000067006e0324604f1340104f12600fff76e
:10a3e0005cff0a2188f800102846bde8f88ffeb50a
:10a3f00015460c46064602ab0c220621fff79dffd0
:10a40000002827d00299607812220a70801c4870b8
:10a4100008224a80a07002982988052381806988d3
:10a42000c180a9880181e988418100250c20cde9fe
:10a430000005062221463046fff73fff294600224d
:10a4400066f31f41f02310460cf0dcfa6078801ca4
:10a4500060700120febdfeb514460d46062206467c
:10a4600002ab1146fff769ff002812d0029b1320b0
:10a4700000211870a8785870022058809c8006200f
:10a48000cde900010246052329463046fff715ffb6
:10a490000120febd2de9fe430c46804644e002aba0
:10a4a0000e2207214046fff748ff002841d0606890
:10a4b0001c2267788678bf1c06eb860102ebc1017f
:10a4c000451802981421017047700a214180698a59
:10a4d0000181e98a4181a9888180a98981813046e9
:10a4e00001f056fb029905230722c8806f700420f3
:10a4f000287000250e20cde9000521464046fff7d3
:10a50000dcfe294666f30f2168f31f41f023002289
:10a5100006200cf077fa6078fd49801c6070626854
:10a520002046921cfff793fe606880784028b6d1e1
:10a530000120bde8fe83feb50d46064638e002abbd
:10a540000e2207213046fff7f8fe002835d0686854
:10a550001c23c17801eb810203ebc202841802982c
:10a5600015220270627842700a224280a2894281da
:10a57000a2888281084601f00bfb01460298818087
:10a58000618ac180e18a0181a088b8b10020207071
:10a5900000210e20cde9000105230722294630467f
:10a5a000fff78bfe6a68db492846d21cfff74ffe97
:10a5b0006868c0784028c2d10120febd0620e6e7c9
:10a5c0002de9fe430c46814644e0204601f002fba3
:10a5d000d0b302ab082207214846fff7aefe0028a1
:10a5e000a7d060681c2265780679ad1c06eb860151
:10a5f00002ebc10147180298b7f8108006210170dc
:10a60000457004214180304601f0c2fa01460298ab
:10a6100005230722c180a0f804807d7008203870cf
:10a620000025cde9000521464846fff746fe2946ac
:10a6300066f30f2169f31f41f023002206200cf07e
:10a64000e1f96078801c60706268b3492046121d91
:10a65000fff7fdfd606801794029b6d1012068e768
:10a660002de9f34f83b00d4691e0284601f0b2fa90
:10a6700000287dd068681c2290f806a00aeb8a01a9
:10a6800002ebc10144185146284601f097faa1781f
:10a69000cb0069684978ca00014604f1240008f03b
:10a6a00036fb07468188e08b4ff00009091a8eb20d
:10a6b00008b1c84607e04ff00108504601f053fad0
:10a6c00008b9b61cb6b2208bb04200d80646b346d5
:10a6d00002ab324607210398fff72ffe060007d092
:10a6e000b8f1000f0bd0504601f03dfa10b106e072
:10a6f00000201fe60299b8884ff0020908800196f1
:10a70000e28b3968abeb09001ffa80f80a44039822
:10a710004e46009208f067fddde90021f61d434634
:10a72000009608f074f9e08b404480b2e083b98869
:10a73000884201d1012600e00026cde900b6238a37
:10a74000072229460398fff7b8fd504601f00bfa9f
:10a7500010b9e089401ee08156b1a078401ca0707d
:10a760006868e978427811fb02f1cab2012300e07f
:10a7700007e081690e3008f078fa80f800a0002028
:10a78000e0836a6865492846921dfff760fd6868a6
:10a79000817940297ff469af0120cbe570b5064689
:10a7a00048680d4614468179402910d104eb840194
:10a7b0001c2202ebc101084401f043fa002806d034
:10a7c0006868294684713046bde8704048e770bd2e
:10a7d000feb50c460746002645e0204601f0faf992
:10a7e000d8b360681c22417901eb810102ebc10101
:10a7f0004518688900b9ffdf02ab082207213846f7
:10a80000fff79bfd002833d00299607816220a706a
:10a81000801c4870042048806068407901f0b8f9d5
:10a82000014602980523072281806989c18008209a
:10a83000cde9000621463846fff73ffd6078801cd1
:10a840006070a88969890844b0f5803f00d3ffdfb4
:10a85000a88969890844a8816e81626830492046c8
:10a86000521dfff7f4fc606841794029b5d1012001
:10a87000febd30b5438c458bc3f3c704002345b1ff
:10a88000838b641eed1ac38a6d1e1d4495fbf3f382
:10a89000e4b22cb1008918b1a04200d8204603448c
:10a8a0004ff6ff70834200d3034613800c7030bd17
:10a8b0002de9fc41074616460d46486802eb860125
:10a8c0001c2202ebc10144186a4601a92046fff789
:10a8d000d0ffa089618901448ab2bdf8001091427d
:10a8e00012d0081a00d5002060816868407940289d
:10a8f0000ad1204601f09bf9002805d06868294656
:10a9000046713846fff764ffbde8fc812c0000204b
:10a9100025a2000033a2000041a2000043bc0000b9
:10a920002fbc00002de9fe4f0f468146154650888a
:10a93000032108f013fb0190b9f8020001f01bf9a4
:10a9400082460146019801f045f9002824d001987b
:10a950001c2241680aeb8a0002ebc0000c1820465a
:10a9600001f04ef9002817d1b9f80000e18a8842b9
:10a970000ed8a18961b1b8420ed100265146019886
:10a9800001f015f9218c01eb0008608b30b114e067
:10a99000504601f0e8f8a0b3bde8fe8f504601f044
:10a9a000e2f808b1678308e0022ff5d3b9f8040094
:10a9b0006083618a884224d80226b81b87b2b8f81f
:10a9c0000400a28b801a002814dd874200da384682
:10a9d0001ffa80fb688869680291d8f800100a4461
:10a9e000009208f0eefbf61d009a5b460299009675
:10a9f00007f0d9ffa08b384480b2a083618b8842d6
:10aa000007d96888019903b05246bde8f04f01f0bc
:10aa100035b91fd14ff009002872b9f802006881da
:10aa2000d8e90010c5e90410608ba881284601f020
:10aa300090f85146019801f0baf8014601980823b0
:10aa400040680078c20004f1200008f044f90020ba
:10aa5000a0836083504601f086f810b9a089401e9b
:10aa6000a0816888019903b00af0ff02bde8f04fa9
:10aa70001ee72de9f041064615460f461c461846ce
:10aa8000f6f7e7fb18b92068f6f709fc10b11020bb
:10aa9000bde8f0817168688c0978b0ebc10f01d313
:10aaa0001320f5e73946304601f081f80146706819
:10aab00008230078c20005f1200008f0d6f8d4e998
:10aac0000012c0e900120020e2e710b5044603219d
:10aad00008f044fa0146007800f00300022805d08f
:10aae0002046bde8104001f1140280e48a8a204625
:10aaf000bde81040afe470b50446032108f02efa1b
:10ab0000054601462046fff75bfd002816d0294682
:10ab10002046fff75dfe002810d029462046fff7ab
:10ab20000afd00280ad029462046fff7b3fc00287a
:10ab300004d029462046bde8704091e570bd2de95e
:10ab4000f0410c4680461ee0e178427811fb02f1ac
:10ab5000cab2816901230e3008f0bdf80778606839
:10ab60001c22c179491ec17107eb8701606802eba5
:10ab7000c10146183946204601f02cf818b130467c
:10ab800001f037f820b16068c1790029dcd17fe796
:10ab9000fef744fd050000d1ffdf0a202872384689
:10aba00000f0f6ff68813946204601f007f80146bb
:10abb000606808234078c20006f1240008f08bf892
:10abc000d0e90010c5e90310a5f80280284600f07e
:10abd000c0ffb07800b9ffdfb078401eb07057e713
:10abe00070b50c460546032108f0b8f901464068e7
:10abf000c2792244c2712846bde870409fe72de922
:10ac0000fe4f8246507814460f464ff00008002849
:10ac10004fd0012807d0022822d0ffdf2068b8607b
:10ac20006068f860b8e602ab0e2208215046fff7d4
:10ac300084fb0028f2d002981521052301702178a9
:10ac400041700a214180c0f80480c0f80880a0f853
:10ac50000c80628882810e20cde90008082221e064
:10ac6000a678304600f094ff054606eb86012c22bc
:10ac7000786802ebc1010822465a02ab11465046e1
:10ac8000fff75bfb0028c9d00298072101702178eb
:10ac900041700421418008218580c680cde90018db
:10aca00005230a4639465046fff707fb87f8088018
:10acb00072e6a678022516b1022e13d0ffdf2a1df8
:10acc000914602ab08215046fff737fb0028a5d07c
:10acd00002980121022e0170217841704580868002
:10ace00002d005e00625eae7a188c180e18801815c
:10acf000cde900980523082239465046d4e710b51f
:10ad00000446032108f02af9014600f10802204612
:10ad1000bde8104073e72de9f04f0f4605468db0b2
:10ad200014465088032108f019f94ff000088df8f7
:10ad300014800646adf81680042f7bd36a78002a6b
:10ad400078d028784ff6ff794ff01c0a132834d0ba
:10ad500008dc012871d006284ad007286ed01228b6
:10ad60000ed106e014286ad0152869d0162807d11c
:10ad7000aae10c2f04d1307800f00301022907d09a
:10ad8000cdf80880cdf80c8068788df808004ce08c
:10ad900040f0080030706878b07001208df8140021
:10ada000a888adf81800e888adf81a002889adf831
:10adb0001c006889adf81e0011e1b078904239d1cd
:10adc0003078010736d5062f34d120f008003070d6
:10add0006088414660f31f4100200bf0bdfe022059
:10ade0008df81400adf81890a888adf81a00f6e0b8
:10adf000082f1fd1a888ef88814600f0bcfe80464e
:10ae00000146304600f0e6fe18b1404600f0abfec9
:10ae1000b8b1fc48d0e90010cde902106878adf86f
:10ae20000c908df80800adf80e70608802aa3146cb
:10ae3000fff7e5fe0db0bde8f08fb6e01ee041e0a3
:10ae4000ece0716808eb88002c2202ebc000085a85
:10ae5000b842efd1eb4802aad0e90210cde90210c6
:10ae600068788df8080008f0ff058df80a506088b2
:10ae70003146fff7c4fe224629461fe0082fd9d1ec
:10ae8000b5f80480e88800f076fe074601463046b3
:10ae900000f0a0fe0028cdd007eb870271680aeb16
:10aea000c2000844028a4245c4d101780829c1d1b0
:10aeb000407869788842bdd1f9b222463046fff722
:10aec0001ef9b7e70e2f7ff45bafe9886f898b46d9
:10aed000b5f808903046fff775f9abf1400140290d
:10aee00001d309204ae0b9f1170f01d3172f01d27e
:10aef0000b2043e040280ed000eb800271680aeb83
:10af0000c20008440178012903d140786978884259
:10af100090d00a2032e03046fff735f9014640284c
:10af20002bd001eb810372680aebc30002eb00082f
:10af3000012288f800206a7888f801207068aa88c1
:10af40004089b84200d93846ad8903232372a282d2
:10af5000e7812082a4f80c906582084600f018fe74
:10af60006081a8f81490a8f81870a8f80e50a8f8f6
:10af700010b0204600f0edfd5ce7042005212172b1
:10af8000a4f80a80e081012121739e49d1e90421be
:10af9000cde9022169788df80810adf80a006088c3
:10afa00002aa3146fff72bfee3e7062f89d3b078dc
:10afb00090421ad13078010717d520f00800307080
:10afc0006088414660f31f4100200bf0c5fd022060
:10afd0008df81400a888adf81800adf81a906088b4
:10afe000224605a9f9f7edf824e704213046fff7da
:10aff00000f905464028bfd0022083030090224676
:10b000002946304600f003fe4146608865f30f2173
:10b0100060f31f4106200bf09ffd0be70e2fabd115
:10b0200004213046fff7e5f881464028a4d0414688
:10b03000608869f30f2160f31f4106200bf08cfd3f
:10b04000a8890b906889099070682f894089b84257
:10b0500000d938468346b5f80680a8880a90484645
:10b0600000f096fd60810b9818b1022000900b9bb8
:10b0700024e0b8f1170f1ed3172f1cd30420207221
:10b0800009986082e781a4f810b0a4f80c8009eb5d
:10b09000890271680aebc2000d18dde90913a5f8f1
:10b0a0001480a5f818b0e9812b82204600f051fdec
:10b0b00006202870bee601200b2300902246494658
:10b0c000304600f0a4fdb5e6082f8dd1a9883046a2
:10b0d000fff778f80746402886d000f044fd0028a6
:10b0e0009bd107eb870271680aebc20008448046d7
:10b0f00000f086fd002890d1ed88b8f80e002844b5
:10b10000b0f5803f05d360883a46314600f0b6fd81
:10b1100090e6002dced0a8f80e0060883a46314661
:10b12000fff73cfb08202072384600f031fd6081bb
:10b13000a5811ee72de9f05f0c4601281fd0957907
:10b1400092f8048092f8056005eb85011f2202eb5e
:10b15000c10121f0030b08eb060111fb05f14ff6cd
:10b16000ff7202eac10909f1030115fb0611264f1e
:10b1700021f0031abb6840b101283ed125e0616887
:10b18000e57891f800804e78dee75946184607f0da
:10b1900020fd606000b9ffdf5a460021606803f0bf
:10b1a0006ef9e5705146b86807f013fd61684861b3
:10b1b00000b9ffdf6068426902eb090181616068e4
:10b1c00080f800806068467017e060685246416908
:10b1d000184607f029fd5a466168b86807f024fd53
:10b1e000032007f063fe0446032007f067fe201ae1
:10b1f000012802d1b86807f0e1fc0beb0a00bde8ba
:10b20000f09f0000686202002c000020024600212e
:10b2100002208fe7f7b5ff4c0a20164620700098f1
:10b2200060b100254fea0d0007f0b5fc0021a170c8
:10b230006670002d01d10099a160febd012500209e
:10b24000f2e770b50c46154638220021204603f07f
:10b2500016f9012666700a22002104f11c0003f091
:10b260000ef905b9ffdf297a207861f3010020701b
:10b27000a87900282dd02a4621460020fff75aff42
:10b2800061684020e34a88706168c870616808712d
:10b29000616848716168887161682888088161689f
:10b2a00068884881606886819078002811d061683c
:10b2b0000620087761682888c885616828884886dc
:10b2c00060680685606869889288018681864685ff
:10b2d000828570bdc878002802d00022012029e7ad
:10b2e000704770b50546002165f31f4100200bf043
:10b2f00033fc0321284607f031fe040000d1ffdfb4
:10b3000021462846fef71cff002804d0207840f094
:10b3100010002070012070bd70b505460c4603205a
:10b3200007f0b6fd08b1002070bdba488570848072
:10b33000012070bd2de9ff4180460e460f0cfef73f
:10b340006df9050007d06f800321384607f006fe2f
:10b35000040008d106e004b03846bde8f0411321ee
:10b36000f9f758bbffdf5fea080005d0b8f1060f18
:10b3700018d0ffdfbde8ff8120782a4620f00800c2
:10b3800020700020adf8020002208df800004ff67a
:10b39000ff70adf80400adf8060069463846f8f7ce
:10b3a00010ffe7e7c6f3072101eb81021c23606869
:10b3b00003ebc202805c042803d008280ad0ffdf18
:10b3c000d8e7012000904ff440432a46204600f081
:10b3d0001efccfe704b02a462046bde8f041fef748
:10b3e0008ebe2de9f05f05464089002790460c4649
:10b3f0003e46824600f0bffb8146287ac01e0828e0
:10b400006bd2dfe800f00d04192058363c47722754
:10b410001026002c6cd0d5e90301c4e902015ce0e0
:10b4200070271226002c63d00a2205f10c0104f1ca
:10b43000080002f0faff50e071270c26002c57d0cc
:10b44000e868a06049e0742710269cb3d5e90301a1
:10b45000c4e902016888032107f080fd8346fef7f6
:10b46000ddf802466888508049465846fef7fefde2
:10b4700033e075270a26ecb1a88920812de07627d4
:10b480001426bcb105f10c0004f1080307c883e8d9
:10b49000070022e07727102664b1d5e90301c4e94b
:10b4a00002016888032107f059fd01466888fff70b
:10b4b00046fb12e01ce073270826ccb16888032104
:10b4c00007f04cfd01460078c00606d56888fef7f7
:10b4d00037fe10b96888f8f781faa8f800602cb137
:10b4e0002780a4f806a066806888a080002086e6f1
:10b4f000a8f80060fae72de9fc410c461e46174605
:10b500008046032107f02afd05460a2c0ad2dfe80f
:10b5100004f005050505050509090907042303e0ed
:10b52000062301e0ffdf0023cde90076224629460d
:10b530004046fef7c2febde8fc81f8b50546a0f521
:10b540007f40ff382bd0284607f03bfe040000d197
:10b55000ffdf204607f0bff9002821d001466a46e8
:10b56000204607f0daf900980321b0f80560284674
:10b5700007f0f4fc0446052e13d0304600f0fbfa29
:10b5800005460146204600f025fb40b1606805eb0a
:10b5900085013e2202ebc101405a002800d0012063
:10b5a000f8bd007a0028fad00020f8bdf8b50446ae
:10b5b000408807f006fe050000d1ffdf6a462846f6
:10b5c000616800f0c4fa01460098091f8bb230f898
:10b5d000032f0280428842800188994205d1042ac3
:10b5e00008d0052a20d0062a16d022461946fff791
:10b5f00099f9f8bd001d0e46054601462246304623
:10b60000f6f73bff0828f4d1224629463046fcf7de
:10b610007ef9f8bd2c000020636864880a46011d8d
:10b620002046faf7a1f9f4e72246001dfff773fb65
:10b63000efe770b50d460646032107f08ffc0400c6
:10b6400004d02078000704d5112070bd43f2020019
:10b6500070bd2a4621463046fef7c9fe18b9286853
:10b6600060616868a061207840f0080020700020c8
:10b6700070bd70b50d460646032107f06ffc04004f
:10b6800004d02078000704d4082070bd43f20200e3
:10b6900070bd2a4621463046fef7ddfe00b9a58280
:10b6a000207820f008002070002070bd2de9f04fb8
:10b6b0000e4691b08046032107f050fc04464046f8
:10b6c00007f091fd07460020079008900990adf81b
:10b6d00030000a9002900390049004b9ffdf0df14e
:10b6e0000809ffb9ffdf1de038460ba9002206f06c
:10b6f000b5ff9df82c0000f07f050a2d00d3ffdf79
:10b700006019017f491e01779df82c00000609d5bc
:10b710002a460ca907a8fef7c0fd19f80510491c18
:10b7200009f80510761ef6b2ded204f13400f84da9
:10b7300004f1260bdff8dca304f12a07069010e0e1
:10b740005846069900f08cfa064628700a2800d35d
:10b75000ffdf5af8261040468847e08cc05db042b3
:10b7600002d0208d0028ebd10a202870e94d4e46ea
:10b7700028350ee00ca907a800f072fa0446375de0
:10b7800055f8240000b9ffdf55f82420394640461b
:10b790009047bdf81e000028ecd111b0bde8f08f35
:10b7a00010b5032107f0dafb040000d1ffdf0a2205
:10b7b000002104f11c0002f062fe207840f0040039
:10b7c000207010bd10b50c46032107f0c7fb2044c4
:10b7d000007f002800d0012010bd2de9f84f8946d8
:10b7e00015468246032107f0b9fb070004d028461e
:10b7f000f5f72ffd40b903e043f20200bde8f88ff2
:10b800004846f5f74cfd08b11020f7e7786828b1f5
:10b8100069880089814201d90920efe7b9f8000061
:10b820001c2488b100f0a7f980460146384600f094
:10b83000d1f988b108eb8800796804ebc000085c96
:10b8400001280bd00820d9e73846fef79cfc80463b
:10b85000402807d11320d1e70520cfe7fdf7defe12
:10b8600006000bd008eb8800796804ebc0000c18c8
:10b87000b9f8000020b1e88910b113e01120bde74c
:10b880002888172802d36888172801d20720b5e72f
:10b89000686838b12b1d224641463846fff7e9f863
:10b8a0000028abd104f10c0269462046fef7e1ff07
:10b8b000288860826888e082b9f8000030b10220f0
:10b8c0002070e889a080e889a0b12be003202070d7
:10b8d000a889a08078688178402905d180f8028005
:10b8e00039465046fef7d6fd404600f051f9a9f81a
:10b8f000000021e07868218b4089884200d9084601
:10b900002083a6f802a004203072b9f800007081ec
:10b91000e0897082f181208b3082a08ab08130462c
:10b9200000f017f97868c178402905d180f80380c4
:10b9300039465046fef7fffd00205fe770b50d4623
:10b940000646032107f00afb04000ed0284600f04b
:10b9500012f905460146204600f03cf918b1284688
:10b9600000f001f920b1052070bd43f2020070bd66
:10b9700005eb85011c22606802ebc101084400f060
:10b980003ff908b1082070bd2a462146304600f034
:10b9900075f9002070bd2de9f0410c461746804630
:10b9a000032107f0dbfa0546204600f0e4f80446e0
:10b9b00095b10146284600f00df980b104eb8401f1
:10b9c0001c22686802ebc1014618304600f018f9e5
:10b9d00038b10820bde8f08143f20200fae7052003
:10b9e000f8e73b46324621462846fff742f8002852
:10b9f000f0d1e2b229464046fef75aff708c083873
:10ba0000082803d242484078f7f76afa0020e1e7b5
:10ba10002de9f0410d4617468046032107f09efab6
:10ba20000446284600f0a7f8064624b13846f5f744
:10ba300010fc38b902e043f20200cbe73868f5f7b2
:10ba400008fc08b11020c5e73146204600f0c2f8d6
:10ba500060b106eb86011c22606802ebc10145184b
:10ba6000284600f0cdf818b10820b3e70520b1e76b
:10ba7000b888a98a884201d90c20abe76168e88cb4
:10ba80004978b0ebc10f01d31320a3e7314620461c
:10ba900000f094f80146606808234078c20005f180
:10baa000240007f0e2f8d7e90012c0e90012f2b270
:10bab00021464046fef772fe00208be72de9f04755
:10bac0000d461f4690468146032107f047fa04467b
:10bad000284600f050f806463cb14db13846f5f71f
:10bae000fcfb50b11020bde8f08743f20200fae7fa
:10baf000606858b1a0f80c8027e03146204600f07d
:10bb000069f818b1304600f02ef828b10520eae7b0
:10bb10002c0000208062020006eb86011c22606877
:10bb200002ebc1014518284600f06af808b1082068
:10bb3000d9e7a5f80880f2b221464846fef7b8fedc
:10bb40001fb1a8896989084438800020cbe706f036
:10bb5000e4be017821f00f01491c21f0f001103101
:10bb60000170fdf75ebd20b94e48807808b1012014
:10bb70007047002070474b498988884201d10020d6
:10bb80007047402801d2402000e0403880b2704722
:10bb900010b50446402800d9ffdf2046fff7e3ff39
:10bba00010b14048808810bd4034a0b210bd40683c
:10bbb00042690078484302ebc0007047c278406891
:10bbc000037812fb03f24378406901fb032100eb89
:10bbd000c1007047c2788a4209d9406801eb8101ef
:10bbe0001c2202ebc101405c08b10120704700201b
:10bbf00070470078062801d901207047002070475f
:10bc00000078062801d00120704700207047f0b46a
:10bc100001eb81061c27446807ebc6063444049deb
:10bc200005262670e3802571f0bcfef71fba10b51b
:10bc3000418911b1fff7ddff08b1002010bd0120df
:10bc400010bd10b5c18c8278b1ebc20f04d9c18987
:10bc500011b1fff7ceff08b1002010bd012010bdcb
:10bc600010b50c4601230a22011d07f034f80078b4
:10bc70002188012282409143218010bdf0b402eb63
:10bc800082051c264c6806ebc505072363554b68e7
:10bc90001c79402c03d11a71f0bcfef791bcf0bcaa
:10bca000704700002c00002010b5eff3108000f06a
:10bcb000010472b6fc484178491c41704078012863
:10bcc00001d10af013fb002c00d162b610bd70b593
:10bcd000f54ca07848b90125a570fff7e5ff0af0fb
:10bce00016fb20b100200af0e0fa002070bd4ff0f2
:10bcf0008040e570c0f80453f7e770b5eff31080ab
:10bd000000f0010572b6e84c607800b9ffdf60789a
:10bd1000401e6070607808b90af0ecfa002d00d17e
:10bd200062b670bde04810b5817821b10021c170c4
:10bd30008170fff7e2ff002010bd10b504460af045
:10bd4000e6fad9498978084000d001202060002017
:10bd500010bd10b5fff7a8ff0af0d9fa022201239f
:10bd6000d149540728b1d1480260236103200872e9
:10bd700002e00a72c4f804330020887110bd2de976
:10bd8000f84fdff824934278817889f80420002660
:10bd900089f80510074689f806600078dff810b3c7
:10bda000354620b1012811d0022811d0ffdf0af05a
:10bdb000c0fa4ff0804498b10af0c2fab0420fd1f5
:10bdc00030460af0c1fa0028fad042e00126eee738
:10bdd000fff76aff58460168c907fcd00226e6e76c
:10bde0000120e060c4f80451b2490e600107d1f8a7
:10bdf0004412b04ac1f3423124321160ad493431aa
:10be000008604ff0020ac4f804a3a060aa480168c1
:10be1000c94341f3001101f10108016841f010012b
:10be2000016001e0f7f7e0f8d4f804010028f9d048
:10be300030460af089fa0028fad0b8f1000f04d190
:10be40009d48016821f010010160c4f808a3c4f8fe
:10be5000045199f805004e4680b1387870b90af05f
:10be600056fa80460af05cfc6ff00042b8f1000f11
:10be700002d0c6e9032001e0c6e90302dbf80000b6
:10be8000c00701d00af03ffa387810b13572bde82a
:10be9000f88f4ff01808c4f808830127a7614ff402
:10bea0002070adf8000000bfbdf80000411eadf8e5
:10beb0000010f9d2c4f80c51c4f810517a48c01dd2
:10bec0000af0c2fa3570fff744ff676179493079ab
:10bed00020310860c4f80483d9e770b5050000d1ab
:10bee000ffdf4ff080424ff0ff30c2f8080300211f
:10bef000c2f80011c2f80411c2f80c11c2f81011f6
:10bf0000694c61700af00ffa10b10120a0706070e6
:10bf100067480068c00701d00af0f5f92846bde877
:10bf200070402ce76048007a002800d0012070475c
:10bf30002de9f04f61484ff0000a85b0d0f800b00d
:10bf4000d14657465d4a5e49083211608406d4f8ee
:10bf5000080110b14ff0010801e04ff000080af0ad
:10bf600046fa78b1d4f8240100b101208246d4f811
:10bf70001c0100b101208146d4f8200108b101273d
:10bf800000e00027d4f8000100b101200490d4f8ab
:10bf9000040100b101200390d4f80c0100b101208c
:10bfa0000290d4f8100100b101203f4d0190287893
:10bfb00000260090b8f1000f04d0c4f808610120f9
:10bfc0000af073f9baf1000f04d0c4f82461092013
:10bfd0000af06bf9b9f1000f04d0c4f81c610a2013
:10bfe0000af063f927b1c4f820610b200af05df96b
:10bff0002d48c01d0af030fa00b1ffdfdff8ac8039
:10c000000498012780b1c4f80873e87818b1ee707d
:10c0100000200af04af9287a022805d10320287264
:10c020000221c8f800102761039808b1c4f8046120
:10c03000029850b1c4f80c61287a032800d0ffdfc1
:10c04000c8f800602f72fff758fe019838b1c4f8a5
:10c050001061287a012801d100f05cf8676100982e
:10c0600038b12e70287a012801d1fff772fefff750
:10c0700044fe0d48c01d0af005fa1049091dc1f81b
:10c0800000b005b0bde8f08f074810b5c01d0af03c
:10c09000e3f90549b0b1012008704ff0e021c1f883
:10c0a0000002bde81040ffe540000020340c0040d5
:10c0b0000c0400401805004010ed00e0100502409f
:10c0c00001000001087a012801d1fff742febde816
:10c0d000104024480af0d6b970b5224ce41fa0786d
:10c0e00008b90af007f901208507a861207a00261f
:10c0f000032809d1d5f80c0120b900200af024f951
:10c100000028f7d1c5f80c6126724ff0ff30c5f852
:10c11000080370bd70b5134ce41f6079f0b10128bd
:10c1200003d0a179401e814218da0af0f0f80546e2
:10c130000af0f6fa6179012902d9a179491ca171a5
:10c140000db1216900e0e168411a022902da11f11a
:10c15000020f06dc0db1206100e0e060bde8704038
:10c16000f7e570bd470000200f4a12680d498a426a
:10c170000cd118470c4a12680a4b9a4206d101b5f5
:10c180000af0a0fa0af073fdbde80140074909680a
:10c190000958084706480749054a064b70470000fa
:10c1a00000000000bebafeca5800002004000020b3
:10c1b000c8130020c8130020f8b51d46dde9064766
:10c1c0000e000ad007f00ff82346ff1dbcb231461f
:10c1d0002a46009406f01bfcf8bdd01922461946e9
:10c1e00002f023f92046f8bd70b50d460446102232
:10c1f000002102f044f9258117206081a07b40f0e6
:10c200000a00a07370bd4ff6ff720a80014602203b
:10c210000af0a2bc704700897047827bd30701d126
:10c22000920703d48089088000207047052070475a
:10c23000827b920700d581817047014600200988e2
:10c2400041f6fe52114200d00120704700b503466e
:10c25000807bc00701d0052000bd59811846fff73b
:10c26000ecffc00703d0987b40f004009873987be4
:10c2700040f001009873002000bd827b520700d57a
:10c2800009b14089704717207047827b61f3c30270
:10c29000827370472de9fc5f0e460446017896468e
:10c2a000012000fa01f14df6ff5201ea020962682d
:10c2b0004ff6ff7b1188594502d10920bde8fc9f4c
:10c2c000b9f1000f05d041f6fe55294201d00120f9
:10c2d000f4e741ea090111801d0014d000232b70fe
:10c2e00094f800c0052103221f464ff0020abcf15a
:10c2f0000e0f76d2dfe80cf0f909252f47646b7733
:10c30000479193b4d1d80420d8e7616820898b7b0a
:10c310009b0767d517284ad30b89834247d389895e
:10c32000172901d3814242d185f800a0a5f8010068
:10c330003280616888816068817b21f002018173ad
:10c34000c6e0042028702089a5f801006089a5f8be
:10c3500003003180bce0208a3188c01d1ffa80f8bc
:10c36000414524d3062028702089a5f80100608962
:10c37000a5f80300a089a5f805000721208acde9ca
:10c380000001636941e00cf0ff00082810d008208c
:10c3900028702089a5f801006089a5f80300318084
:10c3a0006a1d694604f10c0008f08ffb10b15ee0d5
:10c3b0001020ede730889df800100844308087e0b9
:10c3c0000a2028702089a5f80100328044e00c2062
:10c3d00028702089a5f801006089a5f80300318044
:10c3e0003ae082e064e02189338800eb41021ffae1
:10c3f00082f843453bd3b8f1050f38d30e222a709b
:10c400000bea4101cde90010e36860882a467146d5
:10c41000fff7d2fea6f800805ae04020287060891d
:10c420003188c01c1ffa80f8414520d32878714616
:10c4300020f03f00123028702089a5f801006089a3
:10c44000cde9000260882a46e368fff7b5fea6f84a
:10c450000080287840063bd461682089888037e0d6
:10c46000a0893288401d1ffa80f8424501d2042776
:10c470003de0162028702089a5f801006089a5f804
:10c480000300a089cde9000160882a46714623692e
:10c49000fff792fea6f80080dee718202870207ac9
:10c4a0006870a6f800a013e061680a88920401d4bd
:10c4b00005271ce0c9882289914201d0062716e091
:10c4c0001e21297030806068018821f400510180ac
:10c4d000b9f1000f0bd061887823002202200af006
:10c4e00091fa61682078887006e0338003276068dd
:10c4f000018821ea090101803846dfe62de9ff4f76
:10c5000085b01746129c0d001e461cd03078c1071e
:10c5100003d000f03f00192801d9012100e00021db
:10c520002046fff7aafea8420dd32088a0f57f4140
:10c53000ff3908d03078410601d4000605d508201f
:10c5400009b0bde8f08f0720fae700208df8000061
:10c550008df8010030786b1e00f03f0c0121a81e01
:10c560004ff0050a4ff002094ff0030b9ab2bcf1ed
:10c57000200f75d2dfe80cf08b10745e7468748c39
:10c58000749c74b574ba74c874d474e1747474f11e
:10c5900074ef74ee74ed748b052d78d18df80090e6
:10c5a000a0788df804007088adf8060030798df819
:10c5b0000100707800f03f000c2829d00adca0f1bf
:10c5c0000200092863d2dfe800f0126215621a62e5
:10c5d0001d622000122824d004dc0e281bd0102855
:10c5e000dbd11be016281fd01828d6d11fe02078f9
:10c5f000800701e020784007002848daeee0207844
:10c600000007f9e72078c006f6e720788006f3e710
:10c6100020784006f0e720780006ede72088c00586
:10c62000eae720884005e7e720880005e4e720885e
:10c63000c004e1e72078800729d5032d27d18df8a4
:10c6400000b0b6f8010081e0217849071fd5062d1a
:10c650001dd381b27078012803d0022817d102e0df
:10c66000c9e0022000e0102004228df8002072783a
:10c670008df80420801cb1fbf0f2adf8062092b2d8
:10c6800042438a4203d10397adf80890a6e079e0cf
:10c690002078000776d598b282088df800a0adf812
:10c6a0000420b0eb820f6dd10297adf8061095e033
:10c6b0002178c90666d5022d64d381b206208df893
:10c6c0000000707802285dd3b1fbf0f28df8040011
:10c6d000adf8062092b242438a4253d1adf8089099
:10c6e0007be0207880064dd5072003e020784006c7
:10c6f0007fd508208df80000a088adf80400adf8c3
:10c700000620adf8081068e02078000671d50920f1
:10c71000adf804208df80000adf8061002975de03a
:10c720002188c90565d5022d63d381b20a208df811
:10c730000000707804285cd3c6e72088400558d5ef
:10c74000012d56d10b208df80000a088adf8040013
:10c7500044e021e026e016e0ffe72088000548d508
:10c76000052d46d30c208df80000a088adf80400fc
:10c77000b6f803006d1fadf80850adf80600adf82f
:10c780000aa02ae035e02088c00432d5012d30d13e
:10c790000d208df8000021e02088800429d4b6f80f
:10c7a0000100e080a07b000723d5032d21d3307842
:10c7b00000f03f001b2818d00f208df800002088c3
:10c7c00040f40050a4f80000b6f80100adf80400f1
:10c7d000ed1eadf80650adf808b003976946059810
:10c7e000f5f794fb050008d016e00e208df8000048
:10c7f000eae7072510e008250ee0307800f03f005a
:10c800001b2809d01d2807d0022005990af0a4f999
:10c81000208800f400502080a07b400708d52046e7
:10c82000fff70bfdc00703d1a07b20f00400a0732d
:10c83000284685e61fb5022806d101208df80000a4
:10c8400088b26946f5f762fb1fbd0000f8b51d46ca
:10c85000dde906470e000ad006f0c5fc2346ff1da1
:10c86000bcb231462a46009406f0d1f8f8bdd01982
:10c870002246194601f0d9fd2046f8bd2de9ff4fab
:10c880008db09b46dde91b57ddf87ca00c46082bdc
:10c8900005d0e06901f0fef850b11020d2e0288800
:10c8a000092140f0100028808af80010022617e0c5
:10c8b000e16901208871e2694ff420519180e169ba
:10c8c0008872e06942f601010181e069002181730b
:10c8d0002888112140f0200028808af800100426c2
:10c8e00038780a900a2038704ff0020904f11800d5
:10c8f0004d460c9001f0c6fbb04681e0bbf1100f35
:10c900000ed1022d0cd0a9eb0800801c80b20221b0
:10c91000cde9001005ab52461e990d98fff796ff22
:10c92000bdf816101a98814203d9f74800790f9084
:10c9300004e003d10a9808b138702fe04ff00201eb
:10c94000cde900190df1160352461e990d98fff717
:10c950007dff1d980088401b801b83b2c6f1ff003d
:10c96000984200d203461e990ba8d9b15ff000028d
:10c97000ddf878c0cde9032009eb060189b2cde9e5
:10c9800001c10f980090bdf8161000220d9801f01b
:10c990000efc387070b1c0b2832807d0bdf8160005
:10c9a00020833ae00aeb09018a19e1e7022011b07d
:10c9b000bde8f08fbdf82c00811901f0ff08022db1
:10c9c0000dd09af80120424506d1bdf820108142d1
:10c9d00007d0b8f1ff0f04d09af801801fe08af861
:10c9e0000180c94800680178052902d1bdf81610f8
:10c9f000818009eb08001ffa80f905eb080085b279
:10ca0000dde90c1005ab0f9a01f03ffb28b91d982a
:10ca10000088411b4145bff671af022d13d0bbf119
:10ca2000100f0cd1a9eb0800801c81b20220cde9c7
:10ca3000000105ab52461e990d98fff707ff1d98a0
:10ca40000580002038700020b1e72de9f8439c46ae
:10ca5000089e13460027b26b9ab3491f8cb2f18f20
:10ca6000a1f57f45ff3d05d05518ad882944891da6
:10ca70008db200e000252919b6f83c800831414507
:10ca800020d82a44bcf8011022f8021bbcf803107d
:10ca900022f8021b984622f8024b914606f091fbc1
:10caa0004ff00c0c41464a462346cdf800c005f035
:10cab0007afff587b16b00202944a41d214408802a
:10cac00003e001e0092700e083273846bde8f8834a
:10cad00010b50b88848f9c420cd9846be0180488b5
:10cae00044b1848824f40044a41d23440b801060c6
:10caf000002010bd0a2010bd2de9f0478ab00025a6
:10cb0000904689468246adf8185007274be00598b5
:10cb100006888088000446d4a8f8006007a801951c
:10cb200000970295cde903504ff40073002231467f
:10cb3000504601f03cfb04003cd1bdf81800adf8b4
:10cb40002000059804888188b44216d10a0414d4c0
:10cb500001950295039521f400410097049541f455
:10cb6000804342882146504601f0bff804000bd1b3
:10cb70000598818841f40041818005aa08a94846aa
:10cb8000fff7a6ff0400dcd00097059802950195f9
:10cb9000039504950188bdf81c300022504601f031
:10cba000a4f80a2c06d105aa06a94846fff790ff6b
:10cbb0000400acd0adf8185004e00598818821f449
:10cbc0000041818005aa06a94846fff781ff002899
:10cbd000f3d00a2c03d020460ab0bde8f08700202d
:10cbe000fae710b50c46896b86b051b10c218df86f
:10cbf0000010a18fadf80810a16b01916946faf7fa
:10cc00001bfb00204ff6ff71a063e187a08706b0f1
:10cc100010bd2de9f0410d460746896b0020069ea8
:10cc20001446002911d0012b0fd13246294638462f
:10cc3000fff762ff002808d1002c06d032462946b3
:10cc40003846bde8f04100f034bfbde8f0812de981
:10cc5000fc411446dde9087c0e46dde90a15521d4b
:10cc6000bcf800e092b2964502d20720bde8fc81f4
:10cc7000acf8002017222a70a5f80160a5f803304f
:10cc80000522cde900423b462a46fff7dffd0020a2
:10cc9000ece770b50c46154648220021204601f00d
:10cca000eefb04f1080044f81c0f00204ff6ff7162
:10ccb000e06161842084a5841720e08494f82a0030
:10ccc00040f00a0084f82a0070bd4ff6ff720a8017
:10ccd0000146032009f040bf30b585b00c4605463b
:10cce000fff77fffa18e284629b101218df80010a2
:10ccf0006946faf7a1fa0020e0622063606305b09c
:10cd000030bdb0f8400070475c00002090f846202d
:10cd1000920703d4408808800020f4e70620f2e759
:10cd200090f846209207eed5a0f84410ebe70146b4
:10cd3000002009880a0700d5012011f0f00f01d06a
:10cd400040f00200ca0501d540f004008a0501d573
:10cd500040f008004a0501d540f010000905d2d581
:10cd600040f02000cfe700b5034690f84600c0072a
:10cd700001d0062000bda3f842101846fff7d7ffe8
:10cd800010f03e0f05d093f8460040f0040083f801
:10cd9000460013f8460f40f001001870002000bd57
:10cda00090f84620520700d511b1b0f84200aae72a
:10cdb0001720a8e710f8462f61f3c3020270a2e71c
:10cdc0002de9ff4f9bb00e00dde92b34dde929781a
:10cdd000289d24d02878c10703d000f03f001928ef
:10cde00001d9012100e000212046fff7d9ffb04220
:10cdf00015d32878410600f03f010cd41e290cd031
:10ce0000218811f47f6f0ad13a8842b1a1f57f429f
:10ce1000ff3a04d001e0122901d1000602d5042016
:10ce20001fb0c5e5fa491d984ff0000a08718df84a
:10ce300018a08df83ca00faa0a60adf81ca0adf8b0
:10ce400050a02978994601f03f02701f5b1c04f145
:10ce5000180c4ff0060e4ff0040bcdf858c01f2ae7
:10ce60007ed2dfe802f07d7d107d267dac7df47df5
:10ce7000f37df27df17df47df07d7d7def7dee7db6
:10ce80007d7d7d7ded0094f84610b5f801008907a1
:10ce900001d5032e02d08df818b01ee34ff40061c7
:10cea000adf85010608003218df83c10adf84000c3
:10ceb000d4e2052eefd1b5f801002083adf81c00b7
:10cec000b5f80310618308b1884201d9012079e1e6
:10ced0000020a07220814ff6ff702084169801f088
:10cee000d1f8052089f800000220029083460aaba1
:10cef0001d9a16991b9801f0c8f890bb9df82e005a
:10cf0000012804d0022089f80100102003e001204c
:10cf100089f8010002200590002203a90ba807f060
:10cf2000d4fde8bb9df80c00059981423dd13988bc
:10cf3000801ca1eb0b01814237db02990220cde975
:10cf400000010df12a034a4641461b98fff77efc7b
:10cf500002980bf1020b801c81b217aa029101e02a
:10cf60009ce228e003a90ba807f0affd02999df809
:10cf70000c00cde9000117ab4a4641461b98fff76c
:10cf800065fc9df80c000aab0beb00011ffa81fb5e
:10cf900002991d9a084480b2029016991b9800e0ed
:10cfa00003e001f072f80028b6d0bbf1020f02d006
:10cfb000a7f800b04fe20a208df818004be20021dc
:10cfc0000391072efff467afb5f801002083adf899
:10cfd0001c00b5f80320628300283ff477af90422d
:10cfe0003ff674af0120a072b5f805002081002043
:10cff000a073e06900f04efd78b9e1690120887105
:10d00000e2694ff420519180e1698872e16942f64a
:10d0100001000881e06900218173f01f20841e98bf
:10d02000606207206084169801f02cf8072089f8c8
:10d0300000000120049002900020adf82a0028e0b2
:10d0400019e29fe135e1e5e012e2a8e080e043e08b
:10d050000298012814d0e0698079012803d1bdf835
:10d060002800adf80e00049803abcde900b04a46a5
:10d0700041461b98fff7eafb0498001d80b204901c
:10d08000bdf82a00adf80c00adf80e00059880b28e
:10d0900002900aab1d9a16991b9800f0f6ff28b96a
:10d0a00002983988001d05908142d1d2029801284a
:10d0b00081d0e0698079012803d1bdf82800adf85e
:10d0c0000e00049803abcde900b04a4641461b98d8
:10d0d000fff7bcfb0298bde1072e02d0152e7ff4ae
:10d0e000daaeb5f801102183adf81c10b5f80320b5
:10d0f000628300293ff4eaae91423ff6e7ae012198
:10d10000a1724ff0000ba4f808b084f80eb0052e01
:10d1100007d0c0b2691de26907f0b8fc00287ff4af
:10d120004aaf4ff6ff70208401a906aa14a8cdf8d3
:10d1300000b081e885032878214600f03f031d9a5e
:10d140001b98fff79bfb8246208badf81c0082e109
:10d150000120032ec3d14021adf85010b5f80110c5
:10d160002183adf81c100aaab8f1000f00d00023eb
:10d17000cde9020304921d98cdf804800090388810
:10d180000022401e83b21b9801f011f88df81800a0
:10d1900090bb0b2089f80000bdf8280035e04ff067
:10d1a000010c052e9bd18020adf85000b5f8011080
:10d1b0002183b5f803002084adf81c10b0f5007f82
:10d1c00003d907208df8180087e140f47c422284bf
:10d1d0000ca8b8f1000f00d00023cde90330cde951
:10d1e000018c1d9800903888401e83b21b9800f077
:10d1f000deff8df8180018b18328a8d10220bfe007
:10d200000d2189f80010bdf83000401c22e100001b
:10d210005c000020032e04d248067ff53cae0020bf
:10d2200018e1b5f80110adf81c102878400602d5b9
:10d230008df83ce002e007208df83c004ff000083c
:10d240000320cde902081e9bcdf810801d980193a4
:10d25000a6f1030b00901ffa8bf342461b9800f0d7
:10d2600044fd8df818008df83c80297849060dd5cd
:10d270002088c00506d5208bbdf81c10884201d13e
:10d28000c4f8248040468df81880e3e0832801d15b
:10d290004ff0020a4ff48070adf85000bdf81c004a
:10d2a0002083a4f820b01e986062032060841321bc
:10d2b000cde0052efff4efadb5f80110adf81c1070
:10d2c000a28f6ab3a2f57f43fe3b29d008228df8d6
:10d2d0003c2000bf4ff0000b0523cde9023bddf8f9
:10d2e00078c0cdf810b01d9a80b2cdf804c040f4db
:10d2f00000430092b5f803201b9800f0f6fc8df86f
:10d300003cb04ff400718df81800adf85010832830
:10d3100010d0f8b1a18fa1f57f40fe3807d0dce036
:10d320000b228df83c204ff6fe72a287d2e7a4f8bc
:10d330003cb0d2e000942b4631461e9a1b98fff772
:10d3400084fb8df8180008b183284bd1bdf81c0070
:10d35000208353e700942b4631461e9a1b98fff713
:10d3600074fb8df81800e8bbe18fa06b0844831da7
:10d370008de888034388828801881b98fff767fc43
:10d38000824668e095f80180022e70d15fea0800bd
:10d3900002d0b8f1010f6ad109208df83c0007a82e
:10d3a00000908df840804346002221461b98fff7ed
:10d3b00030fc8df842004ff0000b8df843b050b9af
:10d3c000b8f1010f12d0b8f1000f04d1a18fa1f56f
:10d3d0007f40ff380ad0a08f40b18df83cb04ff4a9
:10d3e000806000e037e0adf850000de00fa91b9819
:10d3f000f9f722ff82468df83cb04ff48060adf81b
:10d400005000baf1020f06d0fc480068c07928b17c
:10d410008df8180027e0a4f8188044e0baf1000f56
:10d4200003d081208df818003de007a80090434606
:10d43000012221461b98fff7ecfb8df818002146ce
:10d440001b98fff7cefb9df8180020b9192189f829
:10d450000010012038809df83c0020b10fa91b98d6
:10d46000f9f7eafe8246baf1000f33d01be018e06c
:10d470008df818e031e02078000712d5012e10d188
:10d480000a208df83c00e088adf8400003201b998d
:10d4900009f062fb0820adf85000c0e648067ff5b1
:10d4a000faac4ff0040a2088bdf8501008432080e1
:10d4b000bdf8500080050bd5a18fa1f57f40fe3847
:10d4c00006d11e98e06228982063a6864ff0030ad2
:10d4d0005046a5e49df8180078b1012089f80000b5
:10d4e000297889f80110bdf81c10a9f802109df8e0
:10d4f000181089f80410052038802088bdf85010d5
:10d5000088432080e4e72de9ff4f8846087895b0ee
:10d51000012181404ff20900249c0140adf8201008
:10d520002088ddf88890a0f57f424ff0000aff3a8e
:10d5300006d039b1000705d5012019b0bde8f08f3c
:10d540000820fae7239e4ff0000b0ea886f800b0e3
:10d5500018995d460988adf83410a8498df81cb0bb
:10d56000179a0a718df838b0086098f80000012801
:10d570003bd0022809d003286fd1307820f03f003b
:10d580001d303070b8f80400e08098f800100320d7
:10d59000022904d1317821f03f011b31317094f818
:10d5a0004610090759d505abb9f1000f13d000217a
:10d5b00002aa82e80b000720cde90009bdf834007b
:10d5c000b8f80410c01e83b20022159800f0effdd9
:10d5d0000028d1d101e0f11ceae7b8f80400a6f870
:10d5e0000100bdf81400c01c04e198f805108df886
:10d5f0001c1098f80400012806d04ff4007a022885
:10d600002cd00328b8d16ce12188b8f8080011f4b7
:10d610000061adf8201020d017281cd3b4f84010ba
:10d62000814218d3b4f84410172901d3814212d192
:10d63000317821f03f01c91c3170a6f801000321a7
:10d64000adf83410a4f8440094f8460020f002002d
:10d6500084f8460065e105257ee177e1208808f140
:10d66000080700f4fe60adf8200010f0f00f1bd0aa
:10d6700010f0c00f03d03888228b9042ebd199b9bb
:10d68000b878c00710d0b9680720cde902b1cdf84d
:10d6900004b00090cdf810b0fb88ba88398815988e
:10d6a00000f023fb0028d6d12398bdf82010401ca1
:10d6b00080294ed006dc10290dd020290bd040291e
:10d6c00087d124e0b1f5807f6ed051457ed0b1f591
:10d6d000806f97d1dee0c80601d5082000e0102059
:10d6e00082460da907aa0520cde902218df8380050
:10d6f000adf83cb0cde9049608a93888cde9000121
:10d700005346072221461598fff7b8f8a8e09df880
:10d710001c2001214ff00a0a002a9bd105abb9f168
:10d72000000f00d00020cde902100720cde900094c
:10d73000bdf834000493401e83b2218b002215985b
:10d7400000f035fd8df81c000b203070bdf8140082
:10d7500020e09df81c2001214ff00c0a002a22d164
:10d7600013abb9f1000f00d00020cde90210072063
:10d77000cde900090493bdf83400228c401e83b229
:10d78000218b159800f013fd8df81c000d203070d2
:10d79000bdf84c00401cadf8340005208df8380071
:10d7a000208badf83c00bce03888218b88427ff4a8
:10d7b00052af9df81c004ff0120a00281cd1606a7d
:10d7c000a8b1b878c0073ff446af00e018e0ba68e7
:10d7d0000720cde902b2cdf804b00090cdf810b02a
:10d7e000fb88ba88159800f080fa8df81c00132089
:10d7f00030700120adf8340093e000005c000020a0
:10d800003988208b8142d2d19df81c004ff0160a36
:10d810000028a06b08d0e0b34ff6ff7000215f46f0
:10d82000adf808b0019027e068b1b978c907bed15a
:10d83000e18f0dab0844821d03968de80c024388ee
:10d840008288018809e0b878c007bcd0ba680dabff
:10d8500003968de80c02bb88fa881598fff7f7f954
:10d8600005005ed0072d72d076e0019005aa02a9ce
:10d870002046fff72df90146e28fbdf808008242ed
:10d8800001d00029f1d0e08fa16b084407800198f6
:10d89000e08746e09df81c004ff0180a40b1208b4d
:10d8a000c8b13888208321461598fff79af938e0e7
:10d8b00004f118000090237e012221461598fff7fd
:10d8c000a8f98df81c000028edd119203070012036
:10d8d000adf83400e7e7052521461598fff781f9f3
:10d8e0003ae0208800f40070adf8200050452dd1ba
:10d8f000a08fa0f57f41fe3901d006252ce0d8f895
:10d9000008004ff0160a48b1a063b8f80c10a187c0
:10d910004ff6ff71e187a0f800b002e04ff6ff700c
:10d92000a087bdf8200030f47f611ad07823002250
:10d930000320159909f066f898f8000020712088f6
:10d94000bdf82010084320800ee000e00725208865
:10d95000bdf8201088432080208810f47f6f1cd0f1
:10d960003ae02188814321809df8380020b10ea93a
:10d970001598f9f761fc05469df81c000028ebd0ce
:10d9800086f801a001203070208b70809df81c006b
:10d9900030710520adf83400dee7a18ee1b11898b2
:10d9a0000dab0088adf834002398cde90304cde930
:10d9b0000139206b0090e36a179a1598fff700fa77
:10d9c000054601208df838000ea91598f9f734fcaa
:10d9d00000b10546a4f834b094f8460040070ad5d3
:10d9e0002046fff7a4f910f03e0f04d114f8460fbb
:10d9f00020f0040020701898bdf8341001802846eb
:10da00009be500b585b0032806d102208df8000003
:10da100088b26946f9f710fc05b000bd10b5384c66
:10da20000b782268012b02d0022b2ad111e0137847
:10da30000bb1052b01d10423137023688a889a80c7
:10da40002268cb88d38022680b8913814989518150
:10da50000de08b8893802268cb88d38022680b8965
:10da600013814b8953818b899381096911612168e5
:10da7000f9f7e2fb226800210228117003d0002888
:10da800000d0812010bd832010bd806b002800d005
:10da9000012070478178012909d10088b0f5205f05
:10daa00003d042f60101884201d1002070470720cf
:10dab0007047f0b587b0002415460e460746adf80e
:10dac000184011e005980088288005980194811d70
:10dad000cde902410721049400918388428801889e
:10dae000384600f002f930b905aa06a93046fef71b
:10daf000efff0028e6d00a2800d1002007b0f0bdd3
:10db00005c00002010b58b7883b102789a4205d171
:10db10000b885bb102e08b79091d4bb18b789a427f
:10db2000f9d1b0f801300c88a342f4d1002010bd27
:10db3000812010bd072826d012b1012a27d103e089
:10db4000497801f0070102e04978c1f3c2010529d3
:10db50001dd2dfe801f00318080c12000ab10320ff
:10db600070470220704704280dd250b10de00528ff
:10db700009d2801e022808d303e0062803d0032818
:10db800003d005207047002070470f207047812088
:10db90007047c0b282060bd4000607d5fa48807ad7
:10dba0004143c01d01ebd00080b27047084670476a
:10dbb0000020704770b513880b800b781c0625d5a4
:10dbc000f14ca47a844204d843f01000087000207d
:10dbd00070bd956800f0070605ebd0052d78f5407f
:10dbe00065f304130b701378d17803f0030341ea53
:10dbf000032140f20123b1fbf3f503fb15119268f9
:10dc0000e41d00fb012000ebd40070bd906870bde6
:10dc100037b51446bdf804101180117841f00401a5
:10dc200011709df804100a061ed5d74aa368c1f3e7
:10dc30000011927a824208d8fe2811d1d21dd20852
:10dc40004942184600f01bfc0ae003ebd00200f04a
:10dc50000703012510789d40a843994008431070a0
:10dc6000207820f0100020703ebd2de9f0410746dd
:10dc7000c81c0e4620f00300b04202d08620bde84a
:10dc8000f081c14d002034462e60af802881aa72f9
:10dc9000e8801ae0e988491ce980810614d4e1781b
:10dca00000f0030041ea002040f20121b0fbf1f254
:10dcb00001fb12012068fff76cff2989084480b23c
:10dcc0002881381a3044a0600c3420784107e1d410
:10dcd0000020d4e7ac4801220189c08800eb400055
:10dce00002eb8000084480b270472de9ff4f89b0f5
:10dcf0001646dde9168a0f46994623f44045084644
:10dd000000f054fb040002d02078400703d4012027
:10dd10000db0bde8f08f099805f0e6f80290207884
:10dd2000000606d59848817a0298814201d887205a
:10dd3000eee7224601a90298fff73cff8346002048
:10dd40008df80c004046b8f1070f1ad00122214689
:10dd5000fff7f0fe0028dbd12078400611d5022025
:10dd60008df80c00adf81070bdf80400adf812008d
:10dd7000adf814601898adf81650cdf81ca0adf8a9
:10dd800018005fea094004d500252e46a846012761
:10dd90000ce02178e07801f0030140ea012040f234
:10dda0000121b0fbf1f2804601fb12875fea494096
:10ddb00009d5b84507d1a178207901f0030140eadf
:10ddc0000120b04201d3be4201d90720a0e7a81923
:10ddd0001ffa80f9b94501d90d2099e79df80c008b
:10dde00028b103a90998f9f725fa002890d1b84578
:10ddf00007d1a0784fea192161f30100a07084f8df
:10de000004901a9800b10580199850ea0a0027d0aa
:10de1000199830b10beb06002a46199900f005fb62
:10de20000ee00beb06085746189e099805f0c9f955
:10de30002b46f61db5b239464246009504f0b3fdb7
:10de4000224601a90298fff7b5fe9df8040022467c
:10de500020f010008df80400dde90110fff7d8fe76
:10de6000002055e72de9ff4fdff81c91824685b071
:10de7000b9f80610d9f8000001eb410100eb81046c
:10de800040f20120b2fbf0f1174600fb1175dde90d
:10de9000138b4e4629460698fff77bfe0346fff795
:10dea00019ff1844b1880c30884202d9842009b087
:10deb0002fe70698c6b2300603d5b00601d5062076
:10dec000f5e7b9f80620521c92b2a9f80620bbf17a
:10ded000000f01d0abf80020b00602d5c4f80880ce
:10dee0000ae0b9f808201a4492b2a9f80820d9f833
:10def0000000891a0844a0602246fe200699fff718
:10df000087fee77025712078390a61f301002a0a3b
:10df1000a17840f0040062f30101a17020709af82a
:10df200002006071baf80000e08000252573300619
:10df300002d599f80a7000e00127b00601d54ff02c
:10df400000084e4600244ff007090fe0cde90258c3
:10df50000195cdf800900495f1882046129b089a0f
:10df6000fff7c3fe0028a2d1641ce4b2bc42edd38b
:10df700000209ce700b5fff7adfe03490c308a880e
:10df8000904203d9842000bd00060020ca8808689a
:10df900002eb420300eb8300521c037823f00403de
:10dfa0000370ca80002101730846ece72de9f047b1
:10dfb000804600f0fbf9070005d000264446f74de7
:10dfc00040f2012916e00120bde8f087204600f06c
:10dfd000edf90278c17802f0030241ea0222b2fbb5
:10dfe000f9f309fb13210068fff7d3fd3044641ceb
:10dff00086b2a4b2e988601e8142e7dca8f1010084
:10e00000e8802889801b288100203870dce710b563
:10e01000144631b1491e218004f066ffa070002033
:10e0200010bd012010bd70b50446dc48c1880368ee
:10e0300001e0401c20802088884207d200eb40028b
:10e0400013eb820202d015786d07f2d580b28842b8
:10e0500016d2aab15079a072d08820819178107917
:10e0600001f0030140ea0120a081a078e11cfff744
:10e07000a1fd20612088401c2080e080002070bd30
:10e080000a2070bd0121018270472de9ff4f85b044
:10e090004ff6ff798246a3f8009048681e460d4669
:10e0a00080788df8060048680088adf804000020ec
:10e0b0008df80a00088a0c88a04200d304462c82fe
:10e0c00051e03878400708d4641c288aa4b2401c68
:10e0d000288208f10100c0b246e0288a401c28824c
:10e0e000781d6968fff70efdd8bb3188494501d11d
:10e0f000601e30803188a1eb080030806888a04223
:10e1000038d3b878397900f0030041ea002801a932
:10e11000781dfff7f7fc20bb298949452ed0002246
:10e1200039460798fff706fdd8b92989414518d126
:10e13000e9680391b5f80ac0d7f808b05046cdf8a1
:10e1400000c005f03ef8ddf800c05a460cf1070c9f
:10e150001ffa8cfc43460399cdf800c004f0edfb98
:10e1600060b1641ca4b200208046204600f01ef975
:10e170000700a6d1641e2c820a2098e67480787964
:10e18000b071f888b0803978f87801f0030140ea7e
:10e1900001207081a6f80c80504604f0a5fe3a4696
:10e1a00006f10801fff706fd306100207fe62de94a
:10e1b000ff4f87b081461c469246ddf860b0ddf81f
:10e1c0005480089800f0f2f8050002d02878400743
:10e1d00002d401200bb09ce5484604f085fe297866
:10e1e000090605d56d49897a814201d88720f1e772
:10e1f000caf309062a4601a9fff7dcfc0746149872
:10e2000007281cd000222946fff794fc0028e1d102
:10e210002878400613d501208df808000898adf83d
:10e220000c00bdf80400adf80e00adf81060adf8bc
:10e23000124002a94846f8f7fdff0028cad1297804
:10e24000e87801f0030140ea0121aa78287902f078
:10e25000030240ea0220564507d0b1f5007f04d9f9
:10e26000611e814201dd0b20b4e7864201d90720ff
:10e27000b0e7801b85b2a54200d92546bbf1000f4f
:10e2800001d0abf80050179818b1b9192a4600f020
:10e29000ccf8b8f1000f0dd03e4448464446169fd6
:10e2a00004f0a1ff2146ff1dbcb232462b4600946c
:10e2b00004f0adfb00208de72de9f04107461d4637
:10e2c0001646084600f072f8040002d02078400795
:10e2d00001d40120d3e4384604f006fe2178090673
:10e2e00005d52e49897a814201d88720c7e4224684
:10e2f0003146fff75ffc65b12178e07801f003015a
:10e3000040ea0120b0f5007f01d8012000e00020a4
:10e3100028700020b3e42de9f04107461d4616465b
:10e32000084600f043f8040002d02078400701d4ea
:10e330000120a4e4384604f0d7fd2178090605d56c
:10e340001649897a814201d8872098e422463146cd
:10e35000fff75efcff2d14d02178e07801f0030276
:10e3600040ea022040f20122b0fbf2f302fb13006c
:10e3700015b900f2012080b2e070000a60f30101db
:10e38000217000207be410b50c4600f00ff810b1ae
:10e390000178490704d4012010bd000000060020c8
:10e3a000c18821804079a0700020f5e70749ca881c
:10e3b000824209d340b1096800eb40006ff00b02c4
:10e3c00002eb8000084470470020704700060020e0
:10e3d00070b504460d4621462b460ab9002070bd93
:10e3e00001e0491c5b1c501e021e03d008781e78f9
:10e3f000b042f6d008781e78801bf0e730b50c46a6
:10e4000001462346051b954206d202e0521e9d5c42
:10e410008d54002afad107e004e01d780d70491ce4
:10e420005b1c521e002af8d130bdf0b50e460146e5
:10e43000334680ea030404f00304b4b906e002b9e9
:10e44000f0bd13f8017b01f8017b521e01f00307b8
:10e45000002ff4d10c461d4602e080cd80c4121f6f
:10e46000042afad221462b4600bf04e013f8014be0
:10e4700001f8014b521e002af8d100bfe0e7f0b5c9
:10e480000c460146e6b204e002b9f0bd01f8016baa
:10e49000521e01f00307002ff6d10b46e5b245ea04
:10e4a000052545ea054501e020c3121f042afbd2d9
:10e4b000194602e001f8016b521e002afad100bf92
:10e4c000e3e7000010b508f0f6fdf4f7edf908f009
:10e4d0003dfcbde8104008f005bd302834bf0120e8
:10e4e00000207047202834bf4ff0a0420c4a01237f
:10e4f00000f01f0003fa00f0002914bfc2f80c0559
:10e50000c2f808057047202834bf4ff0a0410449e5
:10e5100000f01f00012202fa00f0c1f81805704750
:10e520000003005070b50346002002466ff02f052f
:10e530000ee09c5ca4f130060a2e02d34ff0ff30af
:10e5400070bd00eb800005eb4000521c2044d2b2ad
:10e550008a42eed370bd30b50a230be0b0fbf3f472
:10e5600003fb1404b0fbf3f08d183034521e05f891
:10e57000014cd2b2002af1d130bd30b500234ff6a4
:10e58000ff7510e0040a44ea002084b2c85c6040d1
:10e59000c0f30314604005ea00344440e0b25b1c61
:10e5a00084ea40109bb29342ecd330bd2de9f04198
:10e5b000fe4b0026012793f864501c7893f868c03e
:10e5c000b8b183f89140a3f8921083f8902083f8b3
:10e5d0008e70bcf1000f0cbf83f8946083f89450e8
:10e5e000f3488068008804f0ecfdbde8f04104f0d9
:10e5f00081ba4ff6ff7083f89140a3f8920083f838
:10e60000902083f88e70bcf1000f14bf83f89450f3
:10e6100083f89460bde8f0812de9f041e44d29686c
:10e6200091f89c200024012a23d091f89620012af9
:10e6300030d091f86c301422dc4e0127012b32d0ff
:10e6400091f88e30012b4fd091f8a620012a1cbfe3
:10e650000020bde8f08144701f2200f8042b222224
:10e66000a731fff7e2fe286880f8a6400120bde848
:10e67000f08144701b220270d1f89d204260d1f8d5
:10e68000a120826091f8a520027381f89c400120ae
:10e69000bde8f081447007220270d1f898204260f2
:10e6a00081f89640e2e78046447000f8042b20226f
:10e6b0006e31fff7bafe88f80870286880f86c4061
:10e6c00090f86e000028d1d1b6f87000a6f8980036
:10e6d000a868417b86f89a1086f89670008804f046
:10e6e00070fd04f016fac1e791f86c30012b0bd0e5
:10e6f000447017220270d1f890204260b1f8942043
:10e70000028181f88e40b1e78046447000f8042b06
:10e7100020226e31fff789fe88f80870286880f89b
:10e720006c4090f86e000028a0d1cde7a0480068aa
:10e7300090f86c10002914bfb0f870004ff6ff700d
:10e74000704770b59a4c06462068002808bfffdf66
:10e750000025206845706660002808bfffdf20683c
:10e76000417800291cbfffdf70bdcc220021fff7dc
:10e7700086fe2068ff2101707f2180f83810132168
:10e780004184282180f86910012180f85c1080f80c
:10e79000615009f0f7f9bde8704008f004bb844906
:10e7a0000968097881420cbf012000207047804829
:10e7b000006890f82200c0f3400070477c48006871
:10e7c00090f8220000f0010070477948006890f846
:10e7d0002200c0f3001070472de9f043744803682d
:10e7e00093f82400b3f822c0c0f38001c0f34002c4
:10e7f000114400f001000a18ccf30010002460b3ab
:10e80000bcf1130f21d00bdcbcf1100f02bf694823
:10e8100030f81200bde8f083bcf1120f15d008e00b
:10e82000bcf1150f09d0bcf11d0f04bf6248bde853
:10e83000f083ffdf2046bde8f0836049002031f817
:10e84000121012fb0010bde8f0835d49002031f882
:10e85000121012fb0010bde8f08393f85e1093f8dd
:10e860005f002e264ff47a774ff014084ff04009de
:10e87000022904bf4af2d745b5fbf7f510d00129ac
:10e8800004bf4af22f75b5fbf7f510d04af62315f1
:10e89000b5fbf7f5082908bf4e4613d0042918d058
:10e8a000264608290ed0042913d0022949d004f1a4
:10e8b000280604290fd008291cbf4ff01908082189
:10e8c00004d00ae04ff0140806f5a8764ff0400196
:10e8d00003e006f5a8764ff0100118fb016111fb6b
:10e8e0000251c2eb0212374d02eb820205eb8202ab
:10e8f00011441cf0010f4ff4c8724ff4bf7504bff0
:10e90000ccf34006002e7dd0ccf3400601f5a57176
:10e91000eeb1082804bf164640270cd0042804bfd7
:10e920002e46102707d0022807bf04f11806042737
:10e9300004f12806082707eb870808eb87173e44f1
:10e940001be004f118064ff019080421c5e7082858
:10e9500004bf174640260cd0042804bf2f461026bb
:10e9600007d0022807bf04f11807042604f128077e
:10e97000082606eb861607eb8606314401f19c0655
:10e9800093f8691000f00c07002f08bf00213144f4
:10e9900018bf01f5416127d1082804bf164640275a
:10e9a0001bd0042804bf2e4610270de00c060020c3
:10e9b00064000020e46202008f891300ec62020010
:10e9c000dc620200d4feffff07d0022807bf04f17b
:10e9d0001806042704f128060827c7ebc70707eb2a
:10e9e000470706eb4706314498311cf0010f19d058
:10e9f000082808bf40200ed0042804bf2a46102053
:10ea000009d000e04ee0022807bf04f118020420fc
:10ea100004f12802082000eb400303eb001010442f
:10ea200001443be0082804bf944640260cd004284b
:10ea300004bfac46102607d0022807bf04f1180c0b
:10ea4000042604f1280c082606eb8616b3f840309d
:10ea50000ceb860c6144eb2b20d944f2552c0b3384
:10ea600003fb0cf39b0d082807d0042802d00228d2
:10ea700005d008e02a46102008e0402006e004f116
:10ea80001802042002e004f12802082000eb8010a4
:10ea900002eb800000f5a57003fb001101f5b370d7
:10eaa000bde8f08301f5a571082804bf944640260f
:10eab0000cd0042804bfac46102607d0022807bf9c
:10eac00004f1180c042604f1280c082606eb86161f
:10ead000b3f848300ceb860c6144eb2bded944f2e2
:10eae000552c0b3303fb0cf39b0d0828c5d00428d1
:10eaf000c0d00228c7d1c2e7fe4840f271210068a9
:10eb0000806a48437047fb48006890f83700002847
:10eb100018bf0120704710b5f74c207b022818bfa2
:10eb2000032808d1207d04f115010df0a2ff08286b
:10eb30001cbf012010bd207b002816bf022800202a
:10eb40000120bde8104009f037bdeb49087370475c
:10eb5000e849096881f8300070472de9f047e54c35
:10eb60002168087b002816bf022800200120487376
:10eb700001f10e0109f00afd2168087b022816bf89
:10eb800003280122002281f82f204ff0080081f88d
:10eb90002d00487b01f10e034ff001064ff00007f6
:10eba000012804bf5b7913f0c00f0ad001f10e03f6
:10ebb000012804d1587900f0c000402801d000207d
:10ebc00000e0012081f82e00002a04bf91f8220005
:10ebd00010f0040f07d0087d01f115010df049ff79
:10ebe000216881f82d002068476006f01ffb21682e
:10ebf000c14d4ff00009886095f82d000df055ffcc
:10ec0000804695f82f00002818bfb8f1000f04d0f7
:10ec100095f82d000df00efd68b195f83000002834
:10ec20001cbf95f82e0000281dd0697b05f10e0051
:10ec300001290ed012e06e734a4605f10e014046de
:10ec400009f0fafc95f82d1005f10e000ef024f8ed
:10ec500009e0407900f0c000402831d0394605f184
:10ec60000e0009f021fd2068c77690f8220010f010
:10ec7000040f08bfbde8f087002795f82d000df0c0
:10ec80008ffd050008bfbde8f08710210ef03bfda9
:10ec9000002818bfbde8f08720683a4600f11c0143
:10eca000c676284609f0c8fc206800f11c0160689f
:10ecb0000ff0e2f86068bde8f04701210ff0f7b807
:10ecc0000ef027f84a4605f10e0109f0b5fccae737
:10ecd000884a1268137b0370d2f80e000860508acd
:10ece0008880704778b584490446824e407b08731b
:10ecf0003268207810706088adf8000080b200f0b3
:10ed00000101c0f3400341ea4301c0f3800341ea3b
:10ed10008301c0f3c00341eac301c0f3001341ea19
:10ed20000311c0f3401341ea4311c0f3801041eadc
:10ed300080105084e07d012808bf012507d00228fb
:10ed400008bf022503d0032814bfffdf0825306861
:10ed500080f85e50607e012808bf012507d0022898
:10ed600008bf022503d0032814bfffdf0825316840
:10ed700081f85f5091f83500012829d0207b81f877
:10ed80002400488c1d280cbf002060688862607dcc
:10ed900081f83700a07b002816bf02280020012040
:10eda0000875d4f80f00c1f81500b4f81300a1f8e5
:10edb0001900a07e91f86b2060f3071281f86b2098
:10edc000e07e012818bf002081f83400002078bdc3
:10edd00091f85e200420082a08bf81f85e00082d03
:10ede00008bf81f85f00c9e742480068408cc0f363
:10edf000001131b1c0f38000002804bf1f2070470c
:10ee000002e0c0f3400109b10020704710f0010f8b
:10ee100014bfee20ff20704736480068408cc0f3d6
:10ee2000001119b1c0f3800028b102e0c0f3400026
:10ee300008b100207047012070472e490022096860
:10ee40004a664b8c1d2b0cbf81f8682081f8680046
:10ee500070470023274a126882f85d30d164a2f817
:10ee60005000012082f85d007047224a002312689a
:10ee700082f85c30a2f858000120516582f85c00ed
:10ee800070471c49096881f83600704719490968bc
:10ee900081f8610070471748006890f96100704779
:10eea0001448006890f82200c0f3401070471148e1
:10eeb000006890f82200c0f3c0007047012070473e
:10eec0000c48006890f85f00704770b508f044fe89
:10eed00008f023fe08f0eafc08f098fd054c2068d5
:10eee000416e491c416690f83300002558b108f086
:10eef00049fe03e0640000200c06002007f053ffe9
:10ef0000206880f833502068457090f8391021b19e
:10ef1000bde87040042009f0eebf90f86810d9b148
:10ef2000406e814218d8042009f0e5ff206890f86f
:10ef3000220010f0010f07d0a06843220188bde82d
:10ef400070400120fff732bbbde8704043224ff60e
:10ef5000ff710020fff72abbbde87040002009f0d8
:10ef6000cabf2de9f04782b00f468146fe4e4ff0f2
:10ef700000083068458c15f0030f10d015f0010f14
:10ef800005f0020005d0002808bf4ff0010806d0a8
:10ef900004e0002818bf4ff0020800d1ffdf4ff057
:10efa000000a544615f0010f05f002000dd080b99b
:10efb00015f0040f0dd04af00800002f1cbf40f0e0
:10efc000010040f002044dd09ee010b115f0040f96
:10efd0000dd015f0070f10d015f0010f05f002004d
:10efe00043d0002808bf15f0040f34d04ae0002faa
:10eff00018bf4af0090444d141e037b14af0080093
:10f00000044615f0200f1bd07ee0316805f0200289
:10f01000b1f84800104308bf4af0010474d04af028
:10f020001800044615f0200f6ed191f85e1011f013
:10f030000c0118bf0121c94361f30000044663e0dd
:10f04000316891f85e1011f00c0118bf012161f3d5
:10f050000000044658e04af00800002f18bf40f0b6
:10f06000010451d140f010044ee0002818bf15f003
:10f07000040f07d0002f18bf4af00b0444d14af008
:10f08000180441e015f0030f3dd115f0040f3ad0fc
:10f0900077b130684af0080490f85e0010f00c0177
:10f0a00018bf012161f3410415f0200f24d02be09b
:10f0b000306805f02002b0f84810114308bf4af04c
:10f0c000030421d04af0180415f0200f0ad000bf25
:10f0d00090f85e0010f00c0018bf0120c04360f3f0
:10f0e000410411e090f85e1011f00c0118bf0121ed
:10f0f000c94361f30004ebe710f00c0018bf0120d6
:10f1000060f3000400e0ffdf15f0400f1cd0cfb922
:10f110003168b1f84800002804bf488c10f0010f96
:10f120000bd110f0020f08bf10f0200f05d115f021
:10f13000010f08bf15f0020f04d091f85e0010f027
:10f140000c0f01d144f040047068a0f800a00178d1
:10f1500021f0200101704ff007010ef059fe4146e9
:10f1600070680ff04cf8214670680ff054f814f0f6
:10f17000010f0cd04ff006034ff000027b4970687e
:10f180000ff023f83068417b70680ef083fe14f0b6
:10f19000020f18d0d6e90010b9f1000f4ff00603a6
:10f1a0004ff0010207d01c310ff00ff801217068f9
:10f1b0000ef07dfe07e015310ff007f83068017d95
:10f1c00070680ef074fe14f0040f18bfffdf14f027
:10f1d000080f19d0cdf800a03068bdf80020022338
:10f1e000b0f86a1061f30b02adf8002090f86b00e4
:10f1f000032201099df8010061f307108df8010059
:10f20000694670680ef0e1ff012f62d13068b0f8f6
:10f210004810e1b390f82200c0f34000b8bb70681a
:10f220000ef0e9ff401cc7b23068c7f1ff05b0f827
:10f230004820b0f85a10511aa942b8bf0d46aa4248
:10f240003bd990f8220010f0010f36d144f01004a1
:10f25000214670680ef0dffff81cc0b2ed1e284496
:10f2600082b23068b0f86a10436ec1f30b0151faf4
:10f2700083f190f860303e4f1944bc460023e1fb17
:10f2800007c31b096ff0240c03fb0c1100e020e006
:10f2900080f8601090f85f00012101f01ef90090e5
:10f2a000bdf800009df80210032340ea01400190e0
:10f2b000042201a970680ef088ff3068aab2416c80
:10f2c00070680ef0d6ff3068b0f85a102944a0f8e4
:10f2d0005a1014f0400f06d0d6e900100123062280
:10f2e00061310ef072ff14f0200f18bfffdf002015
:10f2f000002818bfffdf02b0bde8f0872de9f0431a
:10f30000194c89b02068002808bfffdf20684178c9
:10f31000002944d10178ff2941d0002680f83160ce
:10f32000a0f85a60867080f83960304608f08efb8d
:10f33000104802ad00f1240191e80e1085e80e108e
:10f34000d0e90d10cde9061002a808f06dfb08f019
:10f3500005f8206890f9610008f0d0f8064808f038
:10f36000d3f806480ce00000640000201a060020d4
:10f3700053e4b36ed0620200d8620200d56202008c
:10f3800008f03efb606808f064fb206890f82400f9
:10f3900010f0010f07d0252008f0bef80ae009b0f0
:10f3a0000c20bde8f08310f0020f18bf262069d0b2
:10f3b00008f0b2f8206890f85e10252007f08cff66
:10f3c000206880f82c6008f03bfb206890f85e1005
:10f3d000002008f068f90f21052008f03af82068ad
:10f3e00090f82e10002901bf90f82f10002990f8f6
:10f3f000220010f0040f74d005f018ff05462068b5
:10f400002946806806f001fcdff82884074690fb57
:10f41000f8f008fb10704142284605f0eefb216829
:10f42000886097fbf8f04a68104448600df01efbb6
:10f4300001462068426891426ed8c0e90165fe4de0
:10f440004ff0010895f82d000df02ffb814695f83f
:10f450002f000127002818bfb9f1000f04d095f83c
:10f460002d000df0e7f8a0b195f8300000281cbf82
:10f4700095f82e00002824d0687b05f10e010128a4
:10f4800015d019e010f0040f14bf2720ffdf8fd133
:10f4900090e73a466f7305f10e01484609f0ccf843
:10f4a00095f82d1005f10e000df0f6fb09e04879f6
:10f4b00000f0c000402815d0414605f10e0009f0cb
:10f4c000f3f8206890f8220010f0040f24d095f88b
:10f4d0002d000df065f905001ed010210ef013f976
:10f4e00040b119e00df015fc3a4605f10e0109f0a6
:10f4f000a3f8e6e720683a4600f11c01c7762846e3
:10f5000009f09af8206800f11c0160680ef0b4fc64
:10f51000012160680ef0cbfc2068417b0e3007f0c3
:10f520007aff206890f85c1061b3b0f85810a0f82a
:10f530004810416d416490f82210c1f30011f1b9f7
:10f54000b0f86a000221c0f30b05adf80050684620
:10f5500006f0fcff28b1bdf80000c0f30b00a84284
:10f5600004d1bdf80000401cadf800002168bdf8d2
:10f570000000b1f86a2060f30b02a1f86a2020684d
:10f5800080f85c60206890f85d1039b1b0f85010d8
:10f59000a0f84010c16cc16380f85d60b0f86a10db
:10f5a000426ec1f30b0151fa82f190f86020dff84e
:10f5b0008cc2114463460022e1fb0c3212096ff049
:10f5c000240302fb031180f860100df0d2fa03212e
:10f5d00060680df051fb216881f8330009b000200c
:10f5e000bde8f0839649886070472de9f043944c5c
:10f5f00083b0226892f831303bb1508c1d2808bf8f
:10f60000ffdf03b0bde8f0435fe401260027f1b15e
:10f61000054692f8600007f07fff206890f85f10c1
:10f62000ff2007f059fe20684ff4a57190f85f2085
:10f63000002008f0fef8206890f8221011f0030f67
:10f6400000f02c81002d00f0238100f027b992f802
:10f6500022108046d07ec1f30011002956d0054605
:10f6600060680780017821f020010170518c132916
:10f6700037d01fdc102908bf022144d0122908bf4f
:10f68000062140d0ffdf6c4d606805f10e010ef0e1
:10f69000e5fb697b60680ef0fdfb2068418c1d294d
:10f6a00018bf152963d0b0f84820416c60680ef08f
:10f6b0000afc5ce0152918bf1d29e3d14ff00101b8
:10f6c0000ef0a6fb6068017841f02001017021680e
:10f6d00085b11c310ef0d0fb012160680ef0e7fb14
:10f6e000d1e700210ef094fb6068017841f0200121
:10f6f0000170c8e715310ef0bffb2068017d60681e
:10f700000ef0d5fbbfe70ef083fbbce70021fff74f
:10f7100028fc6068c17811f03f0f28d0017911f002
:10f72000100f24d00ef072fb2368024693f82410c9
:10f73000c1f38000c1f3400c604401f001010844b2
:10f7400093f82c10c1f3800cc1f34005ac4401f0d8
:10f7500001016144401ac1b293f85e0000f0bdfea1
:10f76000009003230422694660680ef02efd206895
:10f77000002590f8241090f82c0021ea000212f0e5
:10f78000010f18bf01250ed111f0020f04d010f0a7
:10f79000020f08bf022506d011f0040f03d010f0ad
:10f7a000040f08bf0425b8f1000f2bd0012d1bd08a
:10f7b000022d08bf26201bd0042d14bfffdf2720f9
:10f7c00016d0206890f85e10252007f085fd20688f
:10f7d00090f82210c1f3001169b101224ff4967123
:10f7e000002008f026f80de0252007f095fee8e758
:10f7f00007f092fee5e790f85e204ff49671002046
:10f8000008f017f8206890f82c10294380f82c1085
:10f8100090f8242032ea01011cd04670418c132953
:10f820002bd026dc102904bf03b0bde8f0831229d9
:10f8300023d007e040420f000c06002053e4b36ed3
:10f8400064000020c1f30010002818bfffdf03b0e0
:10f85000bde8f083418c1d2908bf80f82c70dcd0f6
:10f86000c1f30011002914bf80f8316080f83170b5
:10f87000d3e7152918bf1d29dbd190f85e2003b00e
:10f880004ff00101bde8f043084608f0c0b900bfe1
:10f8900090f85f200121084608f0b9f92168002d91
:10f8a000c87e7cd04a8c3d46c2f34000002808bf89
:10f8b00047f0080512f0400f18bf45f0400500283a
:10f8c00019bfd1f83c90b1f84080d1f84490b1f81c
:10f8d00048806068072107800ef09afa002160686e
:10f8e0000ef08dfc294660680ef095fc15f0080faf
:10f8f00017d02068bdf800100223b0f86a2062f328
:10f900000b01adf8001090f86b00032201099df87f
:10f91000010061f307108df80100694660680ef080
:10f9200054fc60680ef030fb2168c0f1fe00b1f8b5
:10f930005a20a8eb02018142a8bf0146cfb2d019dc
:10f94000404544d245f0100160680ef064fc6068e8
:10f950000ef01afb2168c0f1fe00b1f85a10a8ebb6
:10f9600001018142a8bf0146cfb260680ef043fc9e
:10f970003844421c2068b0f86a10436ec1f30b0192
:10f9800051fa83f190f86030fe4d1944ac460023e3
:10f99000e1fb05c34fea131c6ff0240300e03ce0d9
:10f9a0000cfb031180f8601090f85f00012100f05b
:10f9b00094fd0090bdf800009df80210032340ea7a
:10f9c00001400190042201a960680ef0fefb21684d
:10f9d00091f8220010f0400f05d00123062261317a
:10f9e00060680ef0f2fb20683a46b0f85a0000eb6f
:10f9f000090160680ef03dfc2068b0f85a103944e7
:10fa0000a0f85a1008f0d5fc002818bfffdf2068c6
:10fa10004670867003b0bde8f0830121fff7a1fabc
:10fa2000f0e7d94810b50068417841b90078ff285f
:10fa300005d000210846fff7d8fd002010bd08f0d2
:10fa40008bf808f06af807f031ff07f0dfff0c20b1
:10fa500010bd2de9f041cc4d0446174628680e46ee
:10fa600090f86c00002818bfffdf2868002f80f88e
:10fa70006e7018bfbde8f0812188a0f87010618811
:10fa8000a0f88610a188a0f88810e188a0f88a1054
:10fa900094f88c1180f88c1090f82f10002749b141
:10faa000427b00f10e01012a04d1497901f0c00125
:10fab000402935d090f8301041b1427b00f10e0161
:10fac000012a04bf497911f0c00f29d000f17a0052
:10fad00016f0e0fa6868ff2e0178c1f380116176b4
:10fae000d0f80310c4f81a10b0f80700e0832868b3
:10faf0001ed0c0f88010e18ba0f8841000f17402d1
:10fb0000511e30460cf0daff002808bfffdf2868de
:10fb100090f8731041f0020180f87310bde8f08195
:10fb2000d0f80e10c0f87a10418aa0f87e10d1e704
:10fb3000c0f88070a0f88470617e80f87310d4f8eb
:10fb40001a104167e18ba0f87810bde8f08170b51c
:10fb50008d4c0125206890f82200c0f3c00038b118
:10fb60003c22ff21a068fff774ff206880f86c50ea
:10fb7000206890f8220010f0010f1cbfa0680188d7
:10fb80004ff03c0212bf01204ff6ff710020fef73c
:10fb90000dfd206880f8395070bd7b49096881f8f7
:10fba000320070472de9f041002509f070f9002876
:10fbb00000f00a81744c2068417801270026012951
:10fbc00006d0022901d003297ed0ffdfbde8f081f5
:10fbd000817802260029418c46d0c1f34002002ad8
:10fbe00008bf11f0010f70d090f85f204ff00101b5
:10fbf0004ff0000008f00bf8216891f82200c0f3e4
:10fc00004000002814bf0c20222091f85f1007f05c
:10fc100063fb2068467090f8330058b107f0aff8e6
:10fc2000206890f85f0010f00c0f0cbf40204520ba
:10fc300007f09eff206890f83400002818bf07f0f6
:10fc4000b6ff216891f85f0091f8691010f00c0f71
:10fc500008bf0021962007f01dff08f0a1fb002837
:10fc600018bfffdfbde8f081c1f3001282b1102997
:10fc70003fd090f8330020b107f081f8402007f022
:10fc800077ff206890f8221011f0040f36d043e07f
:10fc900090f8242090f82c309a422ad1b0f84800ed
:10fca000002808bf11f0010f05d111f0020f08bfa5
:10fcb00011f0200f65d04ff001014ff00000fff769
:10fcc00094fc2068418c01e040e034e011f0010f29
:10fcd00004bfc1f34001002907d1b0f85a10b0f8b1
:10fce0004820914218bfbde8f08180f83170bde82e
:10fcf000f081bde8f0410021012076e490f8371052
:10fd0000012914bf0329102545f00e0190f85e204b
:10fd10004ff0000007f07bff206890f834000028c7
:10fd200018bf07f044ff0021962007f0b3fe2068bb
:10fd30004670bde8f081b0f85a10b0f84800814232
:10fd400042d0bde8f041012108464ee4817809b374
:10fd5000418c11f0010f22d080f86c7090f86e2069
:10fd6000b0f870100120fef721fc2068467007f003
:10fd7000f3fe07f0d2fe07f099fd07f047fe0320df
:10fd800004e021e053e4b36e64000020bde8f041dc
:10fd900009f0b1b88178bde8f041012025e411f007
:10fda000020f04bfffdfbde8f081b0f85a10b0f8d1
:10fdb0004000814208d001210846fff716fc216867
:10fdc00003204870bde8f081bde8f041fff77db841
:10fdd000fff77bb810b5fe4c206890f8341049b19d
:10fde000383007f0f3fe18b921687f2081f8380019
:10fdf00007f0d3fe206890f8330018b107f0c2fe78
:10fe000006f0d1ff09f043f8a8b1206890f822105d
:10fe1000c1f3001179b14078022818bfffdf00213b
:10fe20000120fff7e2fb2068417800291ebf4078df
:10fe30000128ffdf10bdbde81040fff746b82de9ef
:10fe4000f047e34c0f4680462168b8f1030f488c19
:10fe500008bfc0f3400508d000f0010591f832005a
:10fe6000002818bf4ff0010901d14ff0000907f039
:10fe700047fb0646b8f1030f0cbf4ff002084ff0e6
:10fe8000010835ea090008bfbde8f087206890f84e
:10fe9000330068b10cf050fe38700146ff2807d0df
:10fea0006068c01c0cf021fe38780cf052fe06434e
:10feb00060680178c1f3801221680b7d9a4208d1f5
:10fec0000622c01c1531fef783fa002808bf012066
:10fed00000d000203978ff2906d0c8b9206890f8f2
:10fee0002d00884216d113e0a0b1616811f8030b10
:10fef000c0f380100cf0bdfd05460cf01dff38b1bd
:10ff000028460cf04dfc18b110210df0fcfb08b197
:10ff1000012000e00020216891f8221011f0040f68
:10ff200001d0f0b11ae0ceb9aa4890f83700002805
:10ff300018bf404515d1616811f8030bc0f380105c
:10ff40000cf097fd04460cf0f7fe38b120460cf09b
:10ff500027fc18b110210df0d6fb10b10120bde82f
:10ff6000f0870020bde8f0872de9f04f984d04465a
:10ff700083b0286800264078022818bfffdf286871
:10ff80004ff07f0b90f8341049b1383007f01efe67
:10ff9000002804bf286880f838b007f0fefd6868c4
:10ffa0000df058ff8046002c00f0458207f04dfa16
:10ffb000002800f04082012400274ff0ff09b8f12b
:10ffc000050f1ed1686890f8240000f01f0010286b
:10ffd00017d9286890f8360098b18df800906946d6
:10ffe0000520fff72cff002800f02582286880f804
:10fff000a64069682222a730c91cfef716fa00f055
:020000040001f9
:100000001aba68680ef0b1f8002800f01482404671
:10001000dff8c0814ff0030a062880f01e82dfe877
:1000200000f0fcfcfc03fcfb8df80090694603200b
:10003000fff705ff002800f0f180296891f83400ef
:1000400010b191f89c00d8b12868817801294dd071
:100050006868042107800df0dbfe08f10e01686876
:100060000df0fcfe98f80d1068680df013ff28687d
:10007000b0f84020c16b68680df049ff00f063b92b
:100080009df8000081f89c400a7881f89d20ff28a7
:100090000fd001f19f029e310cf010fd002808bf27
:1000a000ffdf286890f89e1041f0020180f89e1052
:1000b0000de068680278c2f3801281f89e20d0f8c3
:1000c0000320c1f89f20b0f80700a1f8a30028681a
:1000d00000f1a50490f838007f2808bfffdf2868ea
:1000e00090f83810217080f838b0ade790f8220011
:1000f0000721c0f3801938480479686869f38614c9
:1001000007800df085fe002168680ef078f8214622
:1001100068680ef080f80623002208f10e01686876
:100120000ef053f82868417b68680df0b3fe6868ec
:100130000df02aff2968b1f84020c0f1fe018a4283
:10014000b8bf1146cfb2ba423cd9f81ec7b244f08c
:10015000100b594668680ef05ef868680ef04bf8b0
:10016000384400f101082868b0f86a10426ec1f303
:100170000b0151fa82f190f86020184c0a44a44611
:100180000023e2fb04c319096ff0240301fb0321e0
:1001900080f8601090f85f004246012100f09df960
:1001a0000190bdf804009df80610032340ea0140c9
:1001b0000290042202a968680ef007f859466868a0
:1001c0000ef029f8b9f1000f0fd0d5e9001007e0c3
:1001d000640000200c060020d062020053e4b36edd
:1001e0000123062261310df0f0ff28683a46c16b09
:1001f00068680ef03ef82868a0f85a70b0f8401011
:100200008f420cbf0121002180f8311008f0d1f895
:10021000002818bfffdf96e007e01ee1286880781d
:10022000002840f00a8100f006b98df80090686857
:100230000178c1f38019d0f803100191b0f80700dc
:10024000adf8080069460520fff7f9fd0028286889
:100250007dd0817800297cd090f85fb0d5e9010489
:10026000d0f80f10c4f80e10b0f813106182417d61
:100270002175817d6175b0f81710e182b0f8191011
:100280006180b0f81b10a180b0f81d10e18000f172
:100290001f0104f1080015f006ff686890f82410ab
:1002a00001f01f01217690f82400400984f88c01a8
:1002b00084f864b084f865b01bf00c0f0cbf00210b
:1002c000012104f130000ef004fa2868002290f8b1
:1002d000691084f8661090f8610084f867009df852
:1002e0000010a868fff7b5fb022008f004feb04834
:1002f0000df1040b08210468686807800df088fd83
:10030000002168680df07bff214668680df083ffcf
:100310000623002208f10e0168680df056ff2868d8
:10032000417b68680df0b6fd494668680df0bffd79
:1003300006230122594668680df047ff08f039f896
:10034000002818bfffdf286880f801a077e06de083
:10035000ffe76868d5f808804ff00109027898f83f
:100360000d10c2f34012114088f80d10d0f80f1094
:10037000c8f80e10b0f81310a8f81210417d88f8d4
:100380001410817d88f81510b0f81710a8f8161011
:10039000b0f81910a8f80210b0f81b10a8f8041053
:1003a000b0f81d10a8f8061000f11f0108f10800b0
:1003b00015f079fe686890f8241001f01f0188f8a4
:1003c000181090f824000021400988f88c0188f862
:1003d000649088f8659008f130000ef07af928688a
:1003e000002290f8691088f8661090f8610088f88b
:1003f00067009df80010a868fff72bfb286880f8bd
:100400006c4090f86e20b0f870100120fef7cef826
:100410002868477007f0a0fb07f07ffb07f046fa5b
:1004200007f0f4fa012008f066fd08e090f82200d9
:10043000c0f3001008b1012601e0fef746fd286870
:1004400090f8330018b107f09dfb06f0acfc66b1e4
:1004500000210120fff7c9f810e0286890f8220079
:10046000c0f300100028e8d0e5e72868817801296a
:1004700004d190f85f10ff2006f02eff2868417825
:10048000002919bf4178012903b0bde8f08f4078f9
:10049000032818bfffdf03b0bde8f08f70b5454cef
:1004a00006460d462068807858b106f03cfe21686b
:1004b0000346304691f85f202946bde8704009f0b8
:1004c000d1ba06f030fe21680346304691f85e202e
:1004d0002946bde8704009f0c5ba78b50c46002140
:1004e0000091082804bf4ff4c87040210dd00428a3
:1004f00004bf4ff4bf70102107d0022807bf01f1dd
:100500001800042101f128000821521d02fb0106f8
:1005100028489df80010006890f8602062f30501fb
:1005200041f040058df8005090f85f0001282ad076
:1005300002282fd004281cbf0828ffdf30d000bfbe
:1005400025f080008df80000c4eb041000eb800063
:100550004ff01e0101eb800006fb040416488442a4
:1005600028bfffdf1548a0fb0410bdf801100009eb
:1005700060f30c01adf80110bdf800009df8021009
:1005800040ea014078bd9df8020020f0e0008df8bf
:100590000200d5e79df8020020f0e000203004e0e2
:1005a0009df8020020f0e00040308df80200c7e71f
:1005b000d062020064000020c4bf030089888888dc
:1005c0000178406829b190f82c1190f88c0038b966
:1005d00001e001f0adbd19b1042901d0012070473f
:1005e0000020704770b50c460546062102f0b6fca7
:1005f000606008b1002006e00721284602f0aefc4a
:10060000606018b101202070002070bd022070bd14
:100610002de9fc470c4606466946fff7e3ff002834
:100620007dd19df8000050b1fef780f8b0427cd03b
:10063000214630460af0c8fb002873d12de00ef0a9
:1006400091f9b04271d02146304613f0b0fa00283b
:1006500068d1019d95f8f00022e0012000e0002023
:10066000804695f839004ff0010a4ff00009f0b1cb
:1006700095f83a0080071ad584f8019084f800a014
:1006800084f80490e68095f83b102172a98f61816f
:10069000e98fa18185f8399044e0019d95f82c01fe
:1006a00070350028dbd1287f0028d8d0d5e7304628
:1006b00002f099fd070000d1ffdf384601f0a7ffe7
:1006c00040b184f801900f212170e680208184f8e8
:1006d00004a027e0304602f074fd070000d1ffdfe0
:1006e000b8f1000f21d0384601f0e9ffb8b19df80c
:1006f000000038b90198d0f818014188b14201d101
:1007000080f80090304607f0bffe84f801900c217d
:10071000217084f80490e680697f217200e004e093
:1007200085f81c900120bde8fc870020fbe71cb584
:100730006946fff757ff00b1ffdf684601f004fd8f
:10074000fe4900208968a1f8f2001cbd2de9fc419a
:1007500004460e46062002f0a9fb0546072002f0db
:10076000a5fb2844c7b20025a8463e4417e02088d0
:10077000401c80b22080b04202d34046a4f80080e2
:1007800080b2b84204d3b04202d20020bde8fc815e
:100790006946fff727ff0028f8d06d1cedb2ae4286
:1007a000e5d84ff6ff7020801220efe738b54ff6fe
:1007b000ff70adf800000de00621bdf8000002f06a
:1007c000dffb04460721bdf8000002f0d9fb0cb1a5
:1007d00000b1ffdf00216846fff7b8ff0028ebd02b
:1007e00038bd70b507f0befe0bf02dffd44c4ff6b0
:1007f000ff76002526836683d2a0257001680079e4
:10080000a4f14002657042f8421fa11c1071601ce7
:1008100013f0e9fa1b2020814ff4a4716181a081bb
:10082000e181072121776177032121740422627419
:100830006082a082a4f13e00e18205704680bf483c
:100840000c300570a4f110000570468084f820502b
:1008500070bd70b5b94c16460d466060217007f04a
:10086000f9fdfff7a3fffff7bcff207810f0b5fffd
:10087000b6480ef0caf92178606813f059fa20786a
:100880000bf00af9284608f0b9feb048fdf759ff09
:10089000217860680af072fb3146207813f01efd63
:1008a000bde870400bf0cfbe10b501240ab10020a6
:1008b00010bd21b1012903d00024204610bd022122
:1008c0000df014fdf9e710b503780446002b4068dd
:1008d00013460a46014609d05ff001000df0b3f857
:1008e0006168496a884203d9012010bd0020f5e7fc
:1008f000002010bd2de9f04117468a781e4680463b
:1009000042b11546c87838b10446690706d52ab100
:10091000012104e00725f5e70724f6e70021620737
:1009200002d508b1012000e00020014206d00122da
:1009300011464046fff7c7ff98b93de051b100228c
:1009400001214046fff7bfff58b9600734d50122a7
:10095000114620e060b1012200214046fff7b3ffbd
:1009600010b10920bde8f081680725d5012206e015
:1009700068074fea44700ad5002814db00220121e1
:100980004046fff7a0ffb8b125f0040514e00028a9
:1009900012da012200214046fff795ff60b100bf47
:1009a00024f0040408e0012211464046fff78bffc3
:1009b00010b125f00405f3e73d7034700020d1e755
:1009c00070b58ab0044600886946fff70bfe002820
:1009d00006d1a08830b1012804d0022802d012200c
:1009e0000ab070bd04ab03aa21466846fff782ff38
:1009f0000500f5d19df8001001200026002901997d
:100a000006d081f8c501019991f81012b1bb2de013
:100a100081f82f01019991f8561139b9019991f88e
:100a20002e1119b9019991f8971009b13a2519e0d9
:100a30000199059681f82e01019a9df80c0082f823
:100a40003001019b9df8102083f83121a388019c7f
:100a5000a4f832318df814008df8152005aa002075
:100a60000df033f8019880f82f6126e0019991f894
:100a7000c41119b9019991f8971009b13a2519e0f3
:100a80000199059681f8c40101989df80c2080f821
:100a9000c621019b9df8100083f8c701a388019c23
:100aa000a4f8c8318df814208df8150005aa01208e
:100ab0000df00bf8019880f8c561284690e710b555
:100ac00004460020a17801b90120e2780ab940f07b
:100ad000020001f048fb002803d12046bde8104089
:100ae0006ee710bd70b5044691f8650091f8663068
:100af0000d4610f00c0f00d100232189a0880cf0c6
:100b000099ff696a814229d2401a401ca188400895
:100b1000091a8ab2a2802189081a2081668895f86c
:100b2000641010460cf064ff864200d230466080ac
:100b3000e68895f8651020890ae000007000002022
:100b400018080020ffffffff1f000000d80600204c
:100b50000cf04eff864200d23046e08070bdf0b50a
:100b600085b00d46064603a9fff73cfd00282dd1b0
:100b70009df80c0060b300220499fb20b1f84e30c0
:100b8000fb2b00d30346b1f85040fb20fb2c00d3d5
:100b90000446dff85cc59ce8811000900197cdf811
:100ba00008c0adf80230adf806406846fff79aff7e
:100bb0006e80bdf80400e880bdf808006881bdf8cb
:100bc0000200a880bdf806002881002005b0f0bd15
:100bd0000122d1e72de9f04186b00446008869463c
:100be000fff700fd002876d12189e08801f0d4fad2
:100bf000002870d1a188608801f0cefa00286ad15f
:100c00002189e08801f0bffa002864d1a1886088ba
:100c100001f0b9fa07005ed1208802a9fff79fff13
:100c200000b1ffdfbdf8101062880920914252d355
:100c3000bdf80c10e28891424dd3bdf81210bdf8fa
:100c40000e2023891144a2881a44914243d39df86f
:100c50000010019d4ff00008012640f6480041b108
:100c600085f8bb61019991f8fc1105f5dd7541b975
:100c70001ae085f82561019991f84a1105f59275f8
:100c800009b13a2724e0e18869806188e9802189f7
:100c9000814200d30146a980a188814200d2084642
:100ca0002881012201990fe0e18869806188e9804b
:100cb0002189814200d30146a980a188814200d2c6
:100cc00008462881019900222846fff70bff2e7065
:100cd00085f80180384606b044e67be770b50446e7
:100ce0000df0f6fdb0b12078182811d12079012837
:100cf0000ed1e088062102f031f9040008d02088e6
:100d000007f0c2fb2088062102f03af900b1ffdfac
:100d1000012070bdf74d28780028fad000266670b3
:100d20001420207020223146201dfdf7a8fb022050
:100d300020712e70ece710b50446fdf76dfc00281d
:100d400013d0207817280fd1207968b1e0880721c7
:100d500002f004f940b1008807f096fbe088072113
:100d600002f00ef900b1ffdf012010bd2de9f047c0
:100d70005fea000800d1ffdfde4802211a30814619
:100d8000fff7e4fc00b1ffdfda4c0620678b02f0ce
:100d90008df80546072002f089f82844c5b2681c82
:100da000c6b2608bb04203d14046fff7c4ff58b9ca
:100db000608ba84203d14046fff790ff20b9608bbb
:100dc0004146fff725fc38b1404601f0f3f9002811
:100dd000e7d10120bde8f08702214846fff7b6fcc5
:100de00010b9608bb842dcd14046bde8f04713f043
:100df000baba10b501f043f908b10c2010bd0bf0e0
:100e000076fc002010bd10b50446007818b101280a
:100e100001d0122010bd01f043f920b10bf018fef3
:100e200008b10c2010bd207801f003f9e21d04f197
:100e30001703611cbde810400bf0ffbc10b5044661
:100e400001f01df908b10c2010bd207828b101284f
:100e500003d0ff280bd0122010bd01f0eaf8611c6e
:100e60000bf005fc08b1002010bd072010bd0120cb
:100e70000bf037fcf7e710b50bf0edfd08b10020e3
:100e800010bd302010bd10b5044601f009f908b1bd
:100e90000c2010bd20460bf0d8fd002010bd10b571
:100ea00001f0fef820b10bf0d3fd08b10c2010bd0d
:100eb0000bf028fd002010bdff2181704ff6ff715f
:100ec00081808d4949680a7882718a8802814988bf
:100ed000418101214170002070477cb50025022a24
:100ee00019d015dc12f10c0f15d009dc12f1280f06
:100ef00011d012f1140f0ed012f1100f11d10ae01f
:100f000012f1080f07d012f1040f04d04ab902e021
:100f1000d31e052b05d8012806d0022808d00328a7
:100f20000ad0122528467cbd1046fdf7affff9e731
:100f300010460df065fef5e7084614466946fff7d2
:100f400051fb08b10225ede79df80000019800254e
:100f500080f86740e6e710b5134601220cf010fc5c
:100f6000002010bd10b5044611f029fa052804d060
:100f7000204610f021fc002010bd0c2010bd10b543
:100f8000044601f08df808b10c2010bd2146002068
:100f900007f0e9fa002010bd10b5044610f09bfce4
:100fa00050b108f08dfd38b1207808f033fb20787f
:100fb0000ef047f9002010bd0c2010bd10b50446fe
:100fc00001f06ef808b10c2010bd2146012007f099
:100fd000cafa002010bd38b504464ff6ff70adf8d0
:100fe0000000a079e179884216d02079fdf775fae2
:100ff00090b16079fdf771fa70b10022a0791146c5
:1010000013f098fd40b90022e079114613f092fdeb
:1010100010b9207a072801d9122038bd08f05dfdeb
:1010200060b911f0ccf948b900216846fff78efb92
:1010300020b1204606f029f9002038bd0c2038bd2b
:101040002de9fc41817805461a2925d00edc1629a8
:101050002ed2dfe801f02d2d2d2d2d212d2d2d2d22
:101060002d2d2d2d2d2d2d2d2d2121212a291fd046
:101070000bdca1f11e010c291ad2dfe801f01919cd
:101080001919191919191919190d3a3904290fd2f1
:10109000dfe801f00e020e022888b0f5706f07d26b
:1010a00001276946fff79efa20b10220bde8fc81c6
:1010b0001220fbe79df8000000f0c2ff019c10b178
:1010c00004f58a7401e004f5c8749df8000000f08e
:1010d000b7ff019e10b106f2151601e006f2911657
:1010e0006846fff76dfa08b1207838b10c20dde7cb
:1010f0000c63020018080020700000202770a878f8
:101100003070684601f020f80020cfe77cb50d462e
:101110006946fff767fa002618b12e602e7102208b
:101120007cbd9df8000000f08bff019c9df8000045
:10113000703400f085ff019884f84260816829606e
:10114000017b297194f842100029f5d100207cbd63
:1011500010b5044600f0a4ff20b10bf079fc08b1f3
:101160000c2010bd207800f064ffe279611c0bf0c8
:10117000f0fd08b1002010bd022010bd10b5886e32
:1011800060b1002241f8682f0120ca718979884036
:1011900013f0c4fc002800d01f2010bd0c2010bd8f
:1011a0001cb50c466946fff71dfa002809d19df8c9
:1011b000000000280198b0f8700000d0401c20808a
:1011c00000201cbd1cb5044600886946fff70afada
:1011d00008b102201cbd606828b1dde9000122468b
:1011e00001f03cf81cbddde90001fff7c7ff1cbda5
:1011f00070b51c460d4618b1012801d0122070bdf3
:101200001946104601f068f830b12146284601f031
:101210006df808b1002070bd302070bd70b5044677
:1012200000780e46012804d018b1022801d0032806
:1012300040d1607828b1012803d0022801d00328ca
:1012400038d1e07b10b9a078012833d1a07830f0f4
:1012500005012fd110f0050f2cd06289e188e078cc
:101260003346fff7c5ff002825d1a07805281dd1fa
:101270006589a289218920793346fff7b9ff0028c3
:1012800019d1012004eb40014a8915442218d37872
:10129000927893420ed1ca8889888a420ad1401c2a
:1012a000c0b20228eed3e088a84203d3a07b08b1e5
:1012b000072801d9122070bd002070bd10b586b07e
:1012c000044600f0d1fe10b10c2006b010bd022182
:1012d00004f10a0001f020f8a0788df80800a07849
:1012e0008df8000060788df8040020788df80300f8
:1012f000a07b8df80500e07b00b101208df8060091
:10130000a078c10717d0e07800f0faff8df801004f
:10131000e088adf80a006089adf80c00a0784007bd
:1013200016d5207900f0ecff8df802002089adf889
:101330000e00a0890ae040070ad5e07800f0e0ff3f
:101340008df80200e088adf80e006089adf810005d
:1013500002a810f0ccfa0028b7d168460df076ff4d
:10136000b3e710b504460121fff758ff002803d169
:101370002046bde81040a1e710bd0278012a01d047
:10138000bab118e042783ab1012a05d0022a12d146
:1013900089b1818879b100e059b1418849b180882b
:1013a00038b101eb8101490000eb8000b1eb002f67
:1013b00001d2002070471220704770b504460078b3
:1013c0000d46012809d010f0faff052803d010f0cf
:1013d0009ef9002800d00c2070bd0df004fe88b1ed
:1013e0000df016fe0df012ff0028f5d125b1607842
:1013f0000df0a6fe0028efd1a1886088bde87040fe
:1014000010f09bba122070bd10b504460121fff701
:10141000b4ff002804d12046bde810400121cce7ec
:1014200010bdf0b5871fdde9056540f67b44a74296
:1014300013d28f1fa74210d288420ed8b2f5fa7f7e
:101440000bd2a3f10a00241fa04206d2521c4a4329
:10145000b2eb830f01daae4201d90020f0bd0120ca
:10146000f0bd2de9fc47477a8946044617f0050f81
:101470007ed0f8087cd194f83a0008b9012f77d1d2
:101480000025a8462e46f90789f0010a19d0208abe
:10149000514600f021ffe8b36089514600f026ff75
:1014a000c0b3208a6189884262d8a18ee08dcde9df
:1014b0000001238d628ca18be08afff7b2ff48b355
:1014c0000125b8070ed504eb4500828ec18dcde90c
:1014d0000012038d428c818bc08afff7a2ffc8b136
:1014e000a8466d1c78071ed504eb45065146308a88
:1014f00000f0f2fe70b17089514600f0f7fe48b17d
:10150000308a7189884253d8b18ef08dcde90001bf
:10151000338d00e00be0728cb18bf08afff781ff16
:1015200028b12e466d1cb9f1000f03d030e03020f9
:10153000bde8fc87f80707d0780705d504eb46011e
:1015400060894989884233d1228a01211be04145c3
:1015500003d004eb4100008a024404eb4100c38a3b
:10156000868ab34224d1838b468bb34220d100e0dc
:101570001ee0438c068cb3421ad1038dc08c83428b
:1015800016d1491cc9b2a942e1d3608990420fd358
:10159000207810b101280bd102e0a0780028f9d101
:1015a000607838b1012805d0022803d0032801d083
:1015b0001220bde70020bbe7002152e70178c907f0
:1015c00002d0406812f0a3be12f070be10b50078d1
:1015d000012800d00020fdf754fc002010bd2de9ab
:1015e000f0478eb00d46aff6a422d2e90092014634
:1015f00090462846fff735ff06000cd100f034fd79
:1016000040b9fe4f387828b90df0acf9a0f57f410c
:10161000ff3903d00c200eb0bde8f087032105f19f
:10162000100000f079fef54809aa3e380990f44808
:101630000a90f248062110380b900ca801f05cfccf
:10164000040037d000210bf005fe04f130017b8a45
:10165000ba8acb830a84797c0091ba463b7cba8ae9
:10166000798a208801f036fd00b1ffdf208806f07e
:101670000aff218804f10e0000f01cfde1a004f136
:10168000120700680590032105a804f055ff00200b
:1016900005a90a5c3a54401cc0b20328f9d3a88bb0
:1016a0006080688ca080288de080687a410703d52f
:1016b00008270ae00920aee7c10701d0012704e0ae
:1016c000800701d5022700e000273a46baf8160045
:1016d000114610f0c7f90146a062204610f0d0f97b
:1016e0003a46214600200cf0d3f900b90926c34a36
:1016f00021461c3200200cf0e8f9002784f87670af
:1017000084f87770a87800f094fc6076d5f8030030
:10171000c4f81a00b5f80700e083c4f8089084f80c
:101720000c80012084f8200101468df80070684685
:1017300004f002ff9df8000000f00701c0f3c102b1
:101740001144c0f3401008448df80000401d20767d
:10175000092801d208302076012120460bf07afdbd
:1017600068780df04bfceebba9782878ea1c0df0e8
:1017700018fc48b10df04cfca9782878ea1c0df053
:10178000b9fc060002d052e0122650e0687a00f060
:1017900005010020ca0700d001208a0701d540f0ca
:1017a0000200490701d540f008000df0e3fb0600f8
:1017b0003dd1214603200df0c7fc060037d10df0c6
:1017c000ccfc060033d1697a01f005018df80810d0
:1017d000697ac90708d06889adf80a00288aadf887
:1017e0000c0000e023e00120697a8a0700d5401c44
:1017f000490707d505eb40004189adf80e10008a76
:10180000adf8100002a810f072f8064695f83a00fc
:1018100000b101200df0c0fb4eb90df0f7fc060041
:1018200005d1a98f204610f003f8060008d02088c3
:1018300006f02afe2088062101f0a2fb00b1ffdf9e
:101840003046e8e601460020c9e638b56b48007826
:1018500078b910f0b4fd052805d00df083f8a0f597
:101860007f41ff3905d0684610f0abf8040002d084
:101870000ce00c2038bd0098008806f005fe0098aa
:101880000621008801f07cfb00b1ffdf204638bd57
:101890001cb582894189cde900120389c2888188fb
:1018a0004088fff7befd08b100201cbd30201cbde4
:1018b00070b50546fff7ecff00280ed128880621f9
:1018c00001f04cfb040007d000f032fc20b1d4f84a
:1018d0001801017831b901e0022070bdd4f864111b
:1018e000097809b13a2070bd05218171d4f8181129
:1018f00000200881d4f81811a8884881d4f818115c
:10190000e8888881d4f818112889c881d4f818018a
:10191000028941898a4204d88279082a01d88a42f8
:1019200001d3122070bd29884180d4f818110220fb
:101930000870002070bd3eb504460bf0b3feb0b198
:101940002e480125a0f140024570236842f8423f2d
:1019500023790021137141706946062001f087fa4e
:1019600000b1ffdf684601f060fa10b10ee012200e
:101970003ebdbdf80440029880f82051684601f051
:1019800054fa18b9bdf80400a042f4d100203ebdbd
:1019900070b505460088062101f0e0fa040007d082
:1019a00000f0c6fb20b1d4f81811087830b901e076
:1019b000022070bdd4f86401007808b13a2070bdef
:1019c000b020005d10f0010f22d0d5f80200486071
:1019d000d5f806008860d4f8180169891022818141
:1019e000d4f8180105f10c010e3004f58c74fcf7e5
:1019f0001cfd216803200870288805e018080020d5
:101a00007c0000201122330021684880002070bd36
:101a10000c2070bd38b504460078ef284dd860889a
:101a2000adf80000009800f089fc88b361880807d1
:101a300008d4d4e9012082423fd8202a3dd3b0f512
:101a4000804f3ad8207b18b3072836d8607b28b15e
:101a5000012803d0022801d003282ed14a0703d43d
:101a6000022801d0032805d1a07b08b1012824d188
:101a7000480707d4607d28b1012803d0022801d08f
:101a800003281ad1c806e07d03d5012815d110e03e
:101a900013e0012801d003280fd1c80609d4607ec5
:101aa000012803d0022801d0032806d1a07e0f28e8
:101ab00003d8e07e18b1012801d0122038bd0020e3
:101ac00038bdf8b514460d46064608f006f808b1cc
:101ad0000c20f8bd3046fff79dff0028f9d1fdf737
:101ae000daf92870b07554b9ff208df80000694606
:101af0000020fdf7baf969460020fdf7aaf9304643
:101b0000bde8f840fdf7eeb80022dae70078c1083a
:101b100001d012207047fd4981f820000020704755
:101b200010b504460078c00704d1608810b1fdf7f5
:101b300073f980b12078618800f00102607800f0cc
:101b400021fc002806d1fdf74ff901466088884244
:101b500003d9072010bd122010bd6168fdf785f97b
:101b6000002010bd10b504460078c00704d160887d
:101b700010b1fcf71cfe70b12078618800f0010202
:101b8000607800f0fffb002804d160886168fdf7f1
:101b900060f9002010bd122010bd7cb504464078cd
:101ba0004225012808d8a078fcf7f9fd20b120785b
:101bb0001225012802d090b128467cbdfdf777f9a7
:101bc00020b1a0880028f7d08028f5d8fdf776f955
:101bd00060b160780028efd02078012808d006f0a6
:101be00075fd044607f067fc00287fd00c207cbd03
:101bf000fcf791ff10b9fdf753f990b307f06dffb3
:101c00000028f3d1fcf792fda0f57f41ff39edd11b
:101c1000fcf7a3ffa68842f210704643a079fdf7b7
:101c20000cf9fcf7cbfdf8b10022072101a801f067
:101c300063f9040058d0b6480021846020460bf0b8
:101c400016fa2046fdf7cefcb04d04f130006a8a4a
:101c5000a98ac2830184fcf7b8fd60b1e88a01213a
:101c60000de0ffe712207cbd3146002007f0d5fcd7
:101c700088b3ffdf44e0fdf723f90146e88a07f067
:101c800077fd0146a0620022204606f022fdfcf707
:101c90009cfd38b9fdf714f90246214601200bf0ee
:101ca000f7fed0b1994a21461c3201200bf00dfffe
:101cb000687c00902b7caa8a698a208801f00afa45
:101cc00000b1ffdf208806f0defb3146204607f03a
:101cd000a4fc00b1ffdf13e008e00721bdf8040019
:101ce00001f04ef900b1ffdf09207cbd44b120882e
:101cf00006f0cafb2088072101f042f900b1ffdf9e
:101d000000207cbd002148e770b50d46072101f099
:101d100025f9040003d094f8930110b10ae00220e1
:101d200070bd94f87d00142801d0152802d194f8d4
:101d3000e00108b10c2070bd1022294604f5ca70dc
:101d4000fcf773fb012084f89301002070bd10b5ef
:101d5000072101f003f918b190f8931111b107e0d0
:101d6000022010bd90f87d10142903d0152901d050
:101d70000c2010bd022180f89311002010bd2de928
:101d8000fc410c464bf68032122194421dd8e4b13e
:101d90006946fef727fc002815d19df8000000f0e9
:101da0004ff9019e9df80000703600f049f9019d41
:101db000ad1c2f882246394630460bf04ef9288854
:101dc000b842f6d10020bde8fc810846fbe77cb5af
:101dd000044600886946fef705fc002810d19df8ee
:101de000000000f02df9019d9df80000703500f015
:101df00027f90198a27890f82c10914201d10c207b
:101e00007cbd7f212972a9720021e972e17880f8f6
:101e10002d10217980f82e10a17880f82c10002048
:101e20007cbd1cb50c466946fef7dcfb00280ad1d8
:101e30009df8000000f004f9019890f88c0000b1c2
:101e40000120207000201cbd7cb50d46144669465b
:101e5000fef7c8fb002809d19df8000000f0f0f85b
:101e6000019890f82c00012801d00c207cbd9df831
:101e7000000000f0e5f8019890f87810297090f8cb
:101e80007900207000207cbd70b50d4616460721f4
:101e900001f064f818b381880124c388428804ebf8
:101ea0004104ac4217d842f210746343a410624359
:101eb000b3fbf2f2521e94b24ff4fa72944200d97c
:101ec0001446a54200d22c46491c641cb4fbf1f216
:101ed0004a43521e91b290f8cc211ab901e0022077
:101ee00070bd01843180002070bd10b50c46072103
:101ef00001f034f870b180f8ff4024b190f8fd1083
:101f000009b107f04bfc002010bd000018080020ac
:101f1000700000200220f7e7017889b1417879b19b
:101f200041881b290cd381881b2909d3c188022928
:101f300006d3f74902680a65406848650020704783
:101f40001220704710b504460ff088fd204607f0b8
